:020000040801F1
:100000005057002025020108C96F01087D650108CD
:10001000C56F01081B1A01083DAE01080000000071
:10002000000000000000000000000000AD9E01087C
:10003000EB300108000000006571010839A60108D5
:10004000FDAE01085571010831A80108458B010872
:10005000115E0108458901083D5C0108415C010809
:100060008D5C0108D95C0108DD5C0108552F010891
:10007000572F0108592F01085B2F01085D2F010838
:100080005F2F0108612F0108731401084FAD0108AB
:1000900051AD0108251A0108271A0108295D010838
:1000A00033A8010839A8010837A8010835A80108B4
:1000B0003BA801083DA801083FA801088365010885
:1000C000816501088765010885650108A79E01080B
:1000D000A99E0108DDAA0108E1AA010885AB010873
:1000E0003F5C0108158A01084DAD010847A80108C9
:1000F0004DA801084BA8010849A80108751401087A
:10010000455E0108A59E010841A80108AB9E0108B3
:10011000D9AA0108DBAA010843A8010845A80108DB
:10012000632F0108652F0108672F0108692F010857
:1001300000F002F800F067F80AA090E8000C824492
:100140008344AAF10107DA4501D100F05CF8AFF26F
:10015000090EBAE80F0013F0010F18BFFB1A43F0A5
:100160000103184758750200787502000A444FF0E1
:10017000000C10F8013B13F0070408BF10F8014B06
:100180001D1108BF10F8015B641E05D010F8016B4B
:10019000641E01F8016BF9D113F0080F1EBF10F8AF
:1001A000014BAD1C0C1B09D16D1E58BF01F801CBD2
:1001B000FAD505E014F8016B01F8016B6D1EF9D555
:1001C0009142D6D37047000000230024002500266A
:1001D000103A28BF78C1FBD8520728BF30C148BFAA
:1001E0000B607047692900F06180002070471FB5DF
:1001F0009DE8030000F0F8FC00F082FE1FBD10B582
:1002000000F0E7FE10BD00F01BFF1146FFF7EFFF07
:100210000DF0F0F901F082F803B4FFF7F0FF03BC32
:100220000BF0A6FA0348004703480449044A054B6B
:100230007047000031010108504D00205057002048
:10024000505200205052002070470FB4014610B5A4
:1002500004AA039800F0A2FB10BC5DF814FB70B573
:10026000044685690068C10601D5302600E02026D5
:10027000C00707D070BDD4E9012130469047206AFD
:10028000401C20626D1EF6D570BD70B504468569B0
:100290000078C00707D170BDD4E901212020904724
:1002A000206A401C20626D1EF6D570BD2DE9F0411C
:1002B0000646002410687529314616A510D0AFF304
:1002C0000080002802DA404213A507E031688A075F
:1002D00001D512A502E0490704D511A5012401E0CA
:1002E000AFF3008000210A2206F1240709E0B0FBE9
:1002F000F2FCB0FBF2F302FB1C00303078541846DD
:10030000491C0028F3D123462A463046BDE8F04177
:1003100000F0EBBA000000002D0000002B000000F0
:10032000200000002DE9F05F894604464FF0000AE6
:10033000DFF824B1FB44C0F820A02046E1688847DC
:1003400000287DD0252806D0D4E901219047206AD5
:10035000401C2062F1E700255F462046E16888479F
:100360002028064607DB312E05D2B81910F8200CDC
:1003700008B10543F1E7A80701D525F00405C4F845
:100380001CA00027C4F818A02A2E09D030460BF074
:10039000DDF938B304EB8708303EC8F8186019E07F
:1003A00059F8041B204604EB87029161E1688847F5
:1003B000012F064618D1E069002820DA25F0200533
:1003C0001DE0D8F8180000EB800006EB4000303844
:1003D000C8F818002046E168884706460BF0B6F9D1
:1003E0000028EED1012F0AD02E2E08D12046E16838
:1003F00088477F1C0646022F45F02005C4DBA06914
:10040000002803DA404245F00105A061E80701D069
:1004100025F01005A6B1A6F14100192802D8203612
:1004200045F400654A463146204625604D46FFF7B3
:10043000D9FE60B1012807D0ED1D25F0070000E0CE
:1004400007E000F1080978E705F1040975E730468F
:100450007AE7206ABDE8F09F6B4B02002DE9F0417E
:1004600017460D4604460646012913DD38460CF0B2
:1004700035FB411C0CD0C0B20A2804F8010B02D095
:100480006D1E012DF2DC002020703046BDE8F081A9
:10049000B44201D10020F9E7384600F091FA002873
:1004A000F1D00026EFE700002DE9F0410C460746A9
:1004B0001646104600F06EF82078611C61280AD0BC
:1004C000722802D077283CD102E00125002405E003
:1004D0000225042402E0082448F2020511F8010B69
:1004E0002B2806D0622809D011F8010C74280AD0F4
:1004F0000BE045F0030544F00204EFE745F0040586
:1005000044F00104EAE744F01004384621460BF0B9
:1005100045F9411C15D00021316171604FF4007123
:10052000F560F1617061200704D530460222002198
:1005300000F04AFA306D40F0010030653046BDE809
:10054000F0810020FBE72DE9F0410D460646104CF6
:10055000206DC10704D0410804D020F00104F7E762
:1005600022460EE0542000F06AF907000ED0206DFC
:1005700047F00101084354212065384600F0F4F8A3
:100580003A4629463046BDE8F0418DE70020D6E7DF
:10059000F04B00202DE9F04704464FF000094FF0E2
:1005A000FF37C568D4E90486A80707D0204600F0C5
:1005B000BBFA30460BF0D1F8002802DA3846BDE825
:1005C000F087280502D5404600F068F94C21204606
:1005D00000F0CAF8206D20F0010020654846EEE7E3
:1005E00010B5431C02E010F8011B71B18107FAD16C
:1005F0004FF0013202C88C1A8C4314EAC211F9D0B0
:10060000C01A0A0603D0C01E10BDC01A10BD0A04CD
:1006100001D0801E10BD0902FCD0401E10BD421E3C
:1006200012F8013F002BFBD111F8013B002B02F81F
:10063000013BF9D17047032A40F2308010F0030CDF
:1006400000F0158011F8013BBCF1020F624498BF25
:1006500011F801CB00F8013B38BF11F8013BA2F1C2
:10066000040298BF00F801CB38BF00F8013B11F03D
:10067000030300F02580083AC0F0088051F8043BDD
:10068000083A51F804CBA0E80810F5E7121D5CBF4A
:1006900051F8043B40F8043BAFF30080D20724BF7D
:1006A00011F8013B11F801CB48BF11F8012B24BF11
:1006B00000F8013B00F801CB48BF00F8012B704760
:1006C00010B5203AC0F00B80B1E81850203AA0E8ED
:1006D0001850B1E81850A0E81850BFF4F5AF5FEA21
:1006E000027C24BFB1E81850A0E8185044BF18C9D4
:1006F00018C0BDE810405FEA827C24BF51F8043B7B
:1007000040F8043B08BF7047D20728BF31F8023BCE
:1007100048BF11F8012B28BF20F8023B48BF00F862
:10072000012B70474FF000020429C0F0128010F036
:10073000030C00F01B80CCF1040CBCF1020F18BFBD
:1007400000F8012BA8BF20F8022BA1EB0C0100F050
:100750000DB85FEAC17C24BF00F8012B00F8012B23
:1007600048BF00F8012B70474FF0000200B5134658
:1007700094469646203922BFA0E80C50A0E80C50C1
:10078000B1F12001BFF4F7AF090728BFA0E80C5072
:1007900048BF0CC05DF804EB890028BF40F8042B6B
:1007A00008BF704748BF20F8022B11F0804F18BFD8
:1007B00000F8012B704700004FF0013C50F8042B6B
:1007C00051F8043B9A4221D1A2EB0C03934313EA64
:1007D000CC1317D150F8042B51F8043B9A4215D191
:1007E000A2EB0C03934313EACC130BD150F8042B68
:1007F00051F8043B9A4209D1A2EB0C03934313EA4C
:10080000CC13DBD04FF00000704700BFD01A01BA04
:10081000B1FA81F101F0180122FA01F0CB40C1F1E7
:100820002001DBB2C0B2C01A2CFA01F3D11A9143F5
:1008300011EAC311E6D1704770477047704770B531
:10084000064600F0B5F9056806F10B0020F0070434
:10085000B4429CBF002070BD2B466A68BAB11068D4
:10086000A04210D304F1080188423CBF5068586090
:1008700007D35168101941601168091B0160586065
:100880001460101D70BD13465268002AE7D121463E
:10089000284600F095F90028DED170BD70B50446F9
:1008A000051F00F085F90068002C14BF446870BD76
:1008B000002C18BFAC423CBF20466468F8D30168E6
:1008C0000A18AA4218BF456003D12A680546114498
:1008D000016028684119A1421CBF6C6070BD61684D
:1008E000696021680844286070BD2DE9F0470D4615
:1008F00099469246044600F124080168880604D50A
:10090000E06921F01001216000E00120A84201DD32
:10091000471B00E00027A1697A1902EB0900081AB9
:10092000A0612078C00602D42046FFF798FC00267C
:1009300008E0D4E901211AF806009047206A401C1B
:10094000761C20624E45F4DB2078C0060AD520468E
:10095000FFF785FC06E0D4E9012130209047206AAA
:10096000401C2062381EA7F10107F4DC07E0D4E93F
:10097000012118F805009047206A401C2062281EBB
:10098000A5F10105F3DC2046FFF77FFC2078000687
:1009900002D50220BDE8F0870120FBE7074B70B5C8
:1009A0000D467B4400F05BF90446284600F008F849
:1009B00010B14FF0FF3070BD204670BDD3C10000B4
:1009C000007B00F0800070472DE9F0410446164698
:1009D0000D464769007B80072ED038460AF0D5FEC9
:1009E00050BB3EB3012E02D0022E25D104E020469A
:1009F00000F065FA05441DE038460AF0BBFEE168E8
:100A0000002841F01001E16005DA204600F058F8B6
:100A10000120BDE8F081C9030BD56268E16A91420B
:100A200000D81146A26911442269891A814200DD69
:100A300008460544002D01DA0220EAE7E16A606811
:100A4000E268814206D29103E06203D522F40031CC
:100A500041F01002A6690027AE4213DCE16A814230
:100A600001D90B4600E0034603EB060C2369ACEB0F
:100A7000030CAC4506DD814201D98C4600E084467A
:100A80009C4505D1A760276042F02000A5620DE0DB
:100A9000AD1BE669AE1B8142A66000D90846C01AAC
:100AA000281A20605819606022F02000034908408D
:100AB000E060002084F84870ABE70000BFCFD7FFAC
:100AC000C16821F4001141F08001C1600021816002
:100AD000016070472DE9F047814614460E464FF0FD
:100AE000FF383248D5685769054209D03846A169B0
:100AF0000AF093FE002811DB2C48C0430540E56056
:100B00002B463246494638460AF095FEA16920F048
:100B10000042B21A11440028A16103D02046FFF719
:100B2000CFFF4046BDE8F08770B504460569C06A4E
:100B30006168884200D80846E16821F42011E1602C
:100B4000C90312D5A84208D02246411B2846FFF708
:100B5000C1FF10B14FF0FF3070BD0020E562C4E965
:100B60000150E06820F48030E060002070BD10B5D6
:100B70000446C06820F02000E060A16AA0698842B5
:100B80000DD02046FFF7D0FFE06820F4405040F041
:100B90001000E060A06AA0612069E062606044F239
:100BA0004001E0688843E06010BD000010000200D2
:100BB00000487047F44C00207047704770477047FA
:100BC00038B504460A4600206946AFF30080002885
:100BD00008BF38BD02460099204600F05BFA0120AC
:100BE00038BD012000F0AABBF8B5AFF30080054680
:100BF00000200C46102000BF0646A819A0420DD9BF
:100C0000324669460020AFF30080070008BF00F0BD
:100C100095FB0098A04218BF0546C419FFF7C8FF0E
:100C200005600746F01D20F007004619284600F031
:100C30000AF8B44208BFF8BDA21B31463868BDE8C7
:100C4000F84000F027BA00210160C0E901107047A8
:100C50001020704701694A1C02610878704700B58E
:100C60008FB0CDE901310021059105497944CDE9E5
:100C7000031011466846FFF755FB0FB000BD00009A
:100C8000E5FFFFFF70B50D4601461446D368506975
:100C90002A460AF0AFFD002807DA411C07D0E168B8
:100CA00020F0004041F48041E160281A70BD2046E8
:100CB000FFF706FF4FF0FF3070BDC16800220260F1
:100CC00021F4805141F0400111F4C06FC16001D0A6
:100CD0008260704702694168891AC269891A816015
:100CE00070472DE9F0470446C06840F48000E0609A
:100CF000010312D520F40020E060810606D4E26AE8
:100D000061688A4200D80A46511A216040F40010F6
:100D1000E06094F82500BDE8F08720F40010E06062
:100D2000800602D52046FFF722FFE06842F28101EB
:100D30004FF0FF390140012903D02046FFF7C0FEE4
:100D4000B6E02168002600290ADAC94340F4805041
:100D50002160C4E902606068411C61600078DAE7E4
:100D600044F2400108420CD020F4A04040F0400082
:100D70002660E06021696068401AE169401AA0605D
:100D800096E0216991B9C00310D4E069FFF757FDDF
:100D90002061B0B1E06840F4006010F4407FE06092
:100DA00002D140F48070E06020696060E068D4F8AF
:100DB00014A0C1061AD5C0030ED52046FFF7B4FE15
:100DC00014E004F1240020610120E061E06820F4D7
:100DD000407040F48060E6E721696068401AA169CC
:100DE000014450460AF019FD0028A6DBE068C00364
:100DF0002AD56168E06A884200D808462169451A08
:100E0000E069471B1BD02046D4F81880FFF78CFE02
:100E100008EB05015046C4F818800AF0FEFC0028D3
:100E20008BDBE06840F40030E060000202D5A0698E
:100E30002844A061E1692069C91B45180DE02046DE
:100E4000FFF772FEE769F5E725696168D4E90607EF
:100E5000491BE56208446560A061E06820F010006D
:100E600010F4C06FE06002D0204600F03BFAE0686A
:100E700040F48050C4E90260000205D52069E062B8
:100E800060606FF0010046E7224639462846FFF7CA
:100E9000F9FE411C0CD02918E16258B1401E2060B7
:100EA000681C6060E06840F40030E060287832E759
:100EB000484630E765602046FFF7FFFEF8E710B5CB
:100EC0000146C268900703D0900607D5886A0AE0F9
:100ED00000F0DCF801210160881E10BD8B694868B4
:100EE00018440B69C01A91F848301BB191F84910A9
:100EF000401A10BD1103FCD50028FADD401E10BDBC
:100F000010B542485421FFF72FFC41485421FFF708
:100F10002BFC40485421FFF727FC3F493B483C4A03
:100F20003F4B08603D490A603A491960531C03650C
:100F3000481C1065012008653B48344A39A17844B3
:100F4000FFF7B2FA20B9384878440A3800F0EFF9D0
:100F500037482F4A35A17844FFF7A6FA20B934481C
:100F600078440A3800F0E3F932482A4A2FA178443D
:100F7000FFF79AFA20B92F4878440A3800F0D7F9D9
:100F800040232248DC000021224600F088F920B1ED
:100F900025487844543800F0CAF91D4822464023B9
:100FA000002100F07CF920B121487844543800F049
:100FB000BEF9184822461023002100F070F90028DD
:100FC00006D01C487844BDE81040563800F0AFB950
:100FD00010BD104870B5006D20F001040B48FFF7FC
:100FE000D9FA0B48FFF7D6FA0A48FFF7D3FA09E017
:100FF000206D20F001052046FFF7CCFA2046FFF7D0
:101000004DFC2C46002CF3D170BD0000F04B0020AD
:10101000444C0020984C0020C4030020C80300204A
:10102000CC030020720000009E3701007700000012
:101030008C3701007B37010000487047EC4C0020E2
:101040007546FFF7F9FFAE4605006946534620F0A6
:101050000700854618B020B5FFF7E6F8BDE8204048
:101060004FF000064FF000074FF000084FF0000B64
:1010700021F00701AC46ACE8C009ACE8C009ACE817
:10108000C009ACE8C0098D467047000000487047B1
:10109000EC4C0020034640688C46002818BF88426C
:1010A0003CBF03464068F8D318681844884207D00C
:1010B0000CF1030020F00700001D411A521A0146EE
:1010C000081D0A60FFF7EABB2DE9F04705460C460C
:1010D000C86820F4201040F48000C860800602D563
:1010E0000846FFF744FDE06841F282014FF0FF3906
:1010F0000140022903D02046FFF7E2FCB5E000F4EE
:101100002041B1F5004F0FD1C00306D56168E06AF8
:10111000884200D80846606006E02069E0626060AE
:1011200060690AF027FBA061A0680022EEB20028E7
:101130000DDAE1688B050AD4C043A06041F4903019
:101140002260E0606068411C61600670A5E0E068B4
:101150009046226040F40050E060206968BB6069FE
:101160000AF013FB012704F12405A0B1A08910F4B3
:10117000407F08D0E069FFF762FB206118B1E068AA
:1011800040F4006016E0E7612561E06820F44070FB
:1011900040F480600EE0E069FFF751FB0028206119
:1011A000F1D0E06840F4006010F4407FE06002D1CC
:1011B00040F48070E06020696060E06825696FF04D
:1011C000010AC1051FD56168E06A884200D8084657
:1011D000411B04D022462846FFF77CFCF0BBE068A8
:1011E000010203D5E562C4E9015854E0691CE162DB
:1011F0006160E16940F48030491EC4E90210304664
:101200002E70BDE8F087010202D500F480320AE0BA
:101210006068411C61600670E0680A2E40F480300E
:10122000E06006D00022E16A6068814203D90B4683
:1012300002E00122F7E70346A7895B1B7F0503D481
:10124000E7699F4200DDE2B1814200D80146E562D4
:101250000F1AC4E90158002B09DD00E005E0224621
:1012600019462846FFF736FC08B14846C9E747B19A
:10127000A069E5626560C01BA061E06840F01000F5
:10128000E060E068000208D56168A069E562491B7A
:1012900008446560A0615046B3E73046B1E770B5D9
:1012A000C468A50713D0650211D4B2F5807F09D0B8
:1012B000B2F5007F06D0B2F5806F08D1012300F1AE
:1012C000240106E05D1E6FF07F46B54201D3012088
:1012D00070BD0161C361416024F470611143C1605C
:1012E000002070BD70B5054640F202260A4C0FE0A2
:1012F00094F85000C00708D0AC4206D0E06836EA47
:10130000000002D1204600F021F8206D20F00104F9
:10131000002CEDD170BD0000F04B002010B504464C
:10132000AFF300802046BDE81040FEF775BF10B552
:1013300000F044F8BDE8104000F03AB810B500F0F5
:1013400057F8BDE8104000F033B8000070B504460F
:10135000C068810713D0800601D5A56A04E0A169A1
:10136000606808442169451A2046FFF7DDFB00222A
:10137000064629462046FFF727FB304670BD002071
:1013800070BD70B510B1BDE87040DFE70025074CB7
:101390006E1E07E02046FFF7D9FF00B13546206DED
:1013A00020F00104002CF5D1284670BDF04B002040
:1013B000002801D00AF0DCB97047000010B50146E2
:1013C00002A000F03DF8012010BD00005349475233
:1013D000545245443A2052656469726563743A20F8
:1013E00063616E2774206F70656E3A200000000004
:1013F00010B5012805D0002103A000F021F801203C
:1014000010BD09A1F8E7000053494752544D454D1E
:101410003A204F7574206F662068656170206D6595
:101420006D6F7279000000003A2048656170206D90
:10143000656D6F727920636F727275707465640088
:1014400070B505460C460A2000E06D1C0AF006FA4D
:1014500035B128780028F8D102E0641C0AF0FEF9C2
:1014600014B120780028F8D1BDE870400A200AF0B5
:10147000F5B9704770470029816802D041F0010139
:1014800001E021F0010181607047000010B50020EB
:10149000214908600120087148714FF4602088607C
:1014A0000020C860032008741C4800F059F8072386
:1014B00001220F21194800F077F8072302220821A2
:1014C000164800F071F8072303220921134800F0A1
:1014D0006BF80121114800F02DF801210F4800F0B0
:1014E0001FF801210D48FFF7C6FF0C4800F096F8E1
:1014F00000BF0A4800F02DF80028FAD1074800F094
:101500009CF800BF054800F01DF80028FAD1012121
:10151000024800F088F810BDA40D0020002401400E
:101520000029816802D041F4807101E021F48071CA
:10153000816070474268491E22F4604242EA4131AC
:1015400041607047014600208968490700D50120A5
:101550007047014600208968090700D501207047BF
:1015600010B542680E4B0C791A400B6842EA04220F
:101570001343436082680B4B1A40D1E90243234373
:101580004C7942EA440213438360C26A097C22F424
:101590007002491EC9B242EA0151C16210BD000089
:1015A000FFFEF0FFFDF7F1FF70B5072509290AD905
:1015B000C468A1F10A0606EB4606B540AC43B34049
:1015C0001C43C46007E0046901EB4106B540AC432D
:1015D000B3401C4304611F23072A09D2446B521EE7
:1015E00002EB820293409C4391400C43446370BDE4
:1015F0000D2A09D2046BD21F02EB820293409C4356
:1016000091400C43046370BDC46A0D3A02EB820240
:1016100093409C4391400C43C46270BD816841F08B
:101620000801816070470029816802D041F4A0015F
:1016300001E021F4A00181607047816841F004015C
:101640008160704710B51848007858B301211748D9
:1016500004F08DFE30BB65211548006809F09EFD41
:1016600000241CE0002240F22551124809F007FB3B
:1016700066220F480168002001F038FC0C48006821
:1016800008F030FB01F052FC012240F225510948DC
:1016900009F0F5FA002004490870601CC4B2032C5C
:1016A000E0DB00BF10BD0000D800002000080140B2
:1016B000D400002000440040114800681149096826
:1016C0000844401C00EB40000F4901EB800080689B
:1016D000A8B10C480068042805DA0A480068401CD4
:1016E0000849086008E006480068182804DA044839
:1016F0000068401C024908600120044908707047D6
:101700000803002030010020100C00203F010020C1
:101710000C480068002808DD0A480068401E094996
:1017200008600120084908700BE00848006800289C
:1017300007DD06480068401E044908600120024990
:1017400008707047300100203F010020080300208E
:1017500000B502460B46184600F010F802EB820175
:1017600000EB410000BD0146092903DD01F137000E
:10177000C0B2704701F13000C0B2FAE7014630292B
:1017800001DB392901DD002001E001F00F00704785
:101790000149405A70470000006C0040014A8152E4
:1017A00070470000006C00402DE9F84300244EA172
:1017B0004E48FEF7C8FE4E490860084600680028FB
:1017C0007ED04FF480614B4804F0DFFD01204A4990
:1017D00008704AA146480068FEF737FD642007F00C
:1017E00053FA642190FBF1F201FB1205084607F061
:1017F0004BFA642190FBF1F090FBF1F201FB120631
:10180000084607F041FA42F2107190FBF1F73346B7
:101810003A4641A1364800950068FEF716FD474854
:1018200000683C2190FBF1F201FB1205434800687F
:1018300090FBF1F62B46324641A12D480068FEF799
:1018400004FD692007F020FA0546682007F01CFA1D
:10185000642190FBF1F6682007F016FA642190FBF2
:10186000F1F201FB120733463A463AA120480095AF
:101870000068FEF7EAFC00BF204604F01BFB804630
:10188000204605F02DFA50B1404604F0DBFD054638
:101890002B46424636A116480068FEF7D6FC04F0F7
:1018A00083FE00F05FFD611C0C46084605F032FA2D
:1018B0000028E1D030A10E480068FEF7C6FC00E029
:1018C00010E04FF4FA502E49086001E004F06CFE7D
:1018D0002B4800680028F9D10749087004480068BF
:1018E000FEF758FEBDE8F88377000000BC4D030802
:1018F000AC030020000C0140D80000202A2A204D13
:1019000069737454696D65206261636B75702066DC
:10191000696C652E0A0000002A2A2050726F6772D7
:10192000616D2056657273696F6E3A2025692E25A8
:101930003032692E253032690A0000003000002064
:101940002A2A2054696D653A20253032693A2530BB
:1019500032690A002A2A20446174653A202530320F
:10196000692D253032692D253034690A00000000C8
:1019700025693D25690A00002A2A20456E640A006F
:1019800018000020F0B506460C461746BC420BD1A5
:10199000C4EBC400104951F82000B04201D12046E8
:1019A000F0BD4FF0FF30FBE7E01900EBD0714D10B8
:1019B000C5EBC500084951F82000B04205DA3A46A7
:1019C000691C3046FFF7DEFFEAE72A46214630462B
:1019D000FFF7D8FFE4E7000058E9010810B500243C
:1019E0000FE004F29310002109F00CFB04F2C51083
:1019F000002109F007FB04F2F710002109F002FBB7
:101A0000641C322CEDD300214FF4C97009F0FAFAAE
:101A10000021662009F0F6FA10BD00BFFEE701467E
:101A200001207047704770470120704710B50121B1
:101A3000224804F09CFC00283FD10BF05FF80028FE
:101A40003BD11F49A1F804011E480AF06BFF10B9F1
:101A500007F094FC31E008F083FC002204210846E2
:101A600008F09AFC01220621042008F095FCFFF7FB
:101A70009BFE00201249A1F8040113A00AF052FFB6
:101A800090B901210A2009F0BDFA01210B2009F0CB
:101A9000B9FA01210C2009F0B5FA0222072104202D
:101AA00008F07AFC00BFFEE700210A2009F0AAFA3C
:101AB00005F0F4F901200649087010BD0008014046
:101AC000C04A0020BC4D03084D545F562A00000058
:101AD0003F0100202DE9FC5F4FF0000B3B48006800
:101AE000C0EBC0003A4951F82090484604F008FA8B
:101AF0000090484604F0A6FC0546009804F0D0F992
:101B00000746009804F0C2F98046009804F0B4F942
:101B10000190009805F0F2F88246BAF5204F3DD1C9
:101B2000642095FBF0F695FBF0F100FB115465B3D2
:101B30000D2E26D2DFE806F0250714081B091C0A23
:101B40000B1D0C1E0D0000BF00BF00BF00BF00BF7B
:101B500000BF012C01DB1F2C01DD4FF0010B13E056
:101B6000012C01DB1D2C01DD4FF0010B0CE000BF4F
:101B700000BF00BF012C01DB1E2C01DD4FF0010B6B
:101B800002E04FF0010B00BF00BFBBF1010F0ED10F
:101B900001224846019909F049FA08E0BD4201DBFB
:101BA000454504DD01224846019909F03FFA0748FE
:101BB0000068401C054908600846006805F0AAF85E
:101BC00010B1002001490860BDE8FC9F2000002002
:101BD00058E9010810B50121294804F0C8FB90BB61
:101BE000682007F051F8044640F2E63225480168C3
:101BF000204609F04FFA00BF07F0A0FB04F0D4FC28
:101C0000214800680F2190FBF1F201FB120080B91E
:101C10004FF480611D4804F0B1FB28B14FF480619E
:101C20001A4804F0B2FB04E04FF48061174804F056
:101C3000AEFB154800680028DED142F6A101642001
:101C400009F0E0F91AE0FFE700BFFFF743FF04F0F7
:101C5000ABFC4FF480610D4804F090FB28B14FF4C9
:101C600080610A4804F091FB04E04FF4806107486A
:101C700004F08DFB044800680028E6D110BD000088
:101C8000000801403000002020000020000C01402E
:101C90007047000010B503480078012801D107F013
:101CA000FFFA10BD3E0100202DE9F041064640F24A
:101CB000831006F0E9FF4FEA8008002422E0301983
:101CC00006F0E2FF07463119481C06F0DDFF054625
:101CD000AF420ADA0D480068B84206DB0B480068DC
:101CE000A84202DA3019BDE8F081AF4209DD0748A9
:101CF0000068A84203DB05480068B84201DB3019E0
:101D0000F1E7241D4445DADB0020ECE73000002039
:101D100010B50B2006F0B8FF012817D108F020FB02
:101D200003220421084608F037FB0422062110464E
:101D300008F032FB00201849086000BF07F0FEFAE7
:101D400004F032FC144800680028F7D100210B2071
:101D500009F058F90C2006F097FF012812D1002055
:101D60000AF0CCFE70B900200C49A1F804010C481F
:101D70000AF0D8FD30B905220621042008F00CFB3A
:101D800007F0FCFA00210C2009F03CF905F086F878
:101D900001200449087010BD20000020C04A002026
:101DA000BC4D03083F0100202DE9F0416B2006F0F7
:101DB0006BFF0746002482E004EBC40000EB400602
:101DC00006F16C0006F060FF0546062D75D2DFE8CF
:101DD00005F0030A131C252E204608F0E1F83C48C4
:101DE00040F8245069E000223146204608F0B2F85D
:101DF000374840F8245060E000223146204608F081
:101E000085F9334840F8245057E0002231462046F7
:101E100008F0CEF82E4840F824504EE0002231461B
:101E2000204608F019F92A4840F8245045E029488E
:101E300050F8240050B9601C06F020FC0020264910
:101E400041F824000120234941F82400601C04F0DB
:101E5000F9FE88BB1E4850F82400052820D2DFE890
:101E600000F003070D131900204608F099F817E059
:101E700001223146204608F06DF811E0012231467A
:101E8000204608F043F90BE001223146204608F0D5
:101E90008FF805E001223146204608F0DDF800BF4A
:101EA00000BF00200B4941F82400094A52F82410D1
:101EB00006F16C0009F0A6F800BF00BF641C4FF4E7
:101EC000BD7006F0E1FEA0423FF776AFBDE8F081BD
:101ED000D40E0020FC0E0020E80B002010B54FF4BB
:101EE000C27006F0D1FE04464FF4BF7006F0CCFE7F
:101EF0002049096888420BDD1E4801684FF4BF7015
:101F000009F080F81C48016840F27F1009F07AF867
:101F10004FF4C07006F0B8FE1649096888420BDA23
:101F2000144801684FF4C07009F06CF81248016859
:101F300040F2811009F066F8DCB10F480068844275
:101F400017D10C4801684FF4BF7009F05BF80A48DC
:101F5000016840F27F1009F055F8064801684FF417
:101F6000C07009F04FF80448016840F2811009F090
:101F700049F810BD340000203000002010B5614841
:101F8000046861480068844204D05F48046001200E
:101F90005E4908605B4844685D480068844204D03C
:101FA0005B480460012059490860564884685948D4
:101FB0000068844204D057480460012053490860F7
:101FC000012004F063FA044653480068844204D0B8
:101FD0005148046001204D490860022004F056FA7F
:101FE00004464E480068844204D04C4804600220F5
:101FF00046490860032004F049FA0446484800684E
:10200000844204D04648046001204049086004200E
:1020100004F03CFA044643480068844204D0414836
:1020200004600120394908603F4800680B2836D217
:10203000DFE800F0060A0E12161A1E22262B3000C8
:1020400000203A4908602EE00220384908602AE062
:1020500004203649086026E008203449086022E060
:102060001020324908601EE02020304908601AE044
:1020700040202E49086016E080202C49086012E0BC
:102080004FF48070294908600DE04FF40070274933
:10209000086008E04FF480602449086003E00020F5
:1020A0002249086000BF00BF21480068012805D10F
:1020B0001E48006880F001001C4908601D48006847
:1020C000012806D11948006840F4006017490860EB
:1020D00005E01648006820F40060144908601648BE
:1020E0000068012806D11148006840F480500F496B
:1020F000086005E00D48006820F480500B49086036
:1021000010BD0000B00B00205C000020E8020020A1
:10211000600000207C000020640000206800002097
:102120006C00002070000020740000204C00002093
:1021300078000020800000208400002010B5414875
:10214000006820B1012831D0022874D155E03E4802
:1021500000683E490968884224D04FF4BE7006F0FA
:1021600093FDB0B13A48006860B901203849086071
:1021700040F27D1006F088FD3649086001203149A3
:10218000086012E000203349086001202D490860F2
:102190000BE000202E4908602E49086001202949E3
:1021A000086002E000202A49086048E029480068E9
:1021B00010BB2548006800EB4000274951F820007B
:1021C000264908602048006800EB4000224901EBE6
:1021D00080004068224908600120224908601A48AE
:1021E000006800EB40001C4901EB80008068194941
:1021F000086002201349086021E016480068C0B951
:102200000020164908601649086001201549086039
:102210000D480068401C142190FBF1F201FB1200F4
:10222000094908600221012006F0CEFF002005497F
:10223000086004E0FFE700200249086000BF00BF1B
:1022400010BD0000D0000020C8000020CC000020FD
:102250008C00002088000020E40D002038000020C1
:102260003C000020E802002070B50025002414E0A6
:1022700004EB4400114901EB8000806801280BD178
:1022800004EB44010D4A52F8211001F2851006F0CA
:10229000FBFC012800D10125641C192CE8DB35B9B1
:1022A0000748006840F001000549086005E004485F
:1022B000006820F001000249086070BD100C002089
:1022C0004C00002010B50221234804F050F830B132
:1022D0002248006840F001002049086005E01F48DE
:1022E000006820F001001D49086004211A4804F02C
:1022F0003EF830B11948006840F002001749086004
:1023000005E01648006820F00200144908608021AA
:10231000114804F02CF830B11048006840F0040077
:102320000E49086005E00D48006820F004000B49E4
:10233000086010210A4804F01AF830B10748006814
:1023400040F008000549086005E00448006820F0F6
:1023500008000249086010BD000801405800002034
:10236000001001402DE9F84F0020009084E07148F2
:102370000068401E6F49086006F0CAFB6E4908609D
:10238000084600686D4988420EDB012000906A48CB
:102390000068401A6849086006F062FC66480068F8
:1023A00006F03EFC06F05CFC6548006820B164481D
:1023B0000068401E624908606248006820B16148B8
:1023C0000068401E5F4908605F48006820B15E48B1
:1023D0000068401E5C4908605C48006820B15B48AA
:1023E0000068401E594908605948006820B15848A3
:1023F0000068401E564908605648006820B155489C
:102400000068401E534908604FF000080CE0524835
:1024100050F8280030B1504850F82800401E4E496E
:1024200041F8280008F10108B8F10A0FEFDB4B482A
:102430000068002805DD49480068401E47490860DB
:1024400005E00A20454908600120454908604548E3
:10245000D0F800B006F05CFB3C21B0FBF1F9B9F517
:10246000B46F01DB40F29F59CB4502D03D48C0F824
:10247000009001203C4908702E48006800287FF435
:1024800076AF0098002853D0692006F0FDFB054682
:10249000E91705EB91718910A5EB810141B9642120
:1024A00095FBF1F201FB125111B14FF01D0A01E051
:1024B0004FF01C0A682006F0E7FB0646642196FBF5
:1024C000F1F496FBF1F201FB1260471C0D2C18D2BF
:1024D000DFE804F0170712081709170A0B170C1783
:1024E0000D0000BF00BF00BF00BF00BF00BF1F2F17
:1024F00001DD641C012709E0574501DD641C01274B
:1025000004E01E2F01DD641C012700BF00BF0C2C5E
:1025100004DD0124691C692008F074FD04EBC4008B
:1025200000EB041007EB80063146682008F06AFDD6
:10253000BDE8F88F04000020BC000020805101009D
:1025400028030020DC020020B0000020A4000020AE
:10255000F800002088000020E80B0020B8000020D0
:10256000E802002030000020AC00002010B5344804
:10257000046804F0010008B106F024FD04F0020034
:1025800010B106F057FD01E006F04CFD04F0040028
:1025900010B106F061FD01E006F054FD04F0080002
:1025A00010B106F06DFD01E006F060FD04F01000D2
:1025B00010B106F079FD01E006F06CFD04F020009A
:1025C00010B106F085FD01E006F078FD04F0400052
:1025D00010B106F091FD01E006F084FD04F08000EA
:1025E00010B106F09DFD01E006F090FD04F480704E
:1025F00010B106F0A9FD01E006F09CFD04F40070A6
:1026000010B106F0B5FD01E006F0A8FD04F480600D
:1026100010B106F0CFFC01E006F0C4FC04F4006049
:1026200010B106F0F5FC01E006F0E8FC04F480507F
:1026300010B106F0DBFC01E006F0D0FC10BD00009C
:102640004C0000204A4800680B287ED2DFE800F0EA
:10265000060F1A25303B46515C67720045480068FA
:1026600020F4FF7020F4C060424908606DE04148EA
:10267000006820F4FF7020F4C06040F002003D4983
:10268000086062E03B48006820F4FF7020F4C060FE
:1026900040F004003749086057E03648006820F4ED
:1026A000FF7020F4C06040F00800324908604CE040
:1026B0003048006820F4FF7020F4C06040F0100043
:1026C0002C49086041E02B48006820F4FF7020F49A
:1026D000C06040F020002749086036E025480068C7
:1026E00020F4FF7020F4C06040F0400021490860F1
:1026F0002BE02048006820F4FF7020F4C06040F018
:1027000080001C49086020E01A48006820F4FF702F
:1027100020F4C06040F480701649086015E0154848
:10272000006820F4FF7020F4C06040F4007011498C
:1027300008600AE00F48006820F4FF7020F4C060D1
:1027400040F480600B49086000BF00BF0A48006881
:1027500030B10848006840F400600649086005E0B0
:102760000448006820F400600249086070470000D7
:10277000380000204C0000208C0000200146A1F110
:102780003000C1B2092901DDC81FC1B201F00F003C
:10279000704700000021002009E0084A525C00EB6D
:1027A000800302EB4302A2F130004A1CD1B2034A7B
:1027B000525C0AB10829F0DB70470000410100209B
:1027C0002DE9F05F4FF0000900240027A046002506
:1027D0000026F7480078002877D009F041F8F5493D
:1027E00001EB0010D0F800A0504603F089FBF2493D
:1027F000086009F035F8EF4901EB0010D0F800B09F
:10280000584603F07DFB824604F078FAB0F5A04FFD
:1028100070D014DCB0F5605F6DD009DCB0F5005FFE
:102820001FD0B0F5205F38D0B0F5405F34D168E0FC
:10283000B0F5804F73D0B0F5904FF7D101E1B0F50E
:10284000304F6DD006DCB0F5084F6AD0B0F5204FA0
:10285000ECD130E2B0F5484F7ED0B0F5943FE5D1F1
:102860007EE114E0D248005D2C2803D0D048005D02
:102870002D2802D14FF0010907E0CD48005D05EB9E
:10288000850100EB4100A0F13005601CC4B2C848CE
:10289000005D08B1082CE5DB85E221E0C448005D5D
:1028A0002D2802D14FF0010918E0C148005D2C2805
:1028B00001D1012712E04FB1BD48005D06EB860152
:1028C00000EB4100A0F1300608E090E2B848005D5E
:1028D00005EB850100EB4100A0F13005601CC4B29E
:1028E000B348005D08B1082CD8DB092E04DD4FF099
:1028F000010905E0E4E03CE005EB850006EB40055E
:1029000051E223E0AA48005D2D2802D14FF00109D1
:102910001AE0A748005D2C2804D1012714E05CE0F0
:102920008CE14BE147B1A248005D06EB860100EB6C
:102930004100A0F1300607E09D48005D05EB8501F0
:1029400000EB4100A0F13005601CC4B29848005D66
:1029500008B1082CD6DB00E0FCE1632E02DD4FF06D
:10296000010905E005EBC50000EB051006EB80054D
:1029700019E220E08E48005D2D2802D14FF00109B8
:1029800017E08B48005D2C2801D1012711E047B1E9
:102990008748005D06EB860100EB4100A0F13006A0
:1029A00007E08348005D05EB850100EB4100A0F1E5
:1029B0003005601CC4B27E48005D08B1082CD9DB2C
:1029C000B6F57A7F02DB4FF0010905E005EB450023
:1029D000C0EBC51006EBC005E5E120E07448005DE2
:1029E0002D2802D14FF0010917E07148005D2C2815
:1029F00001D1012711E047B16D48005D06EB86016A
:102A000000EB4100A0F1300607E06948005D05EBEE
:102A1000850100EB4100A0F13005601CC4B26448A0
:102A2000005D08B1082CD9DB42F20F70864202DD4E
:102A30004FF0010904E040F27120684306EB0015F5
:102A4000B1E15B48007870B3594800782D282BD04D
:102A500057480078A0F130055548407800B35448F5
:102A6000407805EB850100EB4100A0F130055048AE
:102A7000807890B14E488078A0F130064C48C078FC
:102A800040B14B48C07806EB860100EB4100A0F155
:102A900030060BE04FF0010908E04FF0010905E0B6
:102AA0004FF0010902E0FFE74FF001093B2E02DD84
:102AB0004FF0010903E0C5EB051006EB800572E15C
:102AC0003B4800782D2802D14FF00108012419E07D
:102AD0003748005D2C2801D1012711E047B1344867
:102AE000005D06EB860100EB4100A0F1300607E037
:102AF0002F48005D05EB850100EB4100A0F130059A
:102B0000601CC4B22A48005D08B1082CE0DB092E25
:102B100002DD4FF0010922E0B8F1010F06D105EB0B
:102B2000850006EB4000C0F52F7505E005EB85003C
:102B300006EB400000F52F7540F27B1006F0A4F87C
:102B400068B1A5F57F7000EBC00101EB00102D21ED
:102B500001EB40005A2190FBF1F000F52F7522E1C6
:102B6000134800782D2802D14FF00108012410E00D
:102B70000F48005D2C2802D14FF0010909E00C48F4
:102B8000005D05EB850100EB4100A0F13005601C04
:102B9000C4B20748005D08B1082CE9DBB8F1010FA9
:102BA00002D1C5F52F7501E005F52F75FBE000009A
:102BB00041010020582C0020000300209948007893
:102BC0002D2802D14FF001091FE019E09548005D62
:102BD0002C2801D1012711E047B19248005D06EB96
:102BE000860100EB4100A0F1300607E08D48005D52
:102BF00005EB850100EB4100A0F13005601CC4B27B
:102C00008848005D08B1082CE0DB092E02DD4FF09A
:102C1000010912E005EB850006EB400540F27B1050
:102C200006F032F848B105EBC50000EB05102D2188
:102C300001EB40005A2190FBF1F5B4E079480078AF
:102C40002D2802D14FF00108012419E07548005DDC
:102C50002C2801D1012711E047B17248005D06EB35
:102C6000860100EB4100A0F1300607E06D48005DF1
:102C700005EB850100EB4100A0F13005601CC4B2FA
:102C80006848005D08B1082CE0DB092E02DD4FF03A
:102C900001090FE0B8F1010F06D105EB850006EB45
:102CA0004000C0F52F7505E005EB850006EB400000
:102CB00000F52F7577E05B4800782D2802D14FF0A2
:102CC000010946E0574841780078303800EB800031
:102CD00001EB4000A0F130055248C17880783038CF
:102CE00000EB800001EB4000A0F130060D2E26D253
:102CF000DFE806F0250714081B091C0A0B1D0C1E33
:102D00000D0000BF00BF00BF00BF00BF00BF012D0E
:102D100001DB1F2D01DD4FF0010913E0012D01DB67
:102D20001C2D01DD4FF001090CE000BF00BF00BF0A
:102D3000012D01DB1E2D01DD4FF0010902E04FF0F6
:102D4000010900BF00BF06EBC60000EB061005EB53
:102D5000800528E0334800782D2802D14FF0010982
:102D600020E0304800783038642148432D494978C4
:102D7000303901EB810100EB41002A498978084490
:102D8000A0F1300527480179C078303800EB800089
:102D900001EB4000A0F1300605EB4500C0EBC5108B
:102DA00006EBC00500BF00BFB9F1000F36D108F037
:102DB00057FD1D4901EB0010D0F800B0584603F054
:102DC0009FF8824603F06CF8A8420EDC08F048FD3C
:102DD000154901EB0010D0F800B0584603F090F808
:102DE000824603F053F8A84202DA4FF0010915E0D9
:102DF00008F036FD0C4901EB001001222946D0F8FD
:102E000000A0504608F012F908F02AFD064901EB2F
:102E10000010006810B9284607F014FA4846BDE8CB
:102E2000F09F000041010020582C002030B5002404
:102E3000002351E0184603F025FF01284AD1284815
:102E40000068CD214843274901EB8000143000EB96
:102E500003100568244800EB041005602048006852
:102E6000CD2148431F4901EB8000143000EB0310D3
:102E700040681D4901EB0411486019480068CD21E4
:102E80004843184901EB8000143000EB03108068C0
:102E9000154901EB0411886011480068CD214843B1
:102EA000104901EB8000143000EB0310C0680E499C
:102EB00001EB0411C8600C4800EB04100068401CD2
:102EC00030B932230121601E074A02EB00108160F5
:102ED000601CC4B2581CC3B2322BABDB30BD000047
:102EE000B80200204C5A0208582C002070B5064643
:102EF0000C46154600200C490860012006F09AFE99
:102F0000304606F0EFFE2C2006F094FE204606F038
:102F1000E9FE2C2006F08EFE284606F0E3FE022095
:102F200006F088FE70BD00000001002010B50320EF
:102F300006F080FE0548006806F060FF042006F0F9
:102F400079FE00200249087010BD00000001002039
:102F50000C010020704770477047704770477047FA
:102F6000704770477047704770470029016802D06A
:102F700041F0010101E021F0010101607047000012
:102F800010B5114800F028F81048114908601148A0
:102F90004860002088600320C8600020086180200D
:102FA0004861400088618000C861202008620002FA
:102FB000486200208862044800F07AF80121024843
:102FC000FFF7D3FF10BD0000080002404C24014071
:102FD000B80D00203C0D0020016821F001010160C6
:102FE0000021016041608160C1602D4B2C49C21AF3
:102FF0008039984243D018DC2A4BA0EB0302984258
:1030000035D00ADC284A801829D014282BD028284B
:1030100024D1486840F4706034E0142A2BD0282A68
:103020001CD1486840F470002CE02048B2F56C7F59
:103030002ED009DCB2F5627F26D0B2F5677F0DD1C4
:10304000016841F0F00108E0B2F5717F24D0B2F5DB
:10305000767F03D1016841F47021016070474868B0
:1030600040F00F000EE0486840F0F0000AE04868C9
:1030700040F4704006E0486840F4702002E0486880
:1030800040F0706048607047016841F00F01E4E76C
:10309000016841F47061E0E7016841F47041DCE7E8
:1030A0008000024044000240F8FFFDBF04040240DB
:1030B00030B5036847F6F07293430C6A8A6822437E
:1030C000D1E904452C4322438C692243CC69224335
:1030D0004C6A22438C6A22431A430260CA684260E7
:1030E0000A6882604968C16030BD7047002000E016
:1030F000401C41F288318842FADB7047002000E032
:10310000401CB0F57A7FFBDB70470000F8B5002467
:103110004748007850B104F075FA0021084603F0E2
:1031200023FA0122A521002004F00EFA00204149D3
:10313000086065E0404800683E490968084400EBC3
:1031400040003E4901EB8000806808B9012457E047
:1031500038480168891C052003F006FA34480078D5
:1031600068B30120334D00902D68354E3668B54266
:1031700001D1012500E000252B462F4D2D682D4E55
:103180003668354405EB45052C4E06EB8505AA68E7
:10319000294D2D68274E3668354405EB4505274EE9
:1031A00006EB85056968244D2D68224E3668354446
:1031B00005EB4505214E56F8250007F0E3FE1D4AB4
:1031C00012681F4B1B689A4201D1012200E00022C5
:1031D0001146194A1268174B1B681A4402EB420247
:1031E000164B03EB8202906803F0A8FE11480068BA
:1031F000401C1049086008460068052800DB0124CF
:10320000002C97D00A48007868B10A48006850B985
:10321000012C08D104210F2003F0A6F90022A621D9
:10322000104607F0FFFF002001490870F8BD0000BC
:103230003F0100200C03002008030020100C002098
:103240003001002038B53E480078002877D00020B3
:103250003B49087001222C2104F06AFA0221002067
:1032600003F082F90020374B00901B68364C24682D
:10327000234403EB4303354C04EB83039A68314B3F
:103280001B68314C2468234403EB43032F4C04EBAD
:10329000830359682B4B1B682B4C2468234403EB96
:1032A00043032A4C54F82300002307F06BFE04214B
:1032B000084603F059F90022C221104607F0B2FF78
:1032C0000521042003F050F90022C121104607F027
:1032D000A9FF0621022003F047F900228D210120D9
:1032E00005F0C4F80621122003F03EF900228E21D9
:1032F000012005F0BBF80621222003F035F9002259
:103300008F21012005F0B2F80621482003F02CF9A6
:1033100000228A21012005F0A9F80621582003F097
:1033200023F900228B21012005F0A0F80621682056
:1033300003F01AF900228C21012005F097F838BD1E
:103340003F0100200803002030010020100C002065
:103350002DE9F041FE48056840F2831005F094FC29
:1033600004464FF4C17005F08FFCFA490860022C46
:1033700015DB0120F8490860F8490860F849086041
:10338000F8490860F8490860F8490860F849086099
:10339000F8490860F8490860F849086014E000201E
:1033A000ED490860ED490860ED490860ED490860A5
:1033B000ED490860ED490860ED490860ED49086095
:1033C000ED490860ED490860032C15DB0120EC494C
:1033D0000860EC490860EC490860EC490860EC4979
:1033E0000860EC490860EC490860EC490860EC4969
:1033F0000860EC49086014E00020E1490860E149F8
:103400000860E1490860E1490860E1490860E14974
:103410000860E1490860E1490860E1490860D7496E
:103420000860042C15DB0120DF490860DF490860D3
:10343000DF490860DF490860DF490860DF4908604C
:10344000DF490860DF490860DF490860DF4908603C
:1034500014E00020D4490860D4490860D4490860C9
:10346000D4490860D4490860D4490860D449086048
:10347000D4490860D4490860D4490860052C15DB9C
:103480000120D3490860D3490860D3490860D34973
:103490000860D3490860D3490860D3490860D3491C
:1034A0000860D3490860D349086014E00020C84987
:1034B0000860C8490860C8490860C8490860C84928
:1034C0000860C8490860C8490860C8490860C84918
:1034D0000860C8490860062C15DB0120C649086051
:1034E000C6490860C6490860C6490860C649086000
:1034F000C6490860C6490860C6490860C6490860F0
:10350000C649086014E00020BB490860BB49086058
:10351000BB490860BB490860BB490860BB490860FB
:10352000BB490860BB490860BB490860BB490860EB
:103530004FF4BD7005F0A8FB0446022C03DB01200C
:10354000B749086002E00020B5490860032C03DB9E
:103550000120B449086002E00020B2490860042C50
:1035600003DB0120B049086002E00020AE4908609A
:10357000052C03DB0120AD49086002E00020AB49C7
:103580000860062C03DB0120A949086002E0002046
:10359000A7490860072C03DB0120A649086002E068
:1035A0000020A4490860082C03DB0120A249086020
:1035B00002E00020A0490860092C03DB01209F499C
:1035C000086002E000209D4908600A2C03DB01200E
:1035D0009B49086002E00020994908606C2005F0D2
:1035E00053FB012806D0022817D003281ED0052837
:1035F00040D12FE00120934908600020564908601F
:103600005F49086068490860714908607A49086044
:103610008D4908608D49086034E0012089490860BF
:10362000894908600020894908602BE0012085490C
:103630000860002048490860514908605A490860FC
:10364000634908606C4908607F49086001207F4930
:10365000086017E000207B4908603F49086048493E
:103660000860514908605A49086063490860774911
:10367000086007E0012073490860744908607249D6
:10368000086000BF00BF872005F0FEFA012806D0C1
:10369000022817D003281ED0052840D12FE0012092
:1036A0006B49086000202D490860364908603F4991
:1036B00008604849086051490860664908606649E1
:1036C000086034E001206249086062490860002017
:1036D000614908602BE001205D49086000201E4917
:1036E0000860274908603049086039490860424944
:1036F00008605849086001205749086017E0002019
:1037000053490860154908601E4908602749086048
:1037100030490860394908604F49086007E00120D6
:103720004B4908604B4908604B49086000BF00BF27
:10373000A22005F0A9FA012806D0022805D0032806
:1037400004D0052803D1B9E088E09AE0A2E0C5E002
:10375000D00200204C010020540100206C01002008
:10376000840100209C010020B4010020CC01002035
:10377000E4010020FC010020140200202C020020A3
:10378000580100207001002088010020A0010020C5
:10379000B8010020D0010020E80100200002002034
:1037A00018020020300200205C010020740100207B
:1037B0008C010020A4010020BC010020D4010020C5
:1037C000EC010020040200201C0200203402002032
:1037D000600100207801002090010020A801002055
:1037E000C0010020D8010020F001002008020020C4
:1037F0002002002038020020640100207C0100200B
:1038000094010020AC010020C4010020DC01002054
:10381000F40100200C020020240200203C020020C1
:10382000680200206C020020700200207402002058
:10383000780200207C020020800200208402002008
:103840008802002050010020400200208C0200204D
:103850006801002044020020900200200120F64967
:1038600008600020F5490860F5490860F5490860DE
:10387000F5490860F5490860F5490860F5490860B0
:1038800034E00120EC490860F14908600020F1496A
:1038900008602BE00120E84908600020E749086043
:1038A000E7490860E7490860E7490860E7490860B8
:1038B000E74908600120E749086017E00020DE4979
:1038C0000860DE490860DE490860DE490860DE49BC
:1038D0000860DE490860DF49086007E00120D6493A
:1038E0000860DB490860DB49086000BF00BFBD20FD
:1038F00005F0CAF9012806D0022817D003281ED0E7
:10390000052840D12FE00120D34908600020D34989
:103910000860D3490860D3490860D3490860D34997
:103920000860D3490860D349086034E00120CA49DF
:103930000860CF4908600020CE4908602BE00120D4
:10394000C54908600020C5490860C5490860C549E7
:103950000860C5490860C5490860C549086001207C
:10396000C449086017E00020BB490860BB490860F3
:10397000BB490860BB490860BB490860BB49086097
:10398000BC49086007E00120B3490860B8490860F5
:10399000B849086000BF00BFD82005F075F90128BC
:1039A00006D0022817D003281ED0052840D12FE0CA
:1039B0000120B14908600020B0490860B0490860A2
:1039C000B0490860B0490860B0490860B049086073
:1039D000B049086034E00120A7490860AC4908609C
:1039E0000020AC4908602BE00120A34908600020BA
:1039F000A2490860A2490860A2490860A24908607B
:103A0000A2490860A24908600120A249086017E0A5
:103A100000209949086099490860994908609949C6
:103A2000086099490860994908609A49086007E068
:103A3000012091490860964908609649086000BFD6
:103A400000BFF32005F020F9012806D0022817D086
:103A500003281ED0052840D12FE001208E490860A0
:103A600000208E4908608E4908608E4908608E49A2
:103A700008608E4908608E4908608E49086034E00D
:103A80000120854908608A4908600020894908604A
:103A90002BE00120804908600020804908608049AF
:103AA0000860804908608049086080490860804952
:103AB000086001207F49086017E00020764908600F
:103AC000764908607649086076490860764908605A
:103AD000764908607749086007E001206E49086070
:103AE000734908607349086000BF00BF4FF48770D6
:103AF00005F0CAF8012806D002280DD0032820D0EE
:103B0000052842D131E001206B49086000206B4953
:103B100008606B49086040E00120674908600020A8
:103B20006849086068490860684908606849086031
:103B30006849086001206149086000206049086008
:103B40002BE001205C49086000205E4908605E4966
:103B500008605E4908605E4908605E490860574930
:103B6000086001205649086017E0002052490860AB
:103B70005449086054490860544908605449086031
:103B8000544908604E49086007E001204A4908602E
:103B90004A4908604A49086000BF00BF40F2291046
:103BA00005F072F8012806D0022817D003281ED08D
:103BB000052840D12FE001204749086000204749EF
:103BC0000860474908604749086047490860474915
:103BD0000860474908604749086095E001203E4970
:103BE0000860434908600020424908608CE00120D9
:103BF0003949086000203949086039490860394965
:103C0000086039490860394908603949086001206D
:103C10003849086078E000202F4908602F49086083
:103C20002F4908602F4908602F4908602F49086014
:103C30003049086068E05FE08001002084010020D6
:103C4000880100208C0100209001002094010020B8
:103C50004802002094020020980100209C010020CE
:103C6000A0010020A4010020A8010020AC01002038
:103C70004C02002098020020B0010020B401002076
:103C8000B8010020BC010020C0010020C4010020B8
:103C9000500200209C020020C8010020CC0100201E
:103CA000D0010020D4010020D8010020DC01002038
:103CB00054020020A0020020E00100205802002051
:103CC000A4020020E4010020E8010020EC01002013
:103CD000F0010020F4010020F8010020FC01002088
:103CE0000002002004020020080200200C02002034
:103CF0005C020020A80200200120FC490860FC4969
:103D00000860FC49086000BF00BF4FF4A27004F0D7
:103D1000BBFF012806D0022817D003281ED0052893
:103D200040D12FE00120F44908600020F3490860E9
:103D3000F3490860F3490860F3490860F3490860F3
:103D4000F3490860F349086034E00120EA4908605B
:103D5000EF4908600020EF4908602BE00120E649A8
:103D600008600020E5490860E5490860E549086009
:103D7000E5490860E5490860E54908600120E54932
:103D8000086017E00020DC490860DC490860DC4975
:103D90000860DC490860DC490860DC490860DD49EE
:103DA000086007E00120D4490860D9490860D94972
:103DB000086000BF00BF40F25F1004F065FF0128FB
:103DC00006D0022817D003281ED0052840D12FE0A6
:103DD0000120D14908600020D0490860D04908601E
:103DE000D0490860D0490860D0490860D0490860CF
:103DF000D049086034E00120C7490860CC49086018
:103E00000020CC4908602BE00120C3490860002055
:103E1000C2490860C2490860C2490860C2490860D6
:103E2000C2490860C24908600120C249086017E021
:103E30000020B9490860B9490860B9490860B94922
:103E40000860B9490860B9490860BA49086007E0E4
:103E50000120B1490860B6490860B649086000BF52
:103E600000BFB54800681D2872D2DFE810F01D00C1
:103E70003F0249027100BD0228035603CD03F80337
:103E800023047100710071007100710071007100F4
:103E9000F3012502EC0071007100710071007602DF
:103EA00081008B002B03A2034FF41670A349086016
:103EB0000020A3490870A349087003F037F9472888
:103EC00047D006DC1B2838D01E2848D02E284DD1DC
:103ED0001AE04D2807D0872825D08D2846D101200B
:103EE0009549086042E0672004F0CEFE0446601C5D
:103EF0000446032800DD00242146672007F082F8ED
:103F000001209149086031E040F27B1004F0BCFED2
:103F1000C0F10106314640F27B1007F073F8012032
:103F20008949086022E000208849086013208249FE
:103F3000086001208449086018E000208449086076
:103F4000844908608449086011207B4908600DE0BD
:103F500002E20020814908604FF47A7506E01320E0
:103F60007D49086019207449086000BF00BFCCE398
:103F700001230022AC21AB2000F0FCFB1A206E498B
:103F80000860C2E304F0CCFE0746172F08D0472F85
:103F900002D0872F50D100BF00206749086050E051
:103FA000FEF7F8FB0646012E42DB4FF4BD7004F02D
:103FB0006BFEB0423CDB0B2E2FD2DFE806F02E0664
:103FC0000A0E12161A1E22262A0005205F490860D2
:103FD00023E00C205D4908601FE013205B49086066
:103FE0001BE01A205949086017E021205749086052
:103FF00013E02820554908600FE02F20534908603E
:104000000BE036205149086007E03D204F49086029
:1040100003E044204D49086000BF00BF00204E4926
:10402000086004204449086001204749086002E014
:1040300019204149086004E00021384602F07CFC68
:1040400000BF00BF61E3002000F0D4FD04F068FE73
:104050000746472F0AD004DC172F11D02D2F09D186
:104060000AE0872F03D08D2F04D104E000BF002089
:1040700031490860ECE000BF384606F06DFEE7E02D
:1040800037480078334909780844C6B20C2E12D25A
:10409000DFE806F006121F6875818E9BA8B5C2CFB7
:1040A00000202B4908602B49086013202A4908602A
:1040B000112021490860C9E0032024490860132029
:1040C0002549086004201C49086001201E49086039
:1040D000BCE005201D49086013201F49086004202A
:1040E00015490860012018490860AFE0F801002078
:1040F0005C020020A8020020100200201402002010
:10410000180200201C0200202002002024020020AF
:1041100060020020AC020020280200202C020020B7
:104120003002002034020020380200203C0200202F
:1041300064020020B0020020D002002028030020EA
:104140003E0100203C010020E8020020B8020020CF
:104150000803002030010020D8020020C002002007
:10416000BC0200200C20FE4908601320FD490860B5
:104170000420FD4908600120FC49086066E0132026
:10418000F7490860F74908600420F74908600120F2
:10419000F64908605AE01A20F14908601320F149F5
:1041A00008600420F04908600120F04908604DE0F3
:1041B0002120EB4908601320EA4908600420EA49FD
:1041C00008600120E949086040E02820E4490860CF
:1041D0001320E44908600420E34908600120E34912
:1041E000086033E02F20DE4908601320DD490860B5
:1041F0000420DD4908600120DC49086026E0362003
:10420000D74908601320D74908600420D6490860C0
:104210000120D649086019E03D20D14908601320EB
:10422000D04908600420D04908600120CF490860C7
:104230000CE04420CA4908601320CA4908600420E1
:10424000C94908600120C949086000BF00BF00BF1C
:1042500000BF5AE2FEF75AFF04F062FD472810D073
:1042600004DC172816D02D2824D104E087280DD08F
:104270008D281FD102E0FDF71FFA1BE0FDF748FA79
:1042800018E0B8480068B849086013E00020B64953
:1042900008600FE0B6480068B6490968084400EBBA
:1042A0004000B54901EB8000806810B11220AE4992
:1042B000086000BF00BF28E2FEF7C4FF04F030FD35
:1042C000172807D047280BD087280DD10020A649F2
:1042D000086009E006F0EEFD1120A349086003E044
:1042E0001120A149086000BF00BF0EE20123002297
:1042F0001C211D2000F03EFA02209B49086004E2C8
:1043000004F00EFD0746172F08D0472F02D0872F45
:104310001CD100BF0020944908601CE0FEF73AFA67
:10432000064640F60A30864202D09448864209D1B9
:1043300001208B49086018208B49086001209049B2
:10434000087002E000208849086004E00121384636
:1043500002F0F2FA00BF00BFD7E1012000F04AFCF2
:1043600004F0DEFC0746002086490870472F0AD07B
:1043700004DC172F13D02D2F34D10CE0872F03D05E
:104380008D2F2FD106E000BF00207E4908707649AE
:10439000086027E000BF384606F0DEFC22E07A48DD
:1043A0000078744909780844C6B216B1012E17D1B5
:1043B00009E002206A49086018206A490860042060
:1043C000694908600CE04B20654908601820654980
:1043D000086004206449086001206A49087000BF31
:1043E00000BF00BF00BF90E15D48006800F022FB05
:1043F00004F096FC06464B2E4CD006DC172E18D047
:104400002D2E09D0472E58D10AE04E2E2ED0872EC1
:104410000BD08D2E51D100BF304606F09DFC4CE0F4
:10442000504800685049086047E000204E49086045
:1044300043E007F015FA554901EB0010D0F8008071
:10444000404601F05DFD074602F04AFC68B10420D9
:104450004F490860052044490860464800684D49B6
:104460000860494800684C49086026E000BF3C48A5
:104470000068CD214843494901EB80004068384934
:1044800008600846006802F055FC0028EFD04FF4A1
:104490007A7512E000BF32480068CD2148433F4999
:1044A00051F820002E4908600846006802F042FCDE
:1044B0000028F0D04FF47A7500BF00BF25E102F06C
:1044C0009FF822E101F050F9172804D0472803D0C3
:1044D000872820D11BE000BF2D48006822490860D2
:1044E0002B4805682B480068224908602A48006864
:1044F000254908601A480068CD225043274A02EB3C
:10450000800001228168002003F012F903E00020FE
:104510001549086000BF00BFF7E001F045F8172813
:1045200004D0472803D0872841D13CE000BF184879
:1045300000680D49086016480568164800680D496E
:104540000860154800681049086005480068CD22D9
:104550005043124A02EB80000122816800201FE0D4
:10456000B8020020D8020020D0020020E80200207B
:104570000803002030010020100C0020C6D53C00AC
:104580003E0100203C010020BC020020582C0020ED
:10459000D402002030030020340300204C5A0208CB
:1045A00003F0C6F803E000206649086000BF00BFC2
:1045B000ABE000F021F9172804D0472803D0872862
:1045C00020D11BE000BF604800685E4908605E487B
:1045D00005685E4800685E4908605E4800685E499C
:1045E00008605E480068CD2250435D4A02EB8000BF
:1045F00001228168002003F09BF803E0002051496C
:10460000086000BF00BF80E000F0DAFD172804D08A
:10461000472803D0872820D11BE000BF4A48006804
:1046200048490860484805684848006848490860A3
:10463000484800684849086048480068CD2250430F
:10464000474A02EB800001228168002003F070F8E5
:1046500003E000203B49086000BF00BF55E000F0C8
:10466000AFFB172804D0472803D0872820D11BE0B0
:1046700000BF35480068334908603348056833484F
:10468000006833490860334800683349086033489C
:104690000068CD225043324A02EB8000012281683B
:1046A000002003F045F803E000202649086000BF21
:1046B00000BF2AE001F050F9172804D0472803D0A2
:1046C000872820D11BE000BF1F4800681D490860F3
:1046D0001D4805681D4800681D4908601D480068A0
:1046E0001D4908601D480068CD2250431C4A02EB5A
:1046F000800001228168002003F01AF803E0002006
:104700001049086000BF00BF00BF00BF1548006827
:1047100058B900200B49086013490860012013496B
:1047200008704FF416700F4908600648006885420B
:1047300005D000200E49086001200C490870BDE832
:10474000F0810000D0020020D402002030030020BD
:104750003001002034030020BC020020B8020020F9
:104760004C5A020828030020C00200203F0100200C
:10477000DC020020F8B504460F4615461E4607F039
:1047800031FA01222146002002F0D2FF0321042049
:1047900001F0EAFE00223946104606F043FD3EB91C
:1047A000062000231A4629460090184603F0E2FD31
:1047B0000421084601F0D8FE00220821022003F05F
:1047C00055FE00220921022003F050FE002209219B
:1047D000022003F04BFE00220921022003F046FED6
:1047E00000220B21022003F041FE04F071FD05219F
:1047F000082001F0B9FEF8BD70B57F480078C1000F
:104800004FF07F40C8407D4908607B480078C10078
:104810004FF0807008417A49086077480078C100FD
:104820004FF0005008417749086073480078C10094
:104830004FF0FE4008417449086004F071FA0446E4
:104840000020724908706C480078042874DA7048B7
:104850000068000E6F4908706D480068000C6E49D2
:1048600008706B480088000A6C4908706848007836
:104870006B49087060480078C0EB00100830694947
:10488000086008206849087068480068B0F5FA7F39
:1048900007DA0846007863490968884201D1012097
:1048A00000E0002002465B480178012003F0DEFDB5
:1048B0005D480078001D5C4908705C480068B0F5F0
:1048C000FA7F07DA0846007856490968884201D11C
:1048D000012000E0002002464F480178012003F04B
:1048E000C5FD51480078001D4F4908704F480068C9
:1048F000B0F5FA7F07DA084600784A490968884225
:1049000001D1012000E00020024644480178012046
:1049100003F0ACFD44480078001D4349087043484B
:104920000068B0F5FA7F08DA084600783D49096862
:10493000884202D1012001E00AE000200246384806
:104940000178012003F092FD36480078364908705E
:104950004B2C33D004DC172C07D02D2C49D137E059
:104960004E2C21D08D2C44D10DE0172406F078FF79
:104970002F4901EB001001220568254801682846EF
:1049800006F054FB35E0224800681C4909680840DD
:104990001D490968884206DA1D48006818490968F7
:1049A00008441B49086024E013480078002804DD0F
:1049B00011480078401E104908701AE00E4800782F
:1049C000032804DA0C480078401C0B49087010E0FA
:1049D0000F4800680949096808400A49096888427F
:1049E00006DD0B48006806490968401A0849086056
:1049F00000BF00BF204670BD3D0100201403002011
:104A0000180300201C030020200300203F01002089
:104A1000F8020020100300201103002012030020E0
:104A2000130300202403002035010020140000207F
:104A3000582C00202DE9F041074600266448076005
:104A40006448007890B1FEF7F1F961480068CD2222
:104A50005043614A02EB800001228168002002F08D
:104A600067FE00205D4908605D49086000205949E3
:104A700008705C480068002877D000205949086019
:104A800001213A2001F070FD5448006850B1002225
:104A90008721104603F0EAFC00228821104603F02B
:104AA000E5FC09E000222021104603F0DFFC002293
:104AB0002021104603F0DAFC07213A2001F054FDD2
:104AC00000E0761C484800EB061080680028F8D00B
:104AD00042480068001DB0420CD0052E0ADB0022BF
:104AE0008521104603F0C2FC00228621104603F007
:104AF000BDFC09E000228921104603F0B7FC00222A
:104B00008921104603F0B2FC02203849087033486E
:104B10000578002457E0344800EB05100068401C7D
:104B200000284DD00120324908702D480068844289
:104B300001D1012000E0002002462021002003F0E6
:104B400095FC04202A49087025480068844201D158
:104B5000012000E000200146284602F0E1FC204848
:104B60000068844202D1012001E02EE000200346CB
:104B700001222946002002F017FF72201C4908700C
:104B800017480068844201D1012000E0002002465D
:104B90002021002003F06AFC11480068844201D102
:104BA000012000E0002002462946002002F01AFC05
:104BB000681CC5B20D480078401C0C49087000E024
:104BC0000524601CC4B2052CA5DBBDE8F081000003
:104BD000B80200203F0100204C5A0208BC0200200D
:104BE00030010020E8020020582C0020360100206F
:104BF0003501002070B50646002568480660684803
:104C00000078A0B1FEF712F964480068CD22504345
:104C1000644A02EB800001228168002002F088FDD6
:104C200000205F490870604908606049086060487A
:104C30000068002879D000205D49086001213A20F1
:104C400001F092FC5848006850B1002287211046BC
:104C500003F00CFC00228821104603F007FC09E059
:104C600000222021104603F001FC002220211046E2
:104C700003F0FCFB07213A2001F076FC00E06D1CFC
:104C80004C4800EB051080680028F8D046480068C2
:104C9000001DA8420CD0052D0ADB002285211046FC
:104CA00003F0E4FB00228621104603F0DFFB09E05D
:104CB00000228921104603F0D9FB002289211046E9
:104CC00003F0D4FB02203C490870002463E036481E
:104CD00000682044374901EB00100068401C0028A0
:104CE00056D001203549087030480068844201D10F
:104CF000012000E0002002462021002003F0B6FB46
:104D00002A480068844201D1012000E000200246C8
:104D10002021002003F0AAFB032028490870234823
:104D20000068844202D1012001E036E00020024602
:104D30001D48006820441F4B03EB00104168002011
:104D400006F070FA0BE019480068844201D1012096
:104D500000E0002002462021002003F087FB1748D6
:104D600000787828EFDB7720144908700F48006836
:104D7000844201D1012000E00020024620210020D1
:104D800003F074FB0C480078401C0B49087000E0ED
:104D90000524601CC4B2052C99DB70BDB80200204C
:104DA0003F0100204C5A0208BC02002030010020C4
:104DB000E8020020582C0020360100203501002098
:104DC00070B503F0ADFF04460020F8490870F848BC
:104DD0000078052814DAF7480068B0F5FA7F05DA9C
:104DE00000225F21012003F041FB04E0002220218A
:104DF000012003F03BFBF04800780B38EE490870C7
:104E00004B2C7DD00EDC2B2C7BD006DC172C16D047
:104E10001D2C19D0272C16D153E12D2C72D02E2CFD
:104E2000F9D1F0E08B2C72D004DC4D2C6CD04E2CE0
:104E3000F1D18BE08D2C45D08E2CECD123E0FDF709
:104E4000BFFC00B10224ADE1D9480078052819DA89
:104E50003021D74802780078401CD54B1870D748CD
:104E600081540022012003F001FBD3480078001D8B
:104E7000D1490870CE480078032803D1084600784D
:104E80000F3008708EE1CA480078052819DA312100
:104E9000C74802780078401CC54B1870C748815439
:104EA0000022012003F0E2FAC3480078001DC24945
:104EB0000870BF480078032803D1084600780F30F7
:104EC00008706FE1BA48007805281FDA3221B84827
:104ED00002780078401CB64B1870B8488154002204
:104EE000012003F0C3FAB4480078001DB2490870ED
:104EF000AF480078032809D1084600780F3004E055
:104F000062E0BEE09EE002E03FE008704AE1A848AF
:104F10000078052819DA3321A54802780078401C6A
:104F2000A34B1870A54881540022012003F09EFA7B
:104F3000A1480078001DA04908709D48007803280A
:104F400003D1084600780F3008702BE198480078AC
:104F5000052819DA3421964802780078401C944BD1
:104F60001870964881540022012003F07FFA92487D
:104F70000078001D904908708D480078032803D1FF
:104F8000084600780F3008700CE189480078052841
:104F900019DA3521864802780078401C844B187055
:104FA000864881540022012003F060FA824800788C
:104FB000001D814908707E480078032803D1084607
:104FC00000780F300870EDE079480078052819DA8C
:104FD0003621774802780078401C754B1870774866
:104FE00081540022012003F041FA73480078001D2B
:104FF000714908706E480078032803D1084600788C
:105000000F300870CEE06A480078052819DA372199
:10501000674802780078401C654B187067488154D7
:105020000022012003F022FA63480078001D624943
:1050300008705F480078032803D1084600780F30D5
:105040000870AFE05A480078052819DA3821584826
:1050500002780078401C564B187058488154002242
:10506000012003F003FA54480078001D52490870EB
:105070004F480078032803D1084600780F300870A5
:1050800090E04B48007805281ADA39224848017820
:105090000078401C464B1870484842540022392181
:1050A000012003F0E3F944480078001D42490870EC
:1050B0003F480078032803D1084600780F30087075
:1050C00070E03B480578062D6AD2DFE805F06953A9
:1050D0003D27110336480078401E354908700020EE
:1050E0003649334A1278885453203349087057E0C0
:1050F0002F480078401E2E49087000202F492C4A66
:105100001278885453202C490870002289210120EC
:1051100003F0ACF944202849087041E024480078A5
:10512000401E2349087000202449214A12788854DF
:1051300044202149087000228921012003F096F9BA
:1051400026201D4908702BE019480078401E184998
:10515000087000211948164A1278815426201649F1
:10516000087000228921012003F080F917201249DC
:10517000087015E00E480078401E0D4908700020A8
:105180000E490B4A1278885417200B4908700022E8
:105190008921012003F06AF908200749087000BF3F
:1051A00000BF00BF00BF204670BD00003F010020CF
:1051B0003D010020140000203501002041010020A5
:1051C00070B503F0ADFD04460020F2490870F248C6
:1051D0000078082814DAF1480068B0F5FA7F05DA9B
:1051E00000225F21012003F041F904E00022202188
:1051F000012003F03BF9EA4800780B38E8490870D1
:105200004B2C7DD00EDC2B2C7BD006DC172C16D043
:105210001D2C19D0272C16D155E12D2C72D02E2CF7
:10522000F9D1F2E08B2C72D004DC4D2C6CD04E2CDA
:10523000F1D18CE08D2C45D08E2CECD123E0FDF704
:10524000BFFA00B10224A1E1D3480078042819DA9A
:105250003021D14802780078401CCF4B1870D148DB
:1052600081540022012003F001F9CD480078001D8F
:10527000CB490870C8480078022803D10846007856
:105280000F30087082E1C4480078042819DA31210F
:10529000C14802780078401CBF4B1870C148815447
:1052A0000022012003F0E2F8BD480078001DBC494F
:1052B0000870B9480078022803D1084600780F30FA
:1052C000087063E1B448007804281FDA3221B2483C
:1052D00002780078401CB04B1870B248815400220C
:1052E000012003F0C3F8AE480078001DAC490870F7
:1052F000A9480078022809D1084600780F3004E058
:1053000064E0C1E0A0E002E040E008703EE1A248B5
:10531000007804281ADA33229F4801780078401C6C
:105320009D4B18709F48425400223321012003F006
:105330009DF89B480078001D9949087096480078B0
:10534000022803D1084600780F3008701EE1924809
:105350000078042819DA34218F4802780078401C3C
:105360008D4B18708F4881540022012003F07EF885
:105370008B480078001D8A49087087480078022809
:1053800003D1084600780F300870FFE082480078AB
:1053900004281ADA3522804801780078401C7E4BB8
:1053A00018708048425400223521012003F05EF835
:1053B0007B480078001D7A490870774800780228F9
:1053C00003D1084600780F300870DFE0724800789B
:1053D000042819DA3621704802780078401C6E4B98
:1053E0001870704881540022012003F03FF86C4887
:1053F0000078001D6A49087067480078022803D1C8
:10540000084600780F300870C0E063480078042830
:1054100019DA3721604802780078401C5E4B18701A
:10542000604881540022012003F020F85C48007895
:10543000001D5B49087058480078022803D10846CF
:1054400000780F300870A1E05348007804281ADA79
:105450003822514801780078401C4F4B1870514851
:10546000425400223821012003F000F84C48007813
:10547000001D4B49087048480078022803D10846AF
:1054800000780F30087081E043480078042819DA6A
:105490003921414802780078401C3F4B1870414840
:1054A00081540022012002F0E1FF3D480078001DF8
:1054B0003B49087038480078022803D10846007834
:1054C0000F30087062E034480578012D46D0022D77
:1054D0002ED0032D16D0042D56D10078401E2E4913
:1054E000087000202F492C4A1278885453202C49E8
:1054F000087000222021012002F0B8FF4420284932
:10550000087041E024480078401E234908700020BC
:105510002449214A127888544420214908700022E5
:105520008921012002F0A2FF35201D4908702BE0DF
:1055300019480078401E1849087000201949164A79
:1055400012788854352016490870002289210120DC
:1055500002F08CFF17201249087015E00E48007801
:10556000401E0D49087000210E480B4A12788154E4
:1055700017200B49087000228921012002F076FFD4
:1055800008200749087000BF00BF00BF00BF2046C9
:1055900070BD00003F0100203D01002014000020EC
:1055A00035010020410100202DE9F0416A480078D2
:1055B00080B101206949087000206749087006F031
:1055C0004FF9674901EB00100668304600F03AFFDA
:1055D0006449086003F0A4FB044606F041F9604901
:1055E00001EB00100768384600F08AFC064601F01F
:1055F00085FB05460521082000F0B6FF57480078D6
:1056000000285CD0002055490870B5F5F04F35D022
:105610000ADCDDB1B5F5C04F10D0B5F5D04F1DD0C7
:10562000B5F5E04F4AD121E0B5F5504F2ED0B5F594
:10563000604F33D0B5F5983F40D137E000231A468C
:1056400048480168012001F08EFD37E000231A462A
:1056500044480168012002F07BF82FE000231A463D
:1056600040480168012002F06DF927E000231A4646
:105670003C480168012001F0A6FD1FE000231A4606
:1056800038480168012002F0FDF817E000231A46AF
:1056900034480168012002F085F90FE000231A4622
:1056A00030480168012002F04EF907E000231A4655
:1056B0002C480168012001F085FD00BF00BF172CB8
:1056C00038D02D2C04D0472C41D08D2C40D118E05F
:1056D00006F0C6F8224901EB00100768384600F0D2
:1056E0000FFC064600F0DCFB1E490968884204DA1C
:1056F0001C480068401E1B490860012017490870BB
:1057000026E006F0ADF8164901EB001007683846B0
:1057100000F0F6FB064600F0B9FB12490968884222
:1057200004DD10480068401C0E49086001200B4948
:1057300008700DE006F094F8094901EB0010012211
:10574000066808480168304605F070FC00E000BFBC
:1057500000BF2046BDE8F0813F010020FC02002090
:10576000582C0020F802002070B57648007880B1EF
:1057700001207549087000207249087006F070F821
:10578000724901EB00100568284600F05BFE704985
:10579000086003F0C5FA04460521082000F0E4FE85
:1057A0006948007810B1002067490870172C73D041
:1057B0002D2C04D0472C70D08D2C55D155E0654848
:1057C000006830B101280AD002281ED003284AD12F
:1057D00030E001205E4908605B49087043E05C48A6
:1057E0000068042802D005280DD106E0052058499C
:1057F000086001205449087005E001205449086000
:105800005149087000BF00BF2DE0514800680228D0
:1058100008D003280CD102204D49086001204A49D4
:10582000087005E001204A4908604749087000BF38
:1058300000BF18E006F014F8444901EB00100668B8
:10584000304600F05DFB054600F02AFB4049096840
:10585000884204DA3E480068401E3D490860012045
:105860003949087000BF00BF68E03A48006830B1AD
:1058700001280AD0022821D003284FD135E0012089
:10588000334908603049087048E031480068012811
:1058900004D0052810D108E042E04EE005202C4954
:1058A000086001202849087006E0042028490860A3
:1058B00001202549087000BF00BF2FE02448006880
:1058C000012802D002280ED106E0022020490860FB
:1058D00001201D49087006E003201D4908600120D1
:1058E0001949087000BF00BF18E005F0B9FF17495B
:1058F00001EB00100668304600F002FB054600F0A0
:10590000C5FA13490968884204DD11480068401C43
:105910000F49086001200C49087000BF00BF0DE06E
:1059200005F09EFF094901EB0010012205680848B7
:105930000168284605F07AFB00E000BF00BF204662
:1059400070BD00003F010020FC020020582C002008
:10595000F8020020EC02002010B50020B1490870C8
:10596000B1480078082814DAB0480068B0F5FA7F2A
:1059700005DA00225F21012002F078FD04E0002218
:105980002021012002F072FDA94800780B38A849B7
:10599000087003F0C5F904462E2C6ED010DC1E2CC6
:1059A0006CD006DC172C1AD01B2C68D01D2C1AD1F9
:1059B0001AE0272C76D02B2C75D02D2CF7D1ADE00A
:1059C0008B2C47D006DC4B2C6ED04D2C6ED04E2C41
:1059D000EDD155E08D2C2BD08E2CE8D116E0FCF7C4
:1059E000EFFE00B102241AE18F48007808280CDA93
:1059F00030218D4802780078401C8B4B18708D4800
:105A000081540022012002F031FD08E1864800782F
:105A100008280CDA3121844802780078401C824B37
:105A20001870844881540022012002F01FFDF6E026
:105A30007D48007808280CDA32217B48027800780B
:105A4000401C794B18707B4881540022012002F0E1
:105A50000DFDE4E07448007808280DDA332272481E
:105A600001780078401C704B187072484254002234
:105A70003321012002F0FAFCD1E03CE08AE071E041
:105A80006948007808280CDA3421674802780078E1
:105A9000401C654B1870674881540022012002F0B9
:105AA000E5FCBCE087E04BE013E0FFE75E480078F0
:105AB00008280DDA35225C4801780078401C5A4BE2
:105AC00018705C48425400223521012002F0CEFCBF
:105AD000A5E05548007808280CDA362152480278AB
:105AE0000078401C504B187052488154002201200D
:105AF00002F0BCFC93E04C48007808280DDA37220D
:105B0000494801780078401C474B18704948425476
:105B100000223721012002F0A9FC80E042480078F1
:105B200008280CDA3821404802780078401C3E4BA7
:105B30001870404881540022012002F097FC6EE06A
:105B40003948007808280CDA39213748027800787B
:105B5000401C354B1870374881540022012002F058
:105B600085FC5CE030480078082812DA324800787A
:105B700078B92C222C4801780078401C2A4B1870E8
:105B80002C48425401202C49087000222E2102F09A
:105B90006DFC44E02448007860B92D212248027849
:105BA0000078401C204B18702248815400220120AC
:105BB00002F05CFC33E01C48007800282EDD1A4817
:105BC0000078401E184908701A480978405C2C2853
:105BD00002D100201849087000201649124A127894
:105BE000885411480078072809DA00222021012072
:105BF00002F03CFC0E4800780B380D4908700C4848
:105C000000780B380A49087000222021012002F098
:105C10002DFC074800780B380549087000BF00BF0D
:105C2000204610BD3F0100203D010020140000204F
:105C300035010020410100204001002070477047DD
:105C400010B5022000F09CF8B8B102210B4800F01A
:105C50008EFB60B90A4800680A49884207DA0A4898
:105C6000007820B906480068401C054908600A20F1
:105C700005490870022000F07DF810BD00080140C1
:105C8000D003002040420F000000002010B5042087
:105C900000F076F8B8B104210B4800F068FB60B959
:105CA0000A4840680A49884207DA0A48007820B959
:105CB00006484068401C054948600A2005490870AC
:105CC000042000F057F810BD00080140D003002068
:105CD00040420F00010000207047000010B5102066
:105CE00000F04EF8B8B110210B4800F040FB60B94D
:105CF0000A48C0680A49884207DA0A48007820B989
:105D00000648C068401C0549C8600A20054908705B
:105D1000102000F02FF810BD00140140D003002027
:105D200040420F000300002010B5802000F028F84A
:105D3000B8B180210B4800F01AFB60B90A488068AE
:105D40000A49884207DA0A48007820B9064880687C
:105D5000401C054988600A2005490870802000F031
:105D600009F810BD00080140D003002040420F0098
:105D7000020000200149086070470000140401403F
:105D8000064A014600201268044B0A4014331B687F
:105D90000B4202D0002A00D00120704700040140CD
:105DA00030B583791949026853B30B6893430B608C
:105DB0000A1D13680468A343136002790A44136838
:105DC000046823431360114A083213680468A3432C
:105DD0001360131D1C680568AC431C604479102CCB
:105DE00005D021440A68006802430A6030BD11688A
:105DF000046821431160196800680143196030BDCF
:105E00000079084401689143016030BD00040140FD
:105E10007047000004490A6822F010020A600A680C
:105E200002430A60704700000020024004490A68EB
:105E300002F038020A600A6802430A6070470000F4
:105E400000200240704710B5044640F27B1002F07B
:105E50001BFF08B9204610BDA4F52F70C0EB001041
:105E600000EB4000192101EB4000322190FBF1F0E2
:105E700000F57F70EFE700000146C1EBC100024A68
:105E800002EB80004069704758E901080146C1EB08
:105E9000C100024A02EB80000069704758E901081E
:105EA0000146C1EBC100024A02EB8000C0687047A6
:105EB00058E901080146C1EBC100024A52F820002E
:105EC0007047000058E9010810B50446002300E0BF
:105ED0005B1CC3EBC300094901EB80008068A04252
:105EE00007D0C3EBC30051F820004FF6FF71884282
:105EF000EED11846FFF7DEFF10BD000058E901089B
:105F000070B504464FF0FF3625460648854206DA4E
:105F100040F2391200212846FBF734FD0646304690
:105F200070BD000078D4030008B50121480202F0DA
:105F300019FC0121084602F0FDFB0121084602F090
:105F400011FC0121042002F00DFC0121082002F0C7
:105F500009FC0121102002F005FC0121202002F0A3
:105F600001FC0121402002F0FDFB0121480402F068
:105F7000EDFB0121880402F0E9FB0121082000F07B
:105F8000CFF90121AE4800F0CBF98620ADF8000032
:105F900004208DF8030003208DF802006946A9480B
:105FA00000F070F94FF40070ADF8000003208DF898
:105FB000020018208DF803006946A24800F062F93B
:105FC0004FF48060ADF8000004208DF803006946AE
:105FD0009C4800F057F90120ADF8000003208DF82F
:105FE000020004208DF803006946964800F04AF943
:105FF0002020ADF8000003208DF8020010208DF85D
:10600000030069468F4800F03DF94FF4D050ADF8D9
:10601000000003208DF8020010208DF8030069466F
:10602000884800F02FF94FF47050ADF800001020B0
:106030008DF8030003208DF802006946824800F0C5
:1060400021F94020ADF8000003208DF80200142053
:106050008DF8030069467C4800F014F98220ADF801
:10606000000003208DF8020004208DF8030069462B
:10607000754800F007F90320ADF8000000208DF806
:1060800003006946704800F0FDF82020ADF80000DC
:1060900000208DF8030069466C4800F0F3F84FF4D7
:1060A0007070ADF8000010208DF803006946674855
:1060B00000F0E8F81020ADF8000004208DF803008F
:1060C0006946624800F0DEF84FF20F00ADF80000BC
:1060D00003208DF8020048208DF8030069465C48D3
:1060E00000F0D0F82020ADF8000003208DF8020069
:1060F00018208DF803006946554800F0C3F8402089
:10610000ADF8000003208DF8020004208DF8030094
:1061100069464F4800F0B6F84FF48070ADF80000C3
:1061200003208DF8020018208DF8030069464848C6
:1061300000F0A8F84FF40070ADF8000003208DF8CF
:10614000020004208DF803006946414800F09AF8E7
:106150004FF44960ADF8000003208DF802001020D4
:106160008DF8030069463A4800F08CF80120ADF83C
:10617000000014208DF8030003208DF8020069460A
:10618000344800F07FF88020ADF8000010208DF832
:10619000030003208DF8020069462E4800F072F8D3
:1061A0004FF47F40ADF8000003208DF80200282056
:1061B0008DF803006946274800F064F801210020AB
:1061C00000F04CF8022024490860002008710C20DF
:1061D0004871012088710846FFF7E2FD0221002086
:1061E00000F03CF804201C490860002008710C20D5
:1061F0004871012088710846FFF7D2FD0721002071
:1062000000F02CF8802014490860002008710C2050
:106210004871012088710846FFF7C2FD0421022061
:1062200000F01CF810200C490860002008710C20B8
:106230004871012088710846FFF7B2FD08BD0000D3
:106240003000140000080140000C01400010014023
:1062500000140140001801409800002010B58A0782
:1062600021F003040649130F21440F228C689A4041
:1062700094438C608A68984002438A6010BD000095
:1062800000000140F0B5CB78002503F00F02DB06DB
:1062900001D58B781A430B884FF00F0E13F0FF0FC8
:1062A0004FF0010C19D004680E880CFA05F31E405B
:1062B0009E420ED1AF000EFA07F6B44302FA07F77A
:1062C000CE783C43282E00D14361CE78482E00D1B1
:1062D00003616D1C082DE7D304600B88FF2B1DD9CB
:1062E0004468002505F108060CFA06F30E881E40E6
:1062F0009E420FD1AF000EFA07F624EA060602FA14
:1063000007F43443CE78282E00D14361CE78482E4E
:1063100000D103616D1C082DE4D34460F0BD000082
:10632000F0B5104D6B68440D260184B2C0F30157DF
:10633000B440C0F30342032F05D0C0020AD50320A6
:106340009040834307E0686823F0706220F070603B
:10635000686002E0A34343F0706201B122436A60C7
:10636000F0BD000000000140806880B27047024626
:10637000002092680A4200D00120704702460020A7
:10638000D2680A4200D00120704741617047016124
:106390007047C1607047000070B506463546472D0E
:1063A00000DA47251A48854200DD0546D222002141
:1063B000284602F0E7FE441E012C00DA0124601C8E
:1063C00000EB4000134951F8200004EB4401114A4E
:1063D00052F82110401A04EB440102EB8101496894
:1063E000691A4843611C01EB410102EB81014968D4
:1063F00004EB4402074B03EB82025268891A90FBBC
:10640000F1F004EB44011A4652F82110084470BD23
:1064100054220E00B00B020810B50446074884420F
:1064200009DA2046FFF76CFDC0EBC000044901EB20
:106430008000806810BD0020FCE7000078D40300D5
:1064400058E9010870B504460E48844218DA20461F
:10645000FFF756FD054600F037FC30B12046FFF748
:10646000DBFF054602F0E0FC70BD2046FFF748FD6B
:10647000C0EBC000044901EB800040680068F3E70E
:106480000020F1E778D4030058E901080146002014
:10649000002201291BDB062919DC072911D2DFE8BC
:1064A00001F0100406080A0C0E00012209E0022285
:1064B00007E0042205E0082203E0102201E0202288
:1064C00000BF00BF024B1B68134003B90120704797
:1064D0005800002002461146002900DA0021B1F5DB
:1064E000805F01DB40F6FF714FF47A704843C1F5DD
:1064F000805390FBF3F0704710B54FF4C17002F079
:10650000C3FBB8B110480468B4F5967F03DB40F2D2
:106510001450844207DD0D48006820B90121002095
:1065200003F022FE0EE00A4804600121002002F080
:106530004BFE07E04FF42F70054908600121002051
:1065400002F042FE10BD0000B00B0020B0000020A1
:1065500034000020014601F114006422504340F64B
:10656000FF7290FBF2F07047024B1970024B1870EB
:1065700070470000360100203501002000BFFEE713
:10658000704770477047704710B501210148FFF709
:10659000FEFE10BD0018014002494CF6CC400860D8
:1065A000704700000030004002494AF6AA20086007
:1065B000704700000030004001494860704700000B
:1065C0000030004001498860704700000030004002
:1065D00001490860704700000030004010B545F2E6
:1065E0005550FFF7F5FF0520FFF7E6FF40F6C41012
:1065F000FFF7E8FFFFF7D8FFFFF7CEFF10BD000061
:1066000070B5C6480078002843D0C5480068CD2240
:106610005043C44A02EB800001228168002001F04F
:1066200087F803210220FFF79FFF02F051FE05F0DB
:1066300017F90446002100F073FF05F011F9C4B208
:10664000002301222146184601F0AEF905F008F9B1
:10665000C4B200222146104600F0C4FE04210846C0
:10666000FFF782FF00220821022001F0FFFE002236
:106670000921022001F0FAFE00220921022001F086
:10668000F5FE00220921022001F0F0FE0020A349BE
:10669000087005F0E5F8A44901EB001005682846EC
:1066A000FFF72EFC044600F029FBC0F30A01002985
:1066B0007ED1C0122A287BD2DFE800F01517181906
:1066C0007A7A7A7A7A517A7A1A1B1C1D1E7A7A247F
:1066D00050167A7A259126271F202122237A7A7A4A
:1066E0003C7A287A7AD900BF00BF00BF00BF00BF44
:1066F00000BF00BF00BF00BF00BF00BF00BF00BFA2
:1067000000BF00BF00BF00BF00BF00BF00220A21C2
:10671000022001F0ABFE05F0A3F8834901EB001065
:1067200004682046FFF78EFE8049086006208049F5
:106730000860F1E000220A21022001F097FE05F036
:106740008FF8794901EB001004682046FFF77AFEC4
:10675000764908601B2076490860DDE000BF002212
:106760000B21022001F082FE05210820FFF7FCFE2C
:1067700000228921012001F079FE6E480078001D79
:106780006C49087000228921012001F06FFE6948E0
:106790000078001D6749087000223A21012001F0AD
:1067A00065FE64480078001D62490870002200E020
:1067B000A5E08921012001F059FE5E480078001D06
:1067C0005C49087000228921012001F04FFE05215B
:1067D0000820FFF7C9FE0720554908609CE0002209
:1067E0000B21022001F042FE05210820FFF7BCFE2C
:1067F00000228921012001F039FE4E480078001D59
:106800004C49087000228921012001F02FFE4948DF
:106810000078001D4749087000228921012001F0FD
:1068200025FE44480078001D4249087000222D21B1
:10683000012001F01BFE3F480078001D3D49087013
:1068400000228921012001F011FE3A480078001D44
:106850003849087000228921012001F007FE052136
:106860000820FFF781FE08203149086054E004F059
:10687000F7FF2D4901EB001004682046FFF7E2FD09
:106880002A49086000220B21022001F0EFFD0521BA
:106890000820FFF769FE25480068010E002201204C
:1068A00001F0E4FD23480078001D22490870002211
:1068B0001E480068C0F30741012001F0D7FD1D48C4
:1068C0000078001D1B490870002218480088C0F39A
:1068D0000721012001F0CAFD16480078001D154966
:1068E0000870124801780022012001F0BFFD052147
:1068F0000820FFF739FE1C200D4908600CE000223B
:106900000B21022001F0B2FD05210820FFF72CFE2B
:1069100009200749086000BF00BF70BD3F0100208B
:10692000B80200204C5A0208582C0020F80200201F
:10693000D00200203501002070B505460C46B54850
:10694000007808287BDCB3480078082814DAB248BD
:106950000068B0F5FA7F05DA00225F21012001F01E
:1069600085FD04E000222021012001F07FFDAB48DD
:1069700000780B38A94908704B2D7BD00CDC2B2DEF
:1069800079D004DC1D2D14D0272D2AD114E12D2D12
:1069900072D02E2DF9D1C3E08B2D57D004DC4D2DB4
:1069A0006BD04E2DF1D16FE08D2D34D08E2DECD1EA
:1069B00018E098480078082813DA302195480278C2
:1069C0000078401C934B18709548815424B90022DC
:1069D000012001F04BFD04E000222A21012001F0FA
:1069E00045FD15E18B480078082813DA31218948E4
:1069F00002780078401C874B18708948815424B96C
:106A00000022012001F032FD04E000222A210120B1
:106A100001F02CFDFCE07F480078082815DA3222CE
:106A20007C4801780078401C7A4B18707C484254AE
:106A300034B900223221012001F018FD05E0E8E020
:106A400000222A21012001F011FDE1E071480078C7
:106A5000082818DA33226F4801780078401C6D4B03
:106A600018706F4842544CB900223321012001F0C4
:106A7000FDFC08E03BE085E06BE01FE000222A21FE
:106A8000012001F0F3FCC3E062480078082814DA22
:106A90003422604801780078401C5E4B18706048D2
:106AA00042542CB900223421012001F0DFFC04E023
:106AB00000222A21012001F0D9FCA9E055480078E4
:106AC000082813DA3521534802780078401C514BCE
:106AD00018705348815424B90022012001F0C6FCEB
:106AE00004E000222A21012001F0C0FC90E0494886
:106AF0000078082813DA3621464802780078401CCE
:106B0000444B18704648815424B90022012001F0FA
:106B1000ADFC04E000222A21012001F0A7FC77E06F
:106B20003C480078082813DA37213A480278007880
:106B3000401C384B18703A48815424B90022012077
:106B400001F094FC04E000222A21012001F08EFCD7
:106B50005EE030480078082813DA38212D480278A2
:106B60000078401C2B4B18702D48815424B900220A
:106B7000012001F07BFC04E000222A21012001F029
:106B800075FC45E023480078082814DA39222148AA
:106B900001780078401C1F4B1870214842542CB9D2
:106BA00000223921012001F061FC04E000222A21A9
:106BB000012001F05BFC2BE016480078002826DD60
:106BC00014480078401E1349087000201449114AE7
:106BD000127888540F480078072809DA002220210B
:106BE000012001F043FC0D4800780B380B49087078
:106BF0000A4800780B38094908700022202101203A
:106C000001F034FC054800780B380449087000BFD7
:106C100000BF70BD3D0100201400002035010020A0
:106C20004101002010B510210448FFF7B0FB4FF4DC
:106C300080610348FFF7A9FB012010BD0008014057
:106C40000010014030B502460B4801680B4803684C
:106C50000EE001EB41000A4C54F82000904201D1B3
:106C6000012030BD481C142490FBF4F504FB1501F1
:106C70009942EED10020F4E7C8000020CC000020AB
:106C8000E40D0020014608480068CD225043074A21
:106C900002EB8000143000EB0110C068006808B1FE
:106CA000012070470020FCE7B80200204C5A02087F
:106CB0000146C1EBC100034A02EB8000008B00F4E7
:106CC000FE60704758E901080146C1EBC100034A64
:106CD00002EB8000007EC0F34000704758E90108D5
:106CE0000146C1EBC100044A02EB8000007E00F0C7
:106CF000010080F00100704758E901080146C1EB2E
:106D0000C100034A02EB8000806900F4FF20704755
:106D100058E901080146C1EBC100054A52F82000BC
:106D20004FF6FF72904201D1012070470020FCE72E
:106D300058E901080146CD204843054A02EB80008E
:106D4000C068006808B1012070470020FCE700001F
:106D50004C5A020838B500250820ADF80000102074
:106D60008DF8030003208DF8020069464A48FFF7BA
:106D700089FA08214848FFF708FBFCF7BFF94648A5
:106D8000FFF7F2FA04130820ADF8000048208DF850
:106D9000030069464048FFF775FA0F2C76D10420AE
:106DA000ADF8000010208DF8030003208DF80200DC
:106DB00069463948FFF766FA04213748FFF7E5FAD4
:106DC000FCF79CF93448FFF7CFFA04130420ADF820
:106DD000000048208DF8030069462F48FFF752FA5B
:106DE0000F2C4FD10220ADF8000010208DF80300C9
:106DF00003208DF8020069462748FFF743FA022175
:106E00002548FFF7C2FAFCF779F92348FFF7ACFAF7
:106E100004130220ADF8000048208DF803006946F5
:106E20001D48FFF72FFA0F2C27D10120ADF80000E5
:106E300010208DF8030003208DF8020069461648E3
:106E4000FFF720FA01211448FFF79FFAFCF756F9E3
:106E50001148FFF789FA04130120ADF8000048201B
:106E60008DF8030069460C48FFF70CFA0F2C00D18F
:106E70000FE0E0B240F010050BE0E0B240F020057A
:106E800007E003E0E0B240F0400502E0E0B240F08D
:106E90008005284638BD00000014014070B500F0A0
:106EA00035F8002417E0002511E0A107080E294657
:106EB00003F0E4F9002606E000222146012004F058
:106EC00013F9701CC6B2402EF6DB681CC5B2082D43
:106ED000EBDB601CC4B2022CE5DB00F023F870BDD4
:106EE00010B548F220010748FFF74FFA4FF48041F0
:106EF0000448FFF74CFA40210348FFF746FAFFF732
:106F0000CDFF10BD000C01400008014010B53E222D
:106F10000021084604F0E8F83E220121002004F098
:106F2000E3F810BD10B53F220021084604F0DCF85C
:106F30003F220121002004F0D7F810BD70B50546AE
:106F40000C466E201C490870012D28D11B48006892
:106F5000C8280CDA00201A490870E2B2FE2101F0BC
:106F600085FAE2B22021002001F080FA23E01348E4
:106F70000068B0F5FA7F1EDD10480068B0F52F7F7D
:106F800019DA01200E490870E2B2F821002001F060
:106F90006DFAE2B22021002001F068FA0BE0022D28
:106FA00009D1E2B2F721002001F060FAE2B2FD213E
:106FB000002001F05BFA70BD3501002014000020B4
:106FC0000403002000BFFEE77047000010B54FF437
:106FD0008031C80200F0A0F84FF4E06000F092F8B1
:106FE000284800F051F826202649087000204870F3
:106FF00001208870C870084600F046F82720214913
:1070000008700020487001208870C870084600F0A1
:107010003BF803201B49087000204870022088704C
:107020000120C870084600F02FF8072015490870A5
:107030000020487088700120C870084600F024F8CD
:107040000820104908700020487088700120C8701E
:10705000084600F019F80A200A4908700020487014
:1070600088700120C870084600F00EF81720054906
:1070700008700020487088700120C870084600F031
:1070800003F810BD91000020F0B50F22C3780178FD
:1070900001244FF0E0263BB3184B1B6803F4E06378
:1070A000C3F5E0631D0AC5F10403EA4045789D403D
:1070B000837813402B431A018B07DF0E21F0030363
:1070C0000F49BA405D182968FF23BB4099431A4015
:1070D00011432960007800F01F018C40400906EB45
:1070E0008000C0F80041F0BD01F01F008440480955
:1070F00006EB8000C0F88041F0BD00000CED00E020
:1071000000E400E0024908430249086070470000BB
:107110000000FA050CED00E0024A1140014302486C
:107120000160704780FFFF1F08ED00E010B50848C0
:10713000006820B901200649086003F089FB03F0CC
:10714000BFF803F03DF901F0EBFD0446204610BD09
:10715000DC0200207047000001490862704700000F
:1071600000000E4270472DE9F04180460C4615465E
:107170001E4604F1920003F011FA074685B104E0BF
:1071800032462021404601F071F938467F1C06281E
:10719000F6DB324604F19201404604F043F80FE07A
:1071A000324604F19201404604F03CF804E03246D5
:1071B0002021404601F05AF938467F1C0628F6DBAC
:1071C000BDE8F081704770472DE9F04107460D4654
:1071D00090461E4680240C4800780C380A490870F6
:1071E0000EE005EA040028B132463021384601F0AD
:1071F0003DF904E032463121384601F037F9641098
:10720000002CEED1BDE8F081350100202DE9F041E0
:1072100006460C4690461D460020244908702A4622
:107220002021304601F022F90A2094FBF0F00A21D7
:1072300090FBF1F201FB12003030C7B22A4639460A
:10724000304601F013F90A2094FBF0F100FB1140E5
:107250003030C7B22A463946304601F007F92A468F
:107260002D21304601F002F94FF47A7094FBF0F0D2
:107270000A2190FBF1F201FB12003030C7B22A461E
:107280003946304601F0F2F8642094FBF0F00A2110
:1072900090FBF1F201FB12003030C7B22A463946AA
:1072A000304601F0E3F8BDE8F08100003401002031
:1072B0002DE9F0470746884691461E464748007824
:1072C000303846490870464D2C6804F00F00FAF734
:1072D0004AFA824632465146384601F0C7F8C4F3AE
:1072E0000320FAF740FA824632465146384601F00A
:1072F000BDF8C4F30340FAF736FA824632465146E7
:10730000384601F0B3F8C4F30360FAF72CFA82466A
:1073100032465146384601F0A9F832462D2138460A
:1073200001F0A4F82D1D2C6804F00F00FAF71BFAE9
:10733000824632465146384601F098F8C4F303209D
:10734000FAF711FA824632465146384601F08EF875
:10735000C4F30340FAF707FA8246324651463846EC
:1073600001F084F8C4F30360FAF7FDF9824632466F
:107370005146384601F07AF832462D21384601F060
:1073800075F82D1D2C6804F00F00FAF7ECF9824611
:1073900032465146384601F069F8C4F30320FAF743
:1073A000E2F9824632465146384601F05FF8C4F3AE
:1073B0000340FAF7D8F9824632465146384601F082
:1073C00055F8C4F30360FAF7CEF9824632465146C7
:1073D000384601F04BF8BDE8F08700003501002089
:1073E000E8F7FF1F2DE9F04105460C4616467120CF
:1073F00049490870494901EB04110868FEF780FD0E
:107400008046FFF755FC074607F00F0000287AD1A9
:107410003811152877D2DFE800F0760B1C22287689
:10742000762E343A40464C52585E767664766B003F
:1074300040F27B1001F028FC28B932460021284692
:1074400003F0F0FE04E032460F21284603F0EAFE86
:107450005FE032460121284603F0E4FE59E032465F
:107460000221284603F0DEFE53E03246032128467F
:1074700003F0D8FE4DE032460421284603F0D2FE48
:1074800047E032460521284603F0CCFE41E0324673
:107490000621284603F0C6FE3BE032460721284677
:1074A00003F0C0FE35E032460821284603F0BAFE5C
:1074B0002FE032460921284603F0B4FE29E0324687
:1074C0000A21284603F0AEFE23E032460B2128466F
:1074D00003F0A8FE1DE032460C21284603F0A2FE70
:1074E00017E032460D21284603F09CFE11E00AE029
:1074F0003246F021284600F0B9FF3246F5212846F1
:1075000000F0B4FF05E032460E21284603F08AFE63
:1075100000BF00BFBDE8F08135010020582C0020DD
:1075200070B504460D46074800EB04102A46416832
:10753000002003F077FE2A460E21002003F072FEA1
:1075400070BD0000582C00202DE9F04105460C4686
:1075500016460027672001F097FB06283FD2DFE898
:1075600000F0030C16202A3404EB4401234A52F89D
:107570003100F9F735F8074631E004EB44011F4AC2
:1075800002EBC1014868F9F72BF8074627E004EB46
:1075900044011A4A02EBC1018868F9F721F807464D
:1075A0001DE004EB4401154A02EBC101C868F9F77C
:1075B00017F8074613E004EB4401104A02EBC1013F
:1075C0000869F9F70DF8074609E004EB44010B4A96
:1075D00002EBC1014869F9F703F8074600BF00BF95
:1075E00007EB4700C0F140000549087032462146CC
:1075F000284603F017FEBDE8F0810000144702089A
:107600003501002010B500210846FEF7ADFF00222D
:107610000221084600F02AFF00212020FEF7A4FFE7
:1076200000220321022000F021FF00214020FEF76C
:107630009BFF00220321022000F018FF00216020A0
:10764000FEF792FF00220421022000F00FFF042128
:107650000020FEF789FF00220521022000F006FF2E
:1076600004212020FEF780FF00220621022000F0E6
:10767000FDFE04214020FEF777FF002206210220B4
:1076800000F0F4FE04216020FEF76EFF00220721C7
:10769000022000F0EBFE10BD10B50020224908705A
:1076A0002249087000220D21022000F0DFFE202078
:1076B0001D49087000220E21022000F0D7FE402054
:1076C0001949087000220E21022000F0CFFE602030
:1076D0001549087000220F21022000F0C7FE00208B
:1076E000114908700420114908700022102102205D
:1076F00000F0BCFE20200C4908700022112102205D
:1077000000F0B4FE40200849087000221121022038
:1077100000F0ACFE60200449087000221221022013
:1077200000F0A4FE10BD000035010020360100204D
:1077300070B504460D461646FFF764FF0021084663
:10774000FEF712FF324629462046FFF7FDFE70BDC8
:107750002DE9F04180460C4615461E4604F1160000
:1077600002F01CFF074685B104E032462021404666
:1077700000F07CFE38467F1C0628F6DB324604F11A
:107780001601404603F04EFD0FE0324604F11601AB
:10779000404603F047FD04E032462021404600F019
:1077A00065FE38467F1C0628F6DBBDE8F0812DE932
:1077B000F04106460D461746284601F065FA044694
:1077C000210E3A46304600F051FE3A46C4F30741D6
:1077D000304600F04BFE3A46C4F30721304600F035
:1077E00045FEE1B23A46304600F040FEBDE8F08189
:1077F0002DE9F04107460C4615461E4605B33246B4
:107800002021384600F032FE32462021384600F072
:107810002DFE210E3246384600F028FE3246C4F3D3
:107820000741384600F022FE3246C4F307213846AD
:1078300000F01CFEE1B23246384600F017FE1FE0B1
:10784000210E3246384600F011FE3246C4F307419D
:10785000384600F00BFE3246C4F30721384600F0EC
:1078600005FEE1B23246384600F000FE32462021E5
:10787000384600F0FBFD32462021384600F0F6FD88
:10788000BDE8F081704700002DE9F04106460C4646
:1078900090461D46002029490870294894FBF0F0C5
:1078A0000A2190FBF1F201FB12003030C7B22A46E8
:1078B0003946304600F0DAFD42F2107094FBF0F0E9
:1078C0000A2190FBF1F201FB12003030C7B22A46C8
:1078D0003946304600F0CAFD4FF47A7094FBF0F060
:1078E0000A2190FBF1F201FB12003030C7B22A46A8
:1078F0003946304600F0BAFD2A462D21304600F0C8
:10790000B5FD0A2094FBF0F00A2190FBF1F201FB97
:1079100012003030C7B22A463946304600F0A6FD84
:107920000A2094FBF0F100FB11403030C7B22A4628
:107930003946304600F09AFDBDE8F0813401002060
:10794000A086010070472DE9F04180460C4615469F
:107950001E4604F1100002F021FE074685B104E046
:1079600032462021404600F081FD38467F1C062823
:10797000F6DB324604F11001404603F053FC0FE001
:10798000324604F11001404603F04CFC04E032465C
:107990002021404600F06AFD38467F1C0628F6DBB1
:1079A000BDE8F081704700002DE9F84F06460D460E
:1079B00017469846A34901EB05110868FEF7A0FA9F
:1079C0008246FFF79BF981469E4901EB0511086845
:1079D000FEF738FD04464C209B490870C9F30A00A5
:1079E000002822D14FEAE9202A281ED2DFE800F041
:1079F000A11D1D1D151E2F363D44521D97ABB5BF51
:107A00001D73251D901DDD1D1DFEC91DD31D1D1DD2
:107A10001DFDFC1D1D4BFB1D1DFA062043463A466D
:107A200021460090304600F0A5FC08E143463A4666
:107A30002146304600F03CFC01E1402082490870BC
:107A400043463A462146304600F05CF9F7E04346AB
:107A50003A462146304600F0C9FBF0E043463A463C
:107A60002146304600F018FAE9E043463A462146FE
:107A7000304600F0EBF8E2E043463A462146304615
:107A800000F0B4F9DBE043463A462146304600F0C8
:107A900065FAD4E040F27B1001F0F6F830B94346C5
:107AA0003A462146304600F0D1FA13E0A4F52F7093
:107AB000C0EB001000EB4000192101EB4000322127
:107AC00090FBF1F000F57F7A43463A465146304646
:107AD00000F0BCFAB3E040F27B1001F0D5F830B909
:107AE00043463A462146304600F0E2FB0FE0C4EB45
:107AF000041000EB4000192101EB4000322190FB03
:107B0000F1FA43463A465146304600F0D1FB96E042
:107B100043463A4621463046FFF778FB8FE04C203B
:107B20004949087043463A4621463046FFF71BFB59
:107B300085E04C204449087043463A462146304689
:107B4000FFF706FE7BE04C203F49087043463A466B
:107B500021463046FFF7F6FE71E04C203A490870A6
:107B600043463A4621463046FFF72DFB67E04C205E
:107B70003549087043463A4621463046FFF782FEB3
:107B80005DE04C203049087043463A462146304675
:107B9000FFF708FF53E04C202B49087043463A4654
:107BA00021463046FFF7CFFE49E040F27B1001F05E
:107BB0006BF830B943463A462146304600F0AEFAFB
:107BC00019E0A4F52F70C0EB001000EB4000192164
:107BD00001EB4000322190FBF1F000F52F7A434693
:107BE0003A4604E024E01CE00DE005E012E05146D6
:107BF000304600F093FA22E043463A4621463046AA
:107C0000FFF7E2FA1BE043463A4621463046FFF7CB
:107C10004FFB14E043463A4621463046FFF734FE18
:107C20000DE043463A4621463046FFF7CBFA06E0E0
:107C300043463A4621463046FFF7DAFD00BF00BF13
:107C4000BDE8F88F582C0020350100202DE9F041C7
:107C500006460C4690461D4600202949087042F20F
:107C6000107094FBF0F00A2190FBF1F201FB12007E
:107C70003030C7B22A463946304600F0F7FB2A4674
:107C80002E21304600F0F2FB4FF47A7094FBF0F0B6
:107C90000A2190FBF1F201FB12003030C7B22A46F4
:107CA0003946304600F0E2FB642094FBF0F00A21F4
:107CB00090FBF1F201FB12003030C7B22A46394680
:107CC000304600F0D3FB0A2094FBF0F00A2190FB31
:107CD000F1F201FB12003030C7B22A463946304675
:107CE00000F0C4FB0A2094FBF0F100FB114030309F
:107CF000C7B22A463946304600F0B8FBBDE8F081ED
:107D0000340100202DE9F04106460C4617461D4679
:107D1000002034490870344894FBF0F000F0FF086C
:107D20002B463A464146002000F088FC42F2107093
:107D300094FBF0F00A2190FBF1F201FB12003030CD
:107D400000F0FF082A464146304600F08FFB2A46E5
:107D50002E21304600F08AFB4FF47A7094FBF0F04D
:107D60000A2190FBF1F201FB1200303000F0FF0815
:107D70002A464146304600F079FB642094FBF0F03F
:107D80000A2190FBF1F201FB1200303000F0FF08F5
:107D90002A464146304600F069FB2A462E213046ED
:107DA00000F064FB0A2094FBF0F00A2190FBF1F252
:107DB00001FB1200303000F0FF082A4641463046F1
:107DC00000F054FB0A2094FBF0F100FB114030302E
:107DD00000F0FF082A464146304600F047FBBDE868
:107DE000F081000034010020A08601002DE9F0415F
:107DF00007460C4615461E4625B132462021384618
:107E000000F034FB4FF4167094FBF0F00A2190FB65
:107E1000F1F201FB1200303000F0FF08324641461B
:107E2000384600F023FB3C2094FBF0F00A2190FB45
:107E3000F1F201FB1200303000F0FF0832464146FB
:107E4000384600F013FB32463A21384600F00EFB6C
:107E50003C2094FBF0F100FB11400A2190FBF1F073
:107E6000303000F0FF0832464146384600F0FEFA56
:107E70003C2094FBF0F100FB11400A2190FBF1F251
:107E800001FB1200303000F0FF0832464146384610
:107E900000F0ECFABDE8F0812DE9F04106460C4611
:107EA00017461D4600202C49087042F2107094FBC2
:107EB000F0F0642190FBF1F201FB120000F0FF08EA
:107EC0002B463A464146304600F0B8FB4FF47A70F4
:107ED00094FBF0F00A2190FBF1F201FB120030302C
:107EE00000F0FF082A464146304600F0BFFA2A4615
:107EF0002E21304600F0BAFA642094FBF0F00A21FB
:107F000090FBF1F201FB1200303000F0FF082A462E
:107F10004146304600F0AAFA0A2094FBF0F00A210C
:107F200090FBF1F201FB1200303000F0FF082A460E
:107F30004146304600F09AFA0A2094FBF0F100FB2B
:107F40001140303000F0FF082A464146304600F02C
:107F50008DFABDE8F0810000340100202DE9F843DE
:107F600007460D4690461E460020374908702C46AD
:107F7000B4F52F7F0ADBA4F52F7406203346424662
:107F800021460090384600F0F5F95BE000202E49CC
:107F90000870C4F52F7442F2107094FBF0F00A21BF
:107FA00090FBF1F201FB120000F0FF09334642465C
:107FB0004946384603F0FCF94FF47A7094FBF0F030
:107FC0000A2190FBF1F201FB120000F0FF09334699
:107FD00042464946384603F0EBF9642094FBF0F042
:107FE0000A2190FBF1F201FB120000F0FF09334679
:107FF00042464946384603F0DBF90A2094FBF0F08C
:108000000A2190FBF1F201FB120000F0FF09334658
:1080100042464946384603F0CBF90B48007820B970
:1080200032462D21384600F021FA0A2094FBF0F167
:1080300000FB1140303000F0FF0932464946384617
:1080400000F014FABDE8F883340100202DE9F04770
:1080500007460D4690461E462C46B4F52F7F08DB9A
:10806000A4F52F74334642462146384600F020F9E5
:108070004FE0002028490870C4F52F744FF47A703F
:1080800094FBF0F00A2190FBF1F201FB120000F0EA
:10809000FF09334642464946384603F089F96420D1
:1080A00094FBF0F00A2190FBF1F201FB120000F0CA
:1080B000FF09334642464946384603F079F91648E7
:1080C000007820B932462D21384600F0CFF90A2039
:1080D00094FBF0F00A2190FBF1F201FB120030302A
:1080E00000F0FF0932464946384600F0BFF93246F3
:1080F0002E21384600F0BAF90A2094FBF0F100FB7B
:108100001140303000F0FF0932464946384600F051
:10811000ADF9BDE8F0870000340100202DE9F047FB
:1081200007460D4690461E462C46B4F52F7F08DBC9
:10813000A4F52F74334642462146384600F0B8F87D
:108140004FE0002028490870C4F52F744FF47A706E
:1081500094FBF0F00A2190FBF1F201FB120000F019
:10816000FF09334642464946384603F021F9642068
:1081700094FBF0F00A2190FBF1F201FB120000F0F9
:10818000FF09334642464946384603F011F916487E
:10819000007820B932462D21384600F067F90A20D0
:1081A00094FBF0F00A2190FBF1F201FB1200303059
:1081B00000F0FF0932464946384600F057F932468A
:1081C0002E21384600F052F90A2094FBF0F100FB12
:1081D0001140303000F0FF0932464946384600F081
:1081E00045F9BDE8F0870000340100202DE9F04199
:1081F00006460C4617461D4600202C49087042F2E0
:10820000107094FBF0F00A2190FBF1F201FB1200D8
:1082100000F0FF082B463A464146304600F00EFA81
:108220004FF47A7094FBF0F00A2190FBF1F201FB1D
:10823000120000F0FF082B463A464146304600F057
:10824000FDF9642094FBF0F00A2190FBF1F201FBB0
:108250001200303000F0FF082A464146304600F058
:1082600005F92A462E21304600F000F90A2094FB39
:10827000F0F00A2190FBF1F201FB1200303000F027
:10828000FF082A464146304600F0F0F80A2094FBE9
:10829000F0F100FB1140303000F0FF082A46414663
:1082A000304600F0E3F8BDE8F08100003401002022
:1082B0002DE9F04106460C4617461D4600202C4984
:1082C000087042F2107094FBF0F00A2190FBF1F27A
:1082D00001FB120000F0FF082B463A4641463046AB
:1082E00000F0ACF94FF47A7094FBF0F00A2190FBA7
:1082F000F1F201FB120000F0FF082B463A4641461E
:10830000304600F09BF9642094FBF0F00A2190FBCA
:10831000F1F201FB120000F0FF082B463A464146FD
:10832000304600F08BF90A2094FBF0F00A2190FB14
:10833000F1F201FB1200303000F0FF082A464146FE
:10834000304600F093F82A462E21304600F08EF891
:108350000A2094FBF0F100FB1140303000F0FF08E0
:108360002A464146304600F081F8BDE8F081000021
:10837000340100202DE9F04707460C4690461E4682
:10838000089D002037490870062D0FDB364894FB06
:10839000F0F00A2190FBF1F201FB120000F0FF095E
:1083A000334642464946384600F048F9052D10DB71
:1083B00042F2107094FBF0F00A2190FBF1F201FB05
:1083C000120000F0FF09334642464946384600F0A5
:1083D00035F9042D10DB4FF47A7094FBF0F00A218C
:1083E00090FBF1F201FB120000F0FF093346424618
:1083F0004946384600F022F9032D0FDB642094FB38
:10840000F0F00A2190FBF1F201FB120000F0FF09ED
:10841000334642464946384600F010F9022D0FDB3C
:108420000A2094FBF0F00A2190FBF1F201FB12000C
:1084300000F0FF09334642464946384600F0FEF850
:10844000012D0CDB0A2094FBF0F100FB11403030D1
:1084500000F0FF0932464946384600F007F8BDE80B
:10846000F087000034010020A086010070B50646A8
:108470000C46154626B1012E07D0022E0FD109E079
:108480002946204600F00EF809E02946204600F073
:1084900043F804E02946204600F08AF800BF00BFF8
:1084A00070BD00002DE9F04105460E46002706B1DB
:1084B000FF27202D00DA202500241EE01348007835
:1084C000802818DA124801781048007801F0D6FEAA
:1084D000A5F120000F4B03EBC000005D80EA07020E
:1084E0000A4800788111012002F0FEFD074800785B
:1084F000401C06490870601CC4B2082CDEDB03482F
:108500000078801E01490870BDE8F0813501002027
:1085100036010020941902082DE9F04105460F4666
:108520004FF000080FB14FF0FF08202D00DA202592
:1085300000242DE0002622E01A48007880281CDA6A
:10854000194800782044C1B21648007801F096FE20
:10855000A5F12000154B03EB401006EB0413C05CA3
:1085600080EA08020F4800788111012002F0BCFD6A
:108570000C480078401C0B490870701CC6B2102EC5
:10858000DADB08480078103806490870601CC4B26D
:10859000022CCFDB034800780B3002490870BDE89D
:1085A000F081000035010020360100209C200208E7
:1085B0002DE9F04106460F464FF000080FB14FF08D
:1085C000FF0800242BE0002520E0194800788028CF
:1085D0001ADA184800782044C1B21548007801F032
:1085E0004DFE154800EBC61005EB4413C05C80EA55
:1085F00008020F4800788111012002F075FD0C4837
:108600000078401C0A490870681CC5B2202DDCDBCC
:1086100007480078203806490870601CC4B2042C52
:10862000D1DB03480078163001490870BDE8F081BD
:108630003501002036010020BC3C02082DE9F04144
:1086400007460C4615461E4614B90B48007850B133
:1086500001200949087004F13000C1B232463846A1
:10866000FFF704FF05E025B1324620213846FFF729
:10867000FDFEBDE8F08100003401002010B5044685
:108680002448006800EB4000234941F82040611E67
:1086900001EBC10101EB410101F16C0000F0F4FAC2
:1086A0001C49096801EB41011B4A02EB810148604A
:1086B000611E01EBC10101EB410101F1860000F0F7
:1086C000E3FA1449096801EB4101134A02EB810105
:1086D000886010480068401C142190FBF1F201FBF7
:1086E00012000C490860084600680C490968884275
:1086F0000ED10221012001F037FD06480068401E1E
:108700000449086008460068002801DA1320086060
:1087100010BD0000CC000020E40D0020C8000020A7
:10872000034A516821F44041014351607047000001
:1087300000100240044A0029516901D0014300E0C1
:10874000814351617047000000100240044A002933
:10875000D16901D0014300E08143D161704700003D
:1087600000100240044A0029916901D0014300E051
:1087700081439161704700000010024010B500F085
:1087800035F84FF4803000F0C3F800F029F91649AD
:10879000087008460078012824D11020FDF73AFB24
:1087A0000220FDF743FB002000F0A8F8002000F0B5
:1087B000E5F84FF4806000F0D7F84FF44040FFF741
:1087C000AFFF00214FF4803000F0E8F8012000F006
:1087D000DFF800BF392000F079F80028FAD0022035
:1087E00000F0F4F810BD0000900000200B48016874
:1087F00041F0010101604168094A1140416001688E
:10880000084A11400160016821F48021016041683B
:1088100021F4FE0141600021816070470010024098
:108820000000FFF8FFFFF6FE224A10B55168224B08
:1088300011F00C0103D0042903D0082903D00360F0
:1088400015E01E4912E05168022301F4701103EB98
:108850009141536813F4803F04D053689B0303D5C0
:10886000174B02E0174B00E0144B5943016051686D
:10887000154B01F0F00109095C5C0168E1404160C1
:10888000546804F4E064240A1C5D21FA04F4846052
:10889000546804F46054E40A1B5DD940C160526816
:1088A000094B02F44042920B1B1F9A5CB1FBF2F1A0
:1088B000016110BD0010024000127A0040787D0175
:1088C00020BCBE0000093D00EA4D0308024600201E
:1088D00053090949012B0BD0022B0BD0D1F82410DE
:1088E00002F01F02012393400B4200D00120704789
:1088F0000968F5E7096AF3E700100240034A516886
:1089000021F0F00101435160704700000010024067
:108910000B490A6822F480320A600A6822F4802235
:108920000A60B0F5803F07D0B0F5802F03D108680A
:1089300040F4A02008607047086840F48030F9E7F0
:108940000010024070470000064900220A7001F83A
:108950002029012802D0042802D1052081F8200016
:108960007047000020100240034A516821F4E06182
:1089700001435160704700000010024003494A68FB
:1089800022F4605242EAC000486070470010024082
:10899000014908667047000000004242034A5368DC
:1089A000084323F47C1318435060704700100240C2
:1089B00001490860704700003C04424202490A6ACB
:1089C00002430A627047000000100240034A5168E7
:1089D00021F0030101435160704700000010024084
:1089E00030B50B4C40F2FF153120FFF76FFF2070C0
:1089F0006068401C6060207810B96068A842F3D1BC
:108A00003120FFF763FF002800D0012030BD0000B7
:108A1000B80300207047000002490A8882430A8098
:108A2000704700000428004010B54FF47A7400BF6E
:108A300001214FF0C050FFF789FE0120FEF78CFBAB
:108A40000120FFF781FF2848046042F21070844241
:108A500001DA04F5FA7400BF4120FFF737FF18B9B7
:108A6000214800680028F7D14120FFF72FFFE8B91F
:108A70000020FFF769FF0020FEF76EFB00214FF09A
:108A8000C050FFF763FE4FF480611848FDF77FFC8C
:108A90004FF4FA701449086000BF134800680028BA
:108AA000FBD14FF480611148FDF76FFC4120FFF7C7
:108AB0000DFF0028BCD04FF48070FFF77FFF01202E
:108AC000FFF776FF00F0D4F800F0CAF8012108465D
:108AD00000F04AF800F0C4F847F6FF7000F0B0F874
:108AE00000F0BEF810BD000018000020000C01408E
:108AF0000248018841F010010180704704280040BD
:108B00000248018821F010010180704704280040CC
:108B1000034800880249091F098840EA014070475C
:108B20001C28004006490988054A0140121FC9B2A5
:108B30001288024202D009B101207047002070471C
:108B40000428004010B50120FFF7ECFF48B100F009
:108B500087F80120FFF760FF02480068401C0149C8
:108B6000086010BD04000020044A0029118801D0CB
:108B7000014300E08143118070470000002800405D
:108B800010B501214FF0C050FFF7E0FD0120FEF7C6
:108B9000E3FA0420F8F7FCFD4AF2A55188422FD0F1
:108BA000FFF742FF00F05CF84AF6C00000F038F82A
:108BB00000F056F84AF2A5510420F8F7EFFD002125
:108BC0000820F8F7EBFD00210C20F8F7E7FD002165
:108BD0001020F8F7E3FD00211420F8F7DFFD002155
:108BE0001820F8F7DBFD00211C20F8F7D7FD002145
:108BF0002020F8F7D3FD00212420F8F7CFFD0DE069
:108C00004120FFF763FE08B9FFF70EFF00F030F8D0
:108C100001210846FFF7A8FF00F022F810BD000070
:108C200000B50246FFF764FF0449100C0880081DD8
:108C300002805DF804EBFFF763BF000018280040D6
:108C400000B50246FFF754FF0449C2F30340088011
:108C5000081D02805DF804EBFFF752BF08280040B2
:108C6000024801888906FCD57047000004280040AE
:108C70000448018821F00801018001880907FCD51A
:108C8000704700000428004010B50446204600F05C
:108C9000CBF810BD70B54FF4C970FFF7F5FF05466E
:108CA000002D01DB322D00DB0025681E051E00DAD9
:108CB00031252C4602221848016818480068FAF746
:108CC00015F900BF04F29310FFF7DEFF064601F02E
:108CD00009F82C2000F0AEFF04F2C510FFF7D4FF16
:108CE000064600F0FFFF2C2000F0A4FF04F2F7106E
:108CF000FFF7CAFF064600F0F5FF641E002C00DAFD
:108D00003124AC4202D02C2000F094FFAC42D9D1E7
:108D1000FAF70CF970BD0000E0000020E40000202C
:108D200070B520480078D0B100BFFEF713F80446B4
:108D3000FAF7DCF9FEF70EF80546FAF7D7F9FEF771
:108D400009F80646FAF7D2F9AC42EED1B442ECD1BA
:108D50000CB1002070BD002012490870FAE700BF76
:108D6000FDF7F8FF04460CB90020F3E7FAF7BEF967
:108D7000FDF7F0FF0546FAF7B9F9FDF7EBFF0646F8
:108D8000FAF7B4F9AC42EBD1B442E9D1054804702A
:108D900034B14FF41670044908600120034908609B
:108DA0002046D7E7A800002028030020E802002082
:108DB00070B504460D464FF480411848FDF7E7FAB8
:108DC00024B980211648FDF7E0FA03E08021144819
:108DD000FDF7DDFA25B140211248FDF7D8FA04E08D
:108DE0004FF400410D48FDF7D2FA20210B48FDF762
:108DF000CEFA0B48FDF7B8FA0646360A2021074896
:108E0000FDF7C3FA40210748FDF7BFFA4FF40041D0
:108E10000248FDF7BAFA304670BD0000000C014070
:108E200000180140000801402DE9F04706460027E0
:108E3000B500C5F30749ADB24FF0030800BF0024E9
:108E40002946484605F0B8FBF0B105F087FAA121A4
:108E500001EB4901C8B205F031FC0746A7B105F0A6
:108E600019F8044605F03EF805F014F800EB042468
:108E700005F038F805F00EF800EB042405F032F8A0
:108E800005F008F800EB042405F078FA27B9A8F1FA
:108E9000010000F0FF0801E04FF00008B8F1000FFA
:108EA000CDDC2046BDE8F08710B51848006820B139
:108EB000012807D0022817D109E01448006804F0FF
:108EC000B9FC15E01148006804F0B4FC10E010494A
:108ED0000E4A126831F81200FDF73CFB0D490B4AAF
:108EE000126841F8220003E000200849086000BF32
:108EF00000BF06480068401C044908600846006836
:108F0000022801DD0020086010BD0000C000002024
:108F10003C0D0020B00B0020F0B502460B460024AB
:108F20000FE0174901EB021516490E680968491C44
:108F3000144F3960A85DF8F721FC04EB840100EBC5
:108F400041040F4800EB02100E490968405C98424A
:108F500013D00B4800EB02100A490968405C302826
:108F60000BDB074800EB021006490968405C392812
:108F700003DC044800681328D3DB2046F0BD000062
:108F8000FC1F0020F400002070B505460E460024AA
:108F900004E0FF2000F09EFF2855641CB442F8D383
:108FA000012070BD10B580210148FDF7EEF910BD1C
:108FB0000014014010B580210148FDF7E8F910BD0B
:108FC0000014014010B580210348FDF7E0F980212D
:108FD0000148FDF7DAF910BD0010014010B510216D
:108FE0000148FDF7D2F910BD0014014010B5102161
:108FF0000148FDF7CCF910BD0014014010B54FF445
:1090000000610248FDF7C1F910BD0000000C0140ED
:1090100010B54FF400610248FDF7B9F910BD00002A
:10902000000C014010B540210148FDF7AEF910BD1C
:109030000010014010B540210148FDF7A8F910BD0E
:109040000010014010B54FF480710248FDF79DF902
:1090500010BD00000010014010B54FF480710248AF
:10906000FDF795F910BD00000010014010B54FF458
:1090700000610248FDF789F910BD000000140140AD
:1090800010B54FF400610248FDF781F910BD0000F2
:109090000014014010B54FF400710248FDF775F956
:1090A00010BD00000010014010B54FF400710248DF
:1090B000FDF76DF910BD00000010014010B54FF430
:1090C00080610248FDF761F910BD00000014014005
:1090D00010B54FF480610248FDF759F910BD00004A
:1090E0000014014010B54FF400610248FDF74DF93E
:1090F00010BD00000008014010B54FF400610248A7
:10910000FDF745F910BD00000008014010B54FF40F
:1091100000510248FDF739F910BD0000000C014074
:1091200010B54FF400510248FDF731F910BD0000B1
:10913000000C014010B54FF480510248FDF725F9AD
:1091400010BD00000008014010B54FF480510248E6
:10915000FDF71DF910BD00000008014010B54FF4E7
:1091600080510248FDF711F910BD0000000C0140CC
:1091700010B54FF480510248FDF709F910BD000009
:10918000000C0140F0B507460C461646B44201D12A
:109190002046F0BDA01900EBD0714D1005EB450045
:1091A000084901EB80004068B84205DD3246691C81
:1091B0003846FFF7E7FFECE72A4621463846FFF737
:1091C000E1FFE6E7B00B020870B50246002000237D
:1091D00017E000EB4004304D55F82440944206D18E
:1091E00000EB400405EB840464688C4206D000EB7D
:1091F0004004294D05EB8404A4680CB9012300E068
:10920000401C192801DA002BE3D0E3B300EB400443
:10921000214D05EB8404A468022C3BD123E0441CBF
:1092200004EB44041C4D55F8244000EB40051A4E55
:1092300046F82540441C04EB4404354605EB840401
:10924000646800EB400506EB85056C60441C04EB8C
:109250004404354605EB8404A46800EB400506EBA6
:109260008505AC60401C1828D9DB002400EB4005C4
:10927000094E46F8254000EB400506EB85056C607D
:1092800000EB400500E005E006EB8505AC6001243D
:10929000024D2C7070BD0000100C00203F0100201A
:1092A000002010E0002100EB4002084B03EB82029B
:1092B000916000EB400243F8221000EB400203EB08
:1092C00082025160401C1928ECDB7047100C002012
:1092D0000021074A1170002004E00021054A1154C2
:1092E000411CC8B20828F8DB0021034A11707047FE
:1092F0003D0100204101002040010020002014E039
:10930000002100EB40020A4B43F8221000EB400220
:1093100003EB8202516000EB400203EB820291609A
:10932000044A1160044A1160401C1428E8DB7047AD
:10933000E40D0020C8000020CC00002070B50E48CD
:109340000068FCF7B7FD04460B480068FCF794FD85
:10935000054601222946204601F068FE06490968B3
:10936000491C054A08461160FDF7D4FC10B10020E5
:109370000149086070BD00002000002070B539A1CF
:109380003948F7F7E0F839490860084600680028CE
:1093900067D04FF480613648FCF7F9FF012035496A
:1093A000087000F0DDFF03220421084600F0F4FFFE
:1093B00005220621042000F0EFFF2AE0002400250A
:1093C0002D48005D2A2822D008E02B48005D05EBDF
:1093D000850100EB4100A0F13005641C2648005DCA
:1093E0003D28F2D1641C002608E02348005D06EB0E
:1093F000860100EB4100A0F13006641C1E48005DB0
:109400000A28F2D100223146284601F00FFEFDF76E
:10941000CBF816481E2102681748F7F71FF80028F6
:10942000CCD1FDF7C1F811480068F7F7B3F8FDF7A4
:10943000BBF812490C4803F0ADFBFDF7B5F841F25B
:1094400088300F49086001E0FDF7AEF80C4800686D
:109450000028F9D107490870FDF720FD01200949CE
:10946000087070BD72000000BC4D0308AC03002002
:10947000000C0140D8000020D04B0020D14D030843
:10948000180000203F01002070B5E5E000F0ACFBC3
:10949000044674480078062870D2DFE800F0031410
:1094A000384C70B3012C0DD1C8206F4908600120E1
:1094B0006C49087000206D4908606D4908602046BD
:1094C00000F0DEFBC7E0204600F0DAFB2C2C16D1C2
:1094D00001266520FFF7D8FB064665480068B042C4
:1094E00002D06348006818B902205E49087002E0A3
:1094F00000205C49087000205E49086006E02146B3
:109500005B480068F8F724F959490860A3E0204651
:1095100000F0B6FB2C2C06D1032052490870002025
:109520005549086006E0214652480068F8F710F9EE
:10953000504908608FE0204600F0A2FB022C15D1B4
:1095400004204849087000204C4908604C490860D4
:10955000002508E000214B48484A126800EB021041
:109560004155681CC5B2102DF4DB06E02146424887
:109570000068F8F7EDF8404908606CE067E02046C5
:1095800000F07EFB032C06D1052036490870002030
:109590003D49086035E02C2C20D138480068401C3B
:1095A0003649086008460068642803DB08460068FE
:1095B000401E0860002032490860002508E00020B5
:1095C00030492E4A126801EB02114855681CC5B299
:1095D000102DF4DBC8202449086012E029482749EF
:1095E000096800EB011026490968445424480068C2
:1095F000401C2349086008460068122801DD12203B
:10960000086028E0042C13D11F4800681749096836
:10961000884209D14FF416701C49086000F038F8F0
:1096200000201049087011E000200E4908700DE07C
:10963000154800680001144908602046F9F79EF8B3
:109640001149098889B208430F49086003E00020E6
:109650000449087000BF00BF00F0DEFA00287FF464
:1096600015AF70BD0B010020FC00002000010020A0
:10967000E0000020E4000020E8000020EC000020D2
:10968000F0000020FC1F002004010020F800002052
:109690002DE9F047FC4800680E2878D009DC0C283A
:1096A00049D2DFE800F048174849788BCC48484851
:1096B000FEFD65286CD006DC0F286AD0102869D022
:1096C000642838D1B2E1662876D0672875D068283A
:1096D000F7D129E20222ED480168ED480068F9F768
:1096E00005FC002400BF0020EA4908600021204654
:1096F000FFF712FC80464046FCF702FC002806DB20
:109700004046FCF79FFE054600F0ECFA05E02D20F0
:1097100000F090FA312000F08DFADF4800688442B2
:1097200002DA2C2000F086FA641CDB4800688442D0
:10973000D9DDF9F7FBFB16E20222D4480168D448D0
:109740000068F9F7D3FBD5480078D54909788842F5
:1097500006D12D2000F06EFA312000F06BFA13E0F4
:10976000CF4805780CE0681CC5B2142D00DB00253D
:10977000CC4951F8250000F0B5FA2C2000F05AFA37
:10978000C6480078A842EED1F9F7D0FBEBE109E139
:1097900096E134E146E1C1480078C14908700222EF
:1097A000BA480168BA480068F9F7A0FB302000F019
:1097B00041FAF9F7BBFBD6E192E195E100250222DF
:1097C000B2480168B2480068F9F790FBB6480078E3
:1097D00030B92D2000F02EFA312000F02BFA1BE0DA
:1097E00016E0B24951F8350000F07CFA2C2000F068
:1097F00021FAAE4901EBC501486800F073FA681C14
:10980000C5B2A9480078854202DA2C2000F012FA8D
:10981000A54800788542E4DBF9F788FB002508E0DD
:109820000020A24941F8350001EBC5014860681CE1
:10983000C5B2782DF4DB00209B49087093E1002528
:1098400002229248016892480068F9F74FFB984855
:10985000007830B92D2000F0EDF9312000F0EAF960
:109860001BE016E0934951F8350000F03BFA2C203C
:1098700000F0E0F98F4901EBC501486800F032FAC9
:10988000681CC5B28A480078854202DA2C2000F0B4
:10989000D1F9874800788542E4DBF9F747FB01E01E
:1098A0007FE010E0002508E00020824941F8350003
:1098B00001EBC5014860681CC5B2782DF4DB0020BF
:1098C0007B4908704FE10024A1467B4800780028BE
:1098D00054D100BF002600206E4908603D2120467B
:1098E000FFF71AFB80466B480068401C6949086016
:1098F0004046FCF705FB002839DB4046FCF700FB3F
:1099000040B900212046FFF707FB0646304600F02D
:1099100099FC2EE04046FCF7F3FA1B2829D00021E1
:109920002046FFF7F9FA06464046FCF7E9FA0546F5
:10993000FDF7D6F9E8B14046FCF7E2FA0546FCF738
:10994000AFFAB04202DD49F0020912E04046FCF7EE
:10995000D7FA0546FCF79AFAB04202DA49F0040950
:1099600007E000223146404601F060FB01E049F08B
:109970000109641C484800688442ABDD4348006824
:1099800070B114224148016841480068F9F7AEFA05
:109990004949097809EBC10000F0A4F9F9F7C6FAC2
:1099A000E1E0E0E00024002717E0002039490860EA
:1099B00000212046FFF7B0FA404941F83700641C07
:1099C00000203449086000212046FFF7A5FA3B49F2
:1099D00001EBC7014860641C7F1C2F48006884426B
:1099E000E3DB09E00020354941F837000022384622
:1099F0007F1C01EBC0004260192FF3DBB3E00020B5
:109A00002449086000210846FFF786FA8046404650
:109A1000FCF718FD012804D101220221404601F083
:109A200005FBA0E000201B4908609CE000201949CC
:109A3000086000210846FFF76FFA804600201549AC
:109A4000086000210120FFF767FA0646FA2E00DDC4
:109A5000FA2602220D4801680D480068F9F746FA17
:109A6000C24600250AE01AF8010B00F03BF9701E0F
:109A7000A84202DD2C2000F0DDF86D1CB542F2DBBF
:109A8000F9F754FA6FE00000E8000020E000002041
:109A9000E4000020F4000020EC000020250000205D
:109AA00024000020E00300200901002030040020F1
:109AB0000A010020F00700200C010020240F0020E4
:109AC00000202A49086000210846FFF725FA2849A6
:109AD00008600846006810B101202649087042E07D
:109AE0000020244908703EE0002020490860002141
:109AF0000846FFF711FA18B1A0F2E73090B902E07A
:109B0000FFF7C8F80EE0F7F769FF02221A4801686C
:109B10001A480068F9F7EAF9002000F0E3F8F9F7CD
:109B200005FA00BF00BF1EE0022213480168134877
:109B30000068F9F7DBF9122000F0D4F82C2000F0CF
:109B400079F86420FFF7A0F8054600F0CBF82C2048
:109B500000F070F86520FFF797F8054600F0C2F8AE
:109B6000F9F7E4F900BF00BFBDE8F087F40000207A
:109B7000D4000020D8000020E0000020E4000020F5
:109B800010B50020114908601149086011490860AA
:109B900011490860114908704FF4164010490860D7
:109BA00000208880C880088188810C2048810D4869
:109BB00001F07EF8012240F225510A4801F05FF8D9
:109BC0000121084801F032F810BD00001401002006
:109BD000100100201C010020180100200B010020B2
:109BE000EC0F00200044004000BF08480068084A0D
:109BF00012689042F9D005480068401CC0F30A0181
:109C0000024801600348405C7047000014010020D6
:109C100010010020FC0F0020044800680449096876
:109C2000884201D0012070470020FCE7100100208D
:109C30001401002070B505460D480068401CC0F3B3
:109C40000A0400BF0B4800688442FBD00A4805554F
:109C500007480460284600F013F8012240F22771FB
:109C6000064801F00CF80121044800F0DFFF70BD48
:109C7000180100201C010020FC17002000440040B7
:109C800007490988C1F307214140064A32F82110EB
:109C9000034A127881EA022189B2014A11607047B1
:109CA000000100209415020810B5044604F13000AC
:109CB000C4B2392C01DDE01DC4B22046FFF7BAFF63
:109CC00010BD000010B50446002C02DD012004493F
:109CD00008700348007810B12046FFF7E5FF10BD7B
:109CE0000801002070B5044600203E490870002C91
:109CF00000DA00243C4894FBF0F00A2190FBF1F2DA
:109D000001FB1200C5B22846FFF7DCFF374894FB81
:109D1000F0F00A2190FBF1F201FB1200C5B22846D7
:109D2000FFF7D0FF324894FBF0F00A2190FBF1F2EC
:109D300001FB1200C5B22846FFF7C4FF2D4894FB73
:109D4000F0F00A2190FBF1F201FB1200C5B22846A7
:109D5000FFF7B8FF284894FBF0F00A2190FBF1F2DE
:109D600001FB1200C5B22846FFF7ACFF42F21070AB
:109D700094FBF0F00A2190FBF1F201FB1200C5B256
:109D80002846FFF79FFF4FF47A7094FBF0F00A210A
:109D900090FBF1F201FB1200C5B22846FFF792FFDB
:109DA000642094FBF0F00A2190FBF1F201FB120019
:109DB000C5B22846FFF786FF0A2094FBF0F00A217F
:109DC00090FBF1F201FB1200C5B22846FFF77AFFC3
:109DD0000A2094FBF0F100FB1140C5B22846FFF7C2
:109DE00063FF70BD0801002000CA9A3B00E1F50541
:109DF0008096980040420F00A086010010B50446EE
:109E0000C4F30330FFF750FFC4F30320FFF74CFF08
:109E1000C4F30310FFF748FF04F00F00FFF744FFFF
:109E200010BD000010B540210248FCF7B0FA02F066
:109E300087F910BD000C014010B540210248FCF725
:109E4000A4FA02F07DF910BD000C014010B580218C
:109E50000748FCF79CFA8020064908800320887098
:109E60000420C8700248FCF70DFA02F069F910BD31
:109E7000000C01402C01002010B58020074908800B
:109E8000032088701420C8700548FCF7FBF9802176
:109E90000348FCF77AFA02F053F910BD2C010020B8
:109EA000000C01407047704770477047704710B50D
:109EB0000446204600F00EF810BD70B505460E466B
:109EC000002403E0285D00F005F8641CB442F9D3D7
:109ED000012070BD2DE9F04105462E4600240027E3
:109EE00025E006F0800028B94FF480511248FCF7B5
:109EF0004CFA04E04FF480510F48FCF748FA700622
:109F0000060E4FF480610C48FCF741FA6006040E1F
:109F10004FF400610848FCF72AFA08B144F0010444
:109F20004FF480610448FCF730FA781CC7B2082F60
:109F3000D7DB2046BDE8F08100100140014609B1A1
:109F4000102001E04FF48010014A1060012070479A
:109F5000100801402DE9F04104460D46164605F172
:109F60008600FEF791FE80460C4850F8240098B910
:109F700016B9601CFEF782FB05F17000FEF784FE47
:109F8000C0EB001106FB08F0C0EB8107474500DA83
:109F90004746024840F82470BDE8F081E80B0020F5
:109FA0000021024A42F8201070470000E80B002010
:109FB0002DE9F84F05460C46164604F18600FEF7DB
:109FC00063FE81466B20FEF75FFE009004F16D009A
:109FD000FEF75AFE83461E480068584535DB1D488B
:109FE00050F8250088BB04F17100FEF74DFE824653
:109FF00004F17000FEF748FE0746009858441449E3
:10A000000968884206DC06FB09F0CAEB0A11C0EBBE
:10A01000810810E00E480068A0EB0B00AAEB0701D6
:10A020004843009990FBF1F03844C0EB001106FB67
:10A0300009F0C0EB8108C84500DAC84616B9681CAB
:10A04000FEF71CFB034840F82580BDE8F88F0000B0
:10A0500034000020E80B00202DE9FC5F05460E4689
:10A06000174606F18600FEF70FFE82466B20FEF7CC
:10A070000BFE019006F16E00F7F716FE00900098B7
:10A0800000283DD006F16D00FEF7FEFD04461D4898
:10A090000168A14234DB1C4850F8250080BB0099C0
:10A0A000C81CFEF7F1FD83460099881CFEF7ECFD05
:10A0B00081460198204413490968884206DC07FB61
:10A0C0000AF0CBEB0B11C0EB81080FE00D480068E4
:10A0D000001BABEB09014843019990FBF1F04844A8
:10A0E000C0EB001107FB0AF0C0EB8108D04500DA95
:10A0F000D04617B9681CFEF7C1FA034840F825801E
:10A10000BDE8FC9F34000020E80B00202DE9F0475B
:10A1100004460D46164605F18600FEF7B5FD80465D
:10A1200005F16E00F7F7C0FD8146B9F1000F17D0B9
:10A130000C4850F8240098B916B9601CFEF79EFA36
:10A1400009F10200FEF7A0FDC0EB001106FB08F0CC
:10A15000C0EB8107474500DA4746024840F82470C3
:10A16000BDE8F087E80B002070B502460020002310
:10A1700017E000EB40042F4D55F82440944206D1DF
:10A1800000EB400405EB840464688C4206D000EBCD
:10A190004004284D05EB8404A4680CB9012300E0B9
:10A1A000401C192801DA002BE3D00BB300EB40046C
:10A1B000204D05EB8404A468022C1AD11E4C24689F
:10A1C000B4B900EB400445F8242000EB400405EB53
:10A1D00084046160012400EB4005164E06EB850502
:10A1E000AC60164C2468112C22D10124144D2C7023
:10A1F0001EE000EB40040F4D05EB8404A468012C25
:10A2000016D000EB400445F8242000EB400405EB99
:10A2100084046160012400EB4005064E06EB8505D1
:10A22000AC60064C2468112C02D10124044D2C7022
:10A2300070BD0000100C0020A4000020D0020020FF
:10A240003F01002010B50446FEF7EEFBFEF708FDC7
:10A25000C4EB04118800FEF7E3FCFEF701FD4AF2AF
:10A26000A5510420F7F79AFAFEF752FC3C21B0FB07
:10A27000F1F00149086010BD3000002070B50446BF
:10A280000D4600F03CFE04F03F0000F14002A11139
:10A29000002000F029FF00F032FE05F1B802A11104
:10A2A000002000F021FF00F02AFEC0220021084615
:10A2B00000F01AFFC0220121002000F015FF70BD40
:10A2C00070B50025202600216C20FCF74DF92148AF
:10A2D000006800283DD14FF496701E4908600024A4
:10A2E0001CE004EB44001C4901EB8000406898B17D
:10A2F00004EB440001EB80008068022802D1012DAC
:10A3000000DA012504EB4400134901EB800080686A
:10A31000012802D1022500E01924641C192CE0DB7D
:10A32000012D02D0022D0ED101E096260BE00B4844
:10A33000007820B9962601200849087002E0002024
:10A340000649087000BF00BF012231461046FEF7E3
:10A350008DF870BDC8020020100C0020F40200200F
:10A3600010B5FCF79BFDFCF7DDFD002004490870EB
:10A3700004490870012204A1104600F0A7FF10BD97
:10A3800035010020360100202020204452414D4D4F
:10A39000202020200000000070B504460D4616461F
:10A3A00005490D7005490C7006F1AD0100221046FB
:10A3B00000F038FF70BD000036010020350100209C
:10A3C0002DE9F0412148006800283CD14FF4AF70DE
:10A3D0001E4908601E48007818B901201C49087001
:10A3E00002E000201A4908704FF4BD70FEF74CFCE3
:10A3F0000446012C01DA3C2604E03C2090FBF4F0FA
:10A40000801EC6B200251CE012480068401EA8420B
:10A4100004D10F48007808B9E32700E0DF27C5EB37
:10A420000510C00090FBF4F000EB06080721404641
:10A43000FCF79AF8002239461046FEF717F8681C18
:10A44000C5B2A542E0DBBDE8F08100003801002084
:10A45000F60200203800002070B5FCF763FD0020F4
:10A460004249087042490870012242A1104600F09A
:10A470002DFF10203D49087004203D49087000223E
:10A4800040A1104600F022FF062039490870222022
:10A49000364908706420FEF7F7FB04460022562177
:10A4A0001046FDF7E3FF3B4894FBF0F03030C5B2B7
:10A4B000002229461046FDF7D9FF42F2107094FBA6
:10A4C000F0F00A2190FBF1F201FB12003030C5B22E
:10A4D000002229461046FDF7C9FF00222E21104612
:10A4E000FDF7C4FF4FF47A7094FBF0F00A2190FB63
:10A4F000F1F201FB12003030C5B2002229461046AD
:10A50000FDF7B4FF642094FBF0F00A2190FBF1F218
:10A5100001FB12003030C5B2002229461046FDF77B
:10A52000A5FF00222E211046FDF7A0FF0A2094FB74
:10A53000F0F00A2190FBF1F201FB12003030C5B2BD
:10A54000002229461046FDF791FF0A2094FBF0F106
:10A5500000FB11403030C5B2002229461046FDF7FD
:10A5600085FF42F210700C49086070BD3501002073
:10A57000360100202020204452414D4D2020202033
:10A58000000000002020204D6973742D54696D6512
:10A5900020202000A08601001400002070B5044691
:10A5A00000256720FEF770FB06283FD2DFE800F0A9
:10A5B000030C16202A3404EB44011E4A52F83100E1
:10A5C000F6F70EF8054631E004EB4401194A02EBB8
:10A5D000C1014868F6F704F8054627E004EB44019A
:10A5E000144A02EBC1018868F5F7FAFF05461DE041
:10A5F00004EB44010F4A02EBC101C868F5F7F0FF14
:10A60000054613E004EB44010A4A02EBC101086964
:10A61000F5F7E6FF054609E004EB4401054A02EBC5
:10A62000C1014869F5F7DCFF054600BF00BF2846B9
:10A6300070BD00001447020810B500F035F810BDD9
:10A640004FF0E021012804D0801C06D00020886152
:10A650007047086940F0010002E0086920F001003D
:10A66000086170474FF0E0210028086902D040F0EF
:10A67000020001E020F002000861704710B541F6C9
:10A680006A0000F00DF80120FFF7ECFF0120FFF752
:10A69000D7FF14200149086010BD000014000020FD
:10A6A0004FF0E0214861704710B54E48006820B176
:10A6B0004C480068401E4B4908604B48006828B170
:10A6C00049480068401E4849086003E04FF47A702A
:10A6D000454908604548007870B143480068C82182
:10A6E00090FBF1F201FB1200642805DD4FF480714C
:10A6F0003F48FBF74CFE04E04FF480713C48FBF709
:10A7000044FE3C48006820B13A480068401E394980
:10A7100008603948006820B137480068401E364953
:10A7200008603648006820B134480068401E33494C
:10A7300008603348006820B131480068401E304945
:10A7400008603048006820B12E480068401E2D493E
:10A7500008602D48007820B12B480078401E2A4917
:10A7600008702A48007820B128480078401E274900
:10A7700008702748007820B125480078401E2449F9
:10A7800008702448007820B122480078401E2149F2
:10A7900008702148006828B11F480068401E1E4903
:10A7A000086002E000201D4908701D48006828B1BB
:10A7B0001B480068401E1A49086002E00020194941
:10A7C00008701948006820B117480068401E1649F3
:10A7D00008601648006820B114480068401E1349FC
:10A7E000086010BD2001002014000020D8000020C7
:10A7F00000080140180000209C030020A403002052
:10A80000A8030020A0030020000000200100002079
:10A810000200002003000020FC0000200B010020AB
:10A82000900300205203002038010020C8020020BD
:10A830007047704770477047704770477047704760
:10A840007047704770477047704770477047000007
:10A850002DE9F0419948007808B1FCF71DFF002070
:10A860009649087000212820FBF77EFE0123002274
:10A87000934801681846FDF7B9FA4FF4C170FEF726
:10A8800003FA40B303210846FBF76EFE00221E21A7
:10A89000104600F0C7FC8B480068FBF7D4FA8046EE
:10A8A00000231A4641461846FDF7D0FB40F27B10C4
:10A8B000FEF7EAF928B900221146104600F0B2FC72
:10A8C00004E000220F21104600F0ACFC0022202101
:10A8D0001046FDF7CBFD04210320FBF745FE7A4827
:10A8E0000068002875D00022B321104600F09AFCC1
:10A8F00076480078801E75490870734800680B28F8
:10A900004DD2DFE800F04C060D141B222930373EF3
:10A910004500002240F287111046FCF748FF3EE058
:10A9200000224FF4C4711046FCF741FF37E00022CB
:10A9300040F289111046FCF73AFF30E000224FF454
:10A94000C5711046FCF733FF29E0002240F28B115D
:10A950001046FCF72CFF22E000224FF4C67110468F
:10A96000FCF725FF1BE0002240F28D111046FCF79A
:10A970001EFF14E000224FF4C7711046FCF717FFCA
:10A980000DE0002240F28F111046FCF710FF06E0A8
:10A9900000224FF4C8711046FCF709FF00BF00BF4A
:10A9A000002220211046FDF761FD48480078801EF6
:10A9B0004649087046480068062823D2DFE800F0C0
:10A9C00022030A10161C0022B521104600F02AFCB2
:10A9D0001EE01EE00022B621104600F023FC17E026
:10A9E0000022B721104600F01DFC11E00022B82122
:10A9F000104600F017FC0BE00022B921104600F0D1
:10AA000011FC05E00022B521104600F00BFC00BF50
:10AA10000DE03048006828B10022BA21104600F04D
:10AA200001FC04E00022BB21104600F0FBFB04E027
:10AA3000002220211046FDF719FD244800787828CF
:10AA4000F6DD4FF4BD70FEF71FF90446092C01DD59
:10AA5000092600E0E6B2012C01DA3C2704E03C20A4
:10AA600090FBF4F0401EC7B2002513E0C5EB0510C3
:10AA7000C00090FBF4F000EB070806214046FBF70E
:10AA800073FD05F13100C1B200221046FDF7EEFC66
:10AA9000681CC5B2B542E9DB0A2C0DD106216E2037
:10AAA000FBF762FD002231211046FDF7DFFC00229A
:10AAB00030211046FDF7DAFCBDE8F0813F010020AF
:10AAC0003000002034000020380000203501002034
:10AAD0003C0000208C000020704770477047000049
:10AAE00070B540F227711E4800F0AAF8C8B11D48A1
:10AAF00000681D49096888420CD01B480068401C4A
:10AB0000C0F30A041948015D154800F01BF9164806
:10AB1000046005E0002240F22771114800F0AFF810
:10AB200000BF40F225510E4800F08AF8B8B10C4839
:10AB300000F004F9C5B20E480068401CC0F30A04D6
:10AB40000B4804600B480068844202D101200A4986
:10AB500008700A48055564200949086000BF70BDA7
:10AB600000440040180100201C010020FC170020B8
:10AB700010010020140100200C010020FC0F002017
:10AB8000FC00002070B540F227711F4800F058F813
:10AB9000C8B11E4800681E49096888420CD01C488C
:10ABA0000068401C00F01F041A48015D164800F0C0
:10ABB000C9F81748046005E0002240F227711248E6
:10ABC00000F05DF800BF40F225510F4800F038F862
:10ABD000C0B10D4800F0B2F8C5B20F480068401C83
:10ABE000C0F308040C4804600C480068844202D199
:10ABF00001200B4908700B4805554FF47A700A493B
:10AC0000086000BF70BD00000048004048030020FD
:10AC10004C03002088310020400300204403002022
:10AC200053030020882F00209003002000298189F1
:10AC300002D041F4005101E021F4005181817047BC
:10AC400070B501F01F0601220025C1F3421302FA7C
:10AC500006F4012B0FD0022B0FD0838A4FEA11216B
:10AC60000088234202FA01F200EA020001D000B19A
:10AC70000125284670BD8389F0E7038AEEE710B509
:10AC8000C1F3421301F01F040121A140012B07D0A1
:10AC9000022B07D01430002A026805D00A4304E0D2
:10ACA0000C30F8E71030F6E78A43026010BD000070
:10ACB00030B50446008A85B00D464CF6FF71084059
:10ACC000E98801432182A1894EF6F3100140A8884A
:10ACD0002A8910436A890A431043A081A08A4FF64B
:10ACE000FF410840A9890143A1826846FDF79CFD08
:10ACF0001148844201D1039800E00298642200EBDD
:10AD0000C00101EB001029686FF018058900B0FB45
:10AD1000F1F0B0FBF2F109010B096B4300EB83008A
:10AD2000322303EB0010B0FBF2F000F00F000843F9
:10AD3000208105B030BD0000003801408088C0F39C
:10AD400008007047C1F30801818070477047704761
:10AD500070470120704700002D2802D08D2842D175
:10AD60002EE022490968042914DA20490968491C9F
:10AD70001E4A11601E490968126811441D4A02EBFF
:10AD800001110968491CD1B918490968491E174AB7
:10AD9000116014E016490968491C154A11601146F2
:10ADA0000968124A12681144124A02EB011109683B
:10ADB000491C21B90E490968491E0D4A116012E06B
:10ADC0000A49096829B109490968491E074A1160F9
:10ADD00008E007490968002904DD05490968491E9A
:10ADE000034A116000BF00BF70470000300100201F
:10ADF000BC020020582C00204FF6FF72904216D063
:10AE000042F21072904212DB520090420FDA084A6E
:10AE10001278521CD1B2142900DB0021054A1278A5
:10AE2000914204D0044A42F82100014A117070474F
:10AE30002500002024000020E003002000BFFEE7E2
:10AE400070B502460020002317E000EB4004174DC8
:10AE500055F82440944206D100EB400405EB8404ED
:10AE600064688C4206D000EB4004104D05EB84046E
:10AE7000A4680CB9012300E0401C192801DA002B5A
:10AE8000E3D093B100EB4004084D05EB8404A468C3
:10AE9000012C0AD1022400EB4005044E06EB850587
:10AEA000AC604FF49674024D2C6070BD100C002005
:10AEB000A400002010B50D4A12680D4B1B681A44FF
:10AEC00002EB42020B4B03EB82025168074A126805
:10AED000074B1B681A4402EB4202064B53F8220050
:10AEE000FFF7AEFF01200449087010BD08030020E1
:10AEF00030010020100C00203F010020704770B589
:10AF000000BF00210846FDF753FFC5B20121002014
:10AF1000FDF74EFFC4B2802D02D00DB1FCF702F850
:10AF2000802C02D00CB1FBF7FDFF05F0800000285B
:10AF3000E7D104F080000028E3D170BD10B515E022
:10AF4000FBF732FB0D480068C82190FBF1F201FBD2
:10AF50001200642805DA4FF480610948FBF717FAFC
:10AF600004E04FF480610648FBF70FFA03480068DD
:10AF700018B1FDF7D5FE0028E2D010BD1400002066
:10AF8000000C01402DE9F04107460D4690461C4655
:10AF9000069E01201A490870E2B220210020FDF728
:10AFA00065FA042016490870E2B220210020FDF75E
:10AFB0005DFA012D02D0022D0CD105E0E2B2BC21D8
:10AFC000002000F02FF905E0E2B2BD21002000F0E2
:10AFD00029F900BF00BF04E0E2B220210020FDF704
:10AFE00045FA074800787828F6DB7720044908708E
:10AFF000E2B220210020FDF739FABDE8F08100001F
:10B000003501002070B505460C462846FDF73CFE8C
:10B01000A04209D02946204600F0C0F82846FAF799
:10B0200053FF0646FFF7E8FE70BD00002DE9F04132
:10B0300005460C4616461548854225DA2846FAF795
:10B040005FFF0746FBF740FEA0B12846FBF7E4F997
:10B050000746FDF719FEA04216D02846FBF7DCF99B
:10B0600007463946204600F099F86EB12846FFF7AA
:10B07000C3FE09E02846FAF743FFC0EBC0000449CD
:10B0800001EB800040680460BDE8F08178D40300E3
:10B0900058E901082DE9F04105460F4616464FF4E0
:10B0A000C970FDF7F1FD0446002C01DB322C00DDF8
:10B0B000002404F293102946FFF7A4FF04F2C51000
:10B0C0003946FFF79FFF04F2F7103146FFF79AFF6A
:10B0D000641C322C00DB002421464FF4C970FFF7BA
:10B0E00091FFBDE8F0810000F8B505460E46174611
:10B0F0004FF480412648FBF748F925B980212548BF
:10B10000FBF743F903E080212248FBF740F926B121
:10B1100040212148FBF73BF904E04FF400411C4873
:10B12000FBF735F920211A48FBF731F94FF47F403E
:10B13000ADF8000010208DF8030003208DF8020008
:10B1400069461448FBF79EF81248FBF70DF90446D0
:10B15000E4B244EA0724A1B20E48FBF71AF9202111
:10B160000B48FBF712F940210B48FBF70EF94FF49F
:10B1700000410748FBF709F94FF47F40ADF80000A4
:10B1800028208DF8030069460248FBF77BF8F8BDDC
:10B19000000C014000180140000801402DE9F04773
:10B1A000074688464FEA8806C6F3074AB6B23D46C8
:10B1B0004FF0030903F0BEF900BF002431465046AA
:10B1C00003F0FAF9A0B1280E03F078FA044624B18E
:10B1D000C5F3074003F072FA044624B1C5F3072013
:10B1E00003F06CFA04461CB1E8B203F067FA0446B7
:10B1F00003F0C4F824B9A9F1010000F0FF0901E04F
:10B200004FF00009B9F1000FD7DC03F089F90448C9
:10B210000068401C024908602046BDE8F087000035
:10B220002401002070B505460C4616466720FDF740
:10B230002BFD062845D2DFE800F0030D18232E3938
:10B2400004EB4400204A52F830103246284600F001
:10B250003DF836E004EB44001B4A02EBC0003246E6
:10B260004168284600F032F82BE004EB4400164A0F
:10B2700002EBC00032468168284600F027F820E043
:10B2800004EB4400104A02EBC0003246C168284675
:10B2900000F01CF815E004EB44000B4A02EBC00080
:10B2A00032460169284600F011F80AE004EB440038
:10B2B000054A02EBC00032464169284600F006F814
:10B2C00000BF00BF70BD0000144702082DE9F04127
:10B2D00006460C46174666E0207823285DD1641C9C
:10B2E0002078A0F13005641C207805EB850100EB87
:10B2F0004100A0F13005641C0B2D4DD2DFE805F0B4
:10B300004C060D141B222930373E45003A4640F2C8
:10B3100087113046FCF74BFA3EE03A464FF4C471D1
:10B320003046FCF744FA37E03A4640F2891130469D
:10B33000FCF73DFA30E03A464FF4C5713046FCF771
:10B3400036FA29E03A4640F28B113046FCF72FFAE4
:10B3500022E03A464FF4C6713046FCF728FA1BE06B
:10B360003A4640F28D113046FCF721FA14E03A4695
:10B370004FF4C7713046FCF71AFA0DE03A4640F236
:10B380008F113046FCF713FA06E03A464FF4C871C5
:10B390003046FCF70CFA00BF05E014F8011B3A46F2
:10B3A0003046FDF763F82078002895D1BDE8F0819C
:10B3B0002DE9F04107460C4615461E461148007817
:10B3C00038B104F13000C1B232463846FDF74EF8CC
:10B3D00016E07CB101200B49087032462D21384619
:10B3E000FDF744F804F13000C1B232463846FDF7AB
:10B3F0003DF805E025B1324620210020FDF736F862
:10B40000BDE8F0813401002070B504461148AFF367
:10B410000080114904EBC40001EB80040026208861
:10B420004FF0FF358107002906D00ADA8006204652
:10B4300004D501F072F903E02C4604E000F0ECFEC4
:10B4400030B1268000240348AFF30080204670BD51
:10B450002680F1E7000000003C26002010B50446DD
:10B460000C48AFF300800C4904EBC40001EB8004EE
:10B470002088810703D0800603D5A46805E0002456
:10B4800003E0204600F0C1FE64680248AFF300808C
:10B49000204610BD000000003C2600202DE9F843A6
:10B4A00006460F466648AFF30080684601F048FC48
:10B4B00004004FF0FF3575D00146304601F08EFC98
:10B4C000814620690028F6D017F00C0004D004282B
:10B4D0000AD0082866D103E0208840F0010006E089
:10B4E000208840F004002080208840F00200208066
:10B4F00017F0060F04D0484601F010FC002851D187
:10B500002088DFF8408180064FF000064BD52146A9
:10B51000484600F015FF012803D02088C00772D1EB
:10B5200033E000214848C4461BE000BFB0F800806B
:10B530005FEA887213D0026923699A420FD1A04250
:10B540000DD0C28AE38A9A4209D1026A236A9A42DA
:10B5500005D15FEA887270D4228892076DD4491CA5
:10B560002430BCF800209142E0DB208810F0050F69
:10B5700006D0B9075AD500BF40F00B00208055E037
:10B580002146484600F077FEE8B3208810F0060F09
:10B5900004D02146484600F043FEA0B3B80745D585
:10B5A0002088E9E743E0B80741D42146484600F047
:10B5B0002AFE012803D02088C0073ED130E00021B8
:10B5C0002148424617E000BFB0F800C05FEA8C7324
:10B5D0000FD003692769BB420BD1A04209D0838AEF
:10B5E000A78ABB4205D15FEA8C7326D423889B07C8
:10B5F00023D4491C243013889942E5DB2088410775
:10B6000005D5204600E018E000F0FFFD0EE0C00781
:10B6100002D0E069206209E0204600F0F0FD60B150
:10B62000A6822146484600F0E8FD30B1009D04485E
:10B63000AFF300802846BDE8F8832680F7E70000D6
:10B6400000000000BC4602083C2600202DE9F04125
:10B6500007460E4615461348AFF3008045F00044F8
:10B66000CEB1114907EBC70001EB800001888A07C2
:10B6700011D001F00F02022A06D089062A4631466F
:10B6800005D500F06BFF04E04FF0FF3403E000F05D
:10B69000BDFD00B12C1A0348AFF300802046BDE881
:10B6A000F0810000000000003C26002070B5044638
:10B6B0000D460E48AFF300800D4904EBC40001EBCA
:10B6C00080004FF0FF3401888A070AD08906294696
:10B6D00002D500F0E5FF01E000F09CFD012800D15B
:10B6E00000240248AFF30080204670BD0000000037
:10B6F0003C2600202DE9F04107460D46164611482C
:10B70000AFF300804FF0FF34B5B10F4907EBC7002E
:10B7100001EB800001888A070ED001F00F02012A98
:10B720000AD089063246294602D501F071F801E0B7
:10B7300000F074FD00B100240248AFF30080204601
:10B74000BDE8F081000000003C26002030380A28C7
:10B7500001D2012070470020704710B50446B4F5AF
:10B76000004F01DD002010BD2046FFF74DFEFAE737
:10B7700000BFFEE710B50446B4F5004F01DD002020
:10B7800010BD2046FFF76AFEFAE70146B1F5004F0B
:10B7900001DD012070470020FCE7000070B5044681
:10B7A0000D460EA12046F5F707F810B948F2010042
:10B7B00070BD0CA12046F4F7FFFF10B948F202005B
:10B7C000F6E70AA12046F4F7F7FF10B948F20300A4
:10B7D000EEE729462046FFF761FEE9E75354444966
:10B7E0004E0000005354444F5554000053544445F8
:10B7F000525200002DE9F04104460D4616461F4600
:10B80000B4F5004F03DD4FF0FF30BDE8F081324664
:10B8100029462046FFF71AFFF7E770B504460D46A4
:10B82000B4F5004F02DD4FF0FF3070BD29462046D1
:10B83000FFF73CFFF9E72DE9F04104460D461646B7
:10B840001F46B4F5004F03DD4FF0FF30BDE8F08137
:10B85000324629462046FFF74DFFF7E770470000C4
:10B860000021094A1268094B1B68D01800E0491CE6
:10B87000074A02EB01121268521C002AF7D18842D3
:10B8800000DB401A70470000BC020020300100209D
:10B89000582C00202DE9F84F05464FF00009C869E3
:10B8A00000900C460127C8464E46284600F0E9F8AD
:10B8B000012808D12846F4F793FE0C300D21B0FB87
:10B8C000F1F0401CC7B22069009901F052FB82469A
:10B8D0000025206990F87B1019B1B5F5007F56D08E
:10B8E0002AE0818FA94227D1016C009A002591425C
:10B8F00000D900916946009E02F0CCFC002847D098
:10B900002069009901F04AFE88B10096012269463B
:10B91000206900F048F800283AD02069009900F02A
:10B9200043F9002834D04FF00008009E34E020692D
:10B93000009900F05BF982460AEB1511206902F0CC
:10B9400033FB002824D02069C16D05F00F0001EB06
:10B950004010007838B1FF2805D0E52803D04FF01B
:10B9600000096D1CB5E7B9F1000F02D1009E1FFA66
:10B9700085F809F10101C9B28946E5280AD0206994
:10B9800090F87B0040B1C7F50070A84204D20020B7
:10B99000BDE8F88FB942E4D12169A1F87880206927
:10B9A00046670120F4E72DE9F041154607460C46AD
:10B9B0000E6801F00DFB002818D0384601F059FA46
:10B9C00002463846216802F007FF00280ED035B144
:10B9D00031463846226802F0FFFE002806D00021DA
:10B9E000384600F005F8002800D00120BDE8F081BD
:10B9F00070B50446806C0D46A8423ED094F85010B5
:10BA0000012928D166697EB1216889060CD5617F3C
:10BA1000022906D0002201463046E36C01F027FAE5
:10BA200014E0218C4218F6E76268E16CD3680122C9
:10BA30009847002820D0607F022809D16268218CB5
:10BA4000A06CD3680844E16C01229847002813D009
:10BA5000002084F8500085B194F85100218C626870
:10BA6000484328449368E16C01229847012806D096
:10BA70004FF0FF30A064002070BD012070BDA564B0
:10BA8000FBE72DE9F04100270446B8463D463E4617
:10BA900025E002F027FD38B32078202824D02E2876
:10BAA00014D0A0F16101192902D92031192907D830
:10BAB000B8F1000F03D088EA0001890614D480464B
:10BAC0004FB13046761C02280ED806E067B9641CD8
:10BAD0000026012703E0082D06D26D1C641C207887
:10BAE0000028D6D10C2D02D30120BDE8F081002022
:10BAF000FBE7012302F0BEBAF8B5C1690446009124
:10BB000000293DD0206900F071F807460025206922
:10BB1000818FA9420FD10025694602F0BBFB0028A6
:10BB20002FD02069009901F039FD58BB2069009998
:10BB300000F05CF8074607EB1511206902F034FAB3
:10BB400000281ED0206905F00F01C06D00EB4116E2
:10BB500030782E2809D10CA13046F4F72DFE68B1BB
:10BB60000DA13046F4F728FE40B1307850B1E528F9
:10BB700004D0F07A0F2803D0000701D56D1CC6E76A
:10BB80000020F8BD0120F8BD2E20202020202020FC
:10BB900020202010000000002E2E20202020202019
:10BBA000202020100000000070B5054600F01EF8AF
:10BBB00006464FF40071E86DF4F7B4FD002406E08A
:10BBC0003119284602F02CFD00280AD0641CA87FF9
:10BBD000A042F5D80021284602F022FD002800D01E
:10BBE000012070BD10B5FBF759F910BD838E826935
:10BBF0001A44037F032B01D0C38E1A44807F891E11
:10BC000000FB012070472DE9F0410446007F00252C
:10BC1000012806D0022838D0032857D00020BDE8DC
:10BC2000F08102262CE03146204601F0B8F980462A
:10BC300001462046FFF7DCFE002867D006EB4600F1
:10BC4000C0F34800B0F5FF7F04D8E16C084401F070
:10BC50002DFC0CE0E06C08F1010190F8FF7120462A
:10BC6000FFF7C6FE88B3E06C007847EA0020F107D2
:10BC700001D0000901E0C0F30B0000B96D1C761C77
:10BC8000206B801CB042CED840E00221204601F05B
:10BC900086F9074601462046FFF7AAFEA8B102260C
:10BCA0000FE016F0FF0F05D17F1C39462046FFF745
:10BCB0009FFE50B1E06CF1B230F8110000B96D1C7C
:10BCC000761C206B801CB042EBD81FE0022120467E
:10BCD00001F065F9074601462046FFF789FEA8B145
:10BCE00002260FE0700605D17F1C39462046FFF77B
:10BCF0007FFE58B1E06C06F07F0150F8210000B9DA
:10BD00006D1C761C206B801CB042EBD8284686E761
:10BD10002DE9F04389B00E46904699460546FFF757
:10BD2000B0FE88B301271B4C1CE04246314604A8F4
:10BD3000FFF7DFFE28B1A74214D9002009B0BDE803
:10BD4000F083694604A800F0ACF90028F6D06846F4
:10BD500001F040FC02463146284600F01DF800285C
:10BD6000ECD007E03A467F1C04A9284601F0BEFA51
:10BD70000128DAD04B4642463146684600F0B0F81A
:10BD80000028DBD00120D9E7FFE76946284600F00C
:10BD900088F9E4E73E420F002DE9F74F086982B0C9
:10BDA0000C46416F0091B0F878504FF0000B0298AC
:10BDB000F4F716FC81462069009901F0DAF8824612
:10BDC000D846464E7DE0206990F87B1031B1B5F53C
:10BDD000007F1DD1002005B0BDE8F08F818FA94202
:10BDE00016D1016C009A0025914200D900910122E0
:10BDF0006946FFF7D8FD0028EDD020690099FFF7CC
:10BE0000D3FE0028E7D020690099FFF7EFFE8246B5
:10BE10000AEB15110191206902F0C6F80028DAD06A
:10BE2000206905F00F010D22C06DBBF1000F00EB82
:10BE3000411109F10C00B0FBF2F0C0B2087001D062
:10BE4000002200E0402210430870049A4A73A1F8CF
:10BE50001A800F2200F01F00CA72401E00EB800201
:10BE600002EBC000029A4FF0010B131800204A1C8D
:10BE70001F5C4FB116F800C001F80C70375C401C15
:10BE80000D2807F80280F3D3002305E0375CCB557B
:10BE9000375CBB54FF23401C0D28F7D3B9F10C0FBE
:10BEA00002D9A9F10D0000E000208146E843000717
:10BEB00006D101222069019902F036FD00288AD0BE
:10BEC0006D1CB9F1000F7FF47EAF216900984867BF
:10BED0002069A0F8785001207DE70000964E030805
:10BEE0002DE9FC5F06460D469A46012A0DD000203A
:10BEF00081462869416F0091B0F8787090F87B20F6
:10BF000042B1B7F5007F02D018E00120F0E7002031
:10BF1000BDE8FC9F828FBA4210D1026C00278A4292
:10BF200000D9009201226946FFF73DFD0028EFD0BD
:10BF300028690099FFF738FE0028E9D028690099A0
:10BF400001F017F800EB17118B46286902F02CF866
:10BF50000028DDD0286907F00F01C06D00EB411407
:10BF60000020315C2154401C0B28FAD35FEA0A0000
:10BF70004FF0000837D00646C07AE07284F80C8093
:10BF800084F80D80F089E081308A208200F0DBFFA8
:10BF9000014604F1120002F0C3F9B08AA08201F058
:10BFA0006DFA014604F1160002F0BAF9608A2083A6
:10BFB000708B6083F069E061F0696860F069C5E9E1
:10BFC000020806F11A0001F071FA044606F11400A5
:10BFD00001F06CFA04EB0040E8610122594628693F
:10BFE00002F0A2FC56E084F80C8084F80D8001F089
:10BFF00045FA014604F10E0002F092F900F0A3FFA9
:10C00000014604F1100002F08BF9208A6082E18978
:10C01000E1822083C4F81C80C5F80C80C5F8048038
:10C02000C5F80880B9F1000F1ED01020E072009909
:10C0300001912869006C884200D90190002201A971
:10C040002869FFF7B0FC00283FF462AF0198E8616F
:10C05000010C04F1140002F063F9019881B204F1BB
:10C060001A0002F05DF907E02020E072A4F81480C5
:10C07000A4F81A80C5F81C8001225946286902F0EC
:10C0800053FC0028E0D0B9F1000F05D028690199D0
:10C09000FFF78AFD0028D7D0EF82009828620120A0
:10C0A00036E72DE9F041002704460D4638462021A9
:10C0B0002954401C0B28FBD3002129542078617897
:10C0C000A2782E2806D111B12E2902D002E02870C4
:10C0D00031E0AAB10026207868B32E2813D020289A
:10C0E0000AD002F0F6F9A0F16101A855192902D889
:10C0F00020F02000A855761C641C082EEBD304E029
:10C100002870687017E00127641C0826207890B119
:10C110002E2813D020280BD057B102F0DAF9A0F165
:10C120006101A855192902D820F02000A855761CD5
:10C13000641C0B2EEAD30120BDE8F0810127F7E74C
:10C140000649096809B9052101E04FF4FA6108467A
:10C1500000BF011EA0F10100FBD1704728010020A3
:10C160002DE9F8430546006990F87A60416F009127
:10C17000B0F8784000F0FDFE07463AE0286990F8F4
:10C180007B1029B1B4F5007F15D10020BDE8F883FC
:10C19000818FA1420FD1016C009A0024914200D9F5
:10C1A0000091694602F076F80028EFD028690099DE
:10C1B000FFF71CFD074607EB14118846286901F0BC
:10C1C000F3FE0028E2D0286904F00F01761EC06D4E
:10C1D000F6B200EB4110E5210170E043000700D00A
:10C1E00036B901224146286902F09EFB0028CDD0D5
:10C1F000641C002EC2D10120C8E700207047002037
:10C20000704700207047002070477047002070473B
:10C2100000207047002070470020704700207047C2
:10C2200070B505460C460869142100F049FD002848
:10C2300020D028785C2800D16D1C2878002819D0DF
:10C240000020E06101222146284600F09FF80028E6
:10C2500010D0206921467C30FFF71CFB002809D054
:10C26000206900237C301A462146FFF751FD002843
:10C2700000D0012070BD70B505460C460869142138
:10C2800000F01EFD002838D028785C2800D16D1CF5
:10C290002878002831D000200246E0612146284657
:10C2A00000F074F8002828D0206990F87C1029B19B
:10C2B0007C300022214600F01DFC02E02046FFF702
:10C2C0001BFC002819D02046FFF74AFF002814D095
:10C2D000E169206902F060F800280ED02069017F32
:10C2E000032909D102F0ECFA002806D000212069C8
:10C2F00002F096F9002800D0012070BD70B5044608
:10C300000E4615460421106900F0DAFC002816D00C
:10C3100020785C2800D1641C207800280FD00020F1
:10C320000246E8612946204600F030F8002806D091
:10C330002946304600F0FAFE002800D0012070BDEA
:10C3400070B505460C460869042100F0B9FC0028C8
:10C350001BD028785C2800D16D1C2878002814D0C8
:10C360000026324621462846E66100F00FF80028F4
:10C370000BD0206900227C30214600F0BBFB002856
:10C3800003D06675E069A061012070BD2DE9F0471A
:10C39000002706460D469146B84620E0286901224E
:10C3A0007C30294600F0A6FBC0B95FEA09002DD019
:10C3B0000127286929467C30FFF76CFA002825D030
:10C3C000286900237C3001222946FFF7A1FC0028C0
:10C3D0001CD0284602F07EF9002817D0264429698F
:10C3E0007C3100242046325D5C2A06D0222A04D00B
:10C3F0004AB10A54401C641CF5E7641C01F8008033
:10C40000002FD6D1CAE701F800800120BDE8F087EF
:10C410002DE9F0414FF0FF3500F148048564806854
:10C4200060604FF000062672667200F5007100F53C
:10C430008060E560C4E90510267766774FF0020852
:10C44000C4F82480A4F148044FF0300104F118002E
:10C45000F4F78AF90021204601F0A6FD08B3E06D4B
:10C4600000F5FF7001F022F8A0F52A41553918D1E6
:10C47000E06D0178E9290AD0EB2902D18178902971
:10C4800005D000F5E37001F016F8A06100E0A661A8
:10C49000204600F000FD38B1E18DB1F5007F40D1BC
:10C4A00004E00220BDE8F0810320FBE7A07F08281C
:10C4B0000DD006DC01280AD0022808D0042830D18B
:10C4C00005E0102803D0202801D0402829D1B4F855
:10C4D00022C0BCF1000F24D0627F012A01D0022AC1
:10C4E0001FD1238C666AB3421BD8A78D02FB03C3FE
:10C4F00005EB471505F5007595FBF1F15A18B21AD1
:10C50000A262B2FBF0F22263A386E1864002A0633E
:10C510004009A08740F6F570824204D201202077BE
:10C5200016E00420BEE74FF6F570824202D284F88E
:10C530001C800DE003202077204600F0B7FD38B9BD
:10C540002046FFF760FBA066204602F0B9F908B16B
:10C550000020A7E70520A5E7012070472DE9F04757
:10C560000446008889461746C00613D40421206972
:10C5700000F0A6FB50B1E068A168C2198A4201D957
:10C580000F1A07D0C0F3080600253AE0208840F0D3
:10C59000100020800020BDE8F087A1692069FFF726
:10C5A00025FB627D81182069837F9A1A01F0A4FC23
:10C5B0000028F0D0A7EB050808EB0600B0F5007FD7
:10C5C00001D9C6F5007820694246C06D811909EB92
:10C5D0000500F4F730F806EB0800C605F60D0FD19C
:10C5E000607D401CC1B261752069827F914207D194
:10C5F0000021617504F1180101F04CFE0028CAD039
:10C600004544BD42C9D3E0682844E0602846C2E7FB
:10C6100070B506460C4615461421106900F050FB13
:10C62000002839D030785C2800D1761C20785C282E
:10C6300000D1641C307880B3207870B300200246AB
:10C64000E86129463046FFF7A1FE002824D028697A
:10C6500090F87C0080B10026324629462046FFF73C
:10C6600048FA01281AD0286900227C30294600F0B7
:10C6700041FA002810D007E001263246294620461C
:10C68000FFF737FA012809D032462946204601F043
:10C69000B4FC002800D0012070BDFFE70020FBE7BC
:10C6A0002DE9F041044600880D46C00602D5002061
:10C6B000BDE8F0810421206900F002FB40B3A068CE
:10C6C000A84200D205462069690A827FB1FBF2F3D5
:10C6D00002FB13116175E769A761806BB5FBF0F68A
:10C6E00056B104F118084146A769206901F0D2FD4E
:10C6F0000028DDD0761EF6D1A169206900F04EFF3A
:10C7000018B12069807F6075A7610120E560CFE7DF
:10C71000208840F010002080C9E7F0B5044600886A
:10C7200089B0C0065FD41421206900F0C9FA00283E
:10C7300055D0D4E9010181424CD9491E2046FFF76A
:10C74000AFFF002850D0206900F093FB0246A1699A
:10C75000206902F041F8002846D06946204601F0E1
:10C7600008FC002840D0E069000CADF81400E06936
:10C77000ADF81A00A068079000F080FE01460DF1A8
:10C78000160001F0CDFD00F0DEFB014606A801F029
:10C79000C7FDBDF81800ADF812006F46E58A216AA2
:10C7A000206900F0E6FB00EB15110E46206901F050
:10C7B000FBFBC0B1206905F00F012022C06D00EB2A
:10C7C00041103946F3F77CFF01223146206902F01F
:10C7D000ABF840B12069017F032907D00AE0208827
:10C7E00040F010002080002009B0F0BD02F068F891
:10C7F0000028F9D00021206901F012FF0028F3D0B1
:10C8000000212069FFF7F4F80028EDD00120EBE7C4
:10C810002DE9F74F0446008882B01746C00603D5BD
:10C82000002005B0BDE8F08F1421206900F048FA1F
:10C8300060B121884FF4007909EA811B04F11800E6
:10C84000E1694FF0000A009029B10EE0208840F025
:10C8500010002080E4E72069009900F0B9FB00286F
:10C86000DFD0A069E06184F815A0E0680025C0F37E
:10C8700008064CE02069617D827F914218D1E16811
:10C88000A2682944914203D2009901F003FD0BE014
:10C89000D4F81880009900F09BFB0028C1D04146D5
:10C8A000A269206901F098FF0028BAD084F815A089
:10C8B000A1692069FFF79AF9617D084401900EB9DA
:10C8C0005F4505D22069019901F06EFB0028A8D0D0
:10C8D000A7EB050808EB0600484501D9C6F5007826
:10C8E0000398424641192069C06D3044F3F7A3FE16
:10C8F0002069019901F094FE002892D006EB08000F
:10C90000C605F60D02D1607D401C60754544BD42F0
:10C91000B0D3E0682844E060A168884200D9A060F4
:10C9200001207EE72DE9F05F05460C466848AFF32D
:10C930000080002000F004FA060055D00146284689
:10C9400000F04CFA8246306900284DD00020514654
:10C95000024604E0401C5C2B00D10246491C0B78C7
:10C96000002BF7D10AEB020083465AA1F3F724FF0C
:10C9700000B32A21584600F06DFA05465846F3F7F1
:10C980002FFE8046681C1AD04FF001090BEB050002
:10C9900051A1F3F711FF18B1A8EB0500A0F10100B8
:10C9A0008046308880060DD5324621465046FFF736
:10C9B000A5FC0BE000254FF00109A846F1E74FF078
:10C9C0000009EEE731462046FFF71BFC60B100206E
:10C9D00084F8FF00B9F1000F08D055EA08001FD015
:10C9E000CDB35946002349E001242EE023465A46A0
:10C9F00010E05B1C12F8011BA0F16107192F01D890
:10CA000020F02000A1F16107192F01D821F02001A9
:10CA10008842C6D118780028EBD111780029E8D1D6
:10CA20003088800603D5307D84F8060109E00020B7
:10CA300084F80601F082B4F80401B0823046FFF7B2
:10CA4000E4FB7068C4F8000100242148AFF30080C3
:10CA50002046BDE8F09F13E011F8012BE05CA2F145
:10CA60006107192F01D822F02002A0F16107192FC8
:10CA700001D820F02000824293D15B1CAB42EBDB5B
:10CA8000B8F1000FCCD02046F3F7AAFD844605EBA1
:10CA90000801614585DC0BEB05035B1CACEB080270
:10CAA00012E000BF13F8010BA15CA0F16107192F80
:10CAB00001D820F02000A1F16107192F01D821F041
:10CAC00020018842A5D1521C6245EBDBA8E700009B
:10CAD000000000002A2E2A002E2A000001680029EA
:10CAE00001DCF4F7FEB8491E016041684A1C42604F
:10CAF00008787047002301F0BDBA0000F0B5044685
:10CB000089B01A48AFF3008000F0AAF8BCB1002049
:10CB1000ADF8000004906946204600F05FF90498E3
:10CB200008B3BDF8000000F02001049800F0CEFC2E
:10CB300004460E48AFF3008009B02046F0BD002443
:10CB40000B4D26460B4F0AE0E87900F004012868F7
:10CB500000F0BCFCA04200DD0446761C0835388895
:10CB60008642F1DBE5E70324E3E700000000000074
:10CB7000D8460208BE4602088A68002A01DCF4F79B
:10CB8000A3BA521E8A604A68C0B2531C4B60107030
:10CB900070470000F0B5044695B00F462F48AFF33C
:10CBA0000080002000F0CCF805004ED00146204661
:10CBB00000F014F90646286980B3288880062ED52F
:10CBC0003046F3F70DFD441E06D4305D5C2802D0DC
:10CBD000641EFAD500E06CB1621C31466846F3F77A
:10CBE0002AFD0DEB04010020487039466846F3F732
:10CBF00016FD07E03846F3F7F3FC0246394668466F
:10CC0000F3F719FD29466846FFF79AFB01281CD067
:10CC10002A4639463046FFF7FBFC14E015E029466A
:10CC20003846FFF7F0FA01280FD029463046FFF7C3
:10CC3000EAFA50B1284600F0A7F8012805D02946A5
:10CC40003846FFF7E5FA012806D001240348AFF380
:10CC5000008015B02046F0BD0024F7E7000000007A
:10CC600070B5124C207800281ED100F041F8002247
:10CC70000F4811460F4B05E0C5796D0750F8085B6A
:10CC8000521C29601D88AA42F6D300200A4B0B4A89
:10CC900005E000BF00EBC005401C23F825101588F7
:10CCA000A842F7D30120207070BD0000C00300200F
:10CCB000D8460208BE4602083C260020BC460208B0
:10CCC00010B504460068814301D0002010BD000764
:10CCD00006D460680021426908469047C00701D029
:10CCE000012010BD206820F006002060EDE7000064
:10CCF00007480021A0F58062C0E90221054A426090
:10CD000000F5C073044A9A604161018270470000D7
:10CD1000CC2A0020C0460208F446020860B101781F
:10CD200051B1012100E0491C425C002AFBD10844BA
:10CD300010F8010C5C2801D00020704701207047DA
:10CD400070B5064600240A4D0A4804E02988890780
:10CD500006D02435641C01888C42F7DB002070BDAE
:10CD600024212846F3F700FD06B13460284670BD43
:10CD70003C260020BC460208004870470101DB0742
:10CD80004FF440207047000030B500221149124B8B
:10CD90001AE00C88A40715D0814213D00C690569EC
:10CDA000AC420FD10488A40609D5CC8AC58AAC420E
:10CDB00008D10C6A056AAC4204D1012030BD8C8ACE
:10CDC000858AF8E7521C24311C88A242E1DB00204E
:10CDD00030BD00003C260020BC460208F0B51B4ACE
:10CDE0001B4CE8B10378DBB123F0200643783A2BE3
:10CDF00003D085783A2D03D012E03023801C01E067
:10CE000073B1C01C002507E01779B74202D15779EA
:10CE10009F420AD06D1C08322788BD42F4DBF0BD6A
:10CE200000230EE0D579ED0709D013680B61D279A4
:10CE30005207F4D50A8842F020020A80F0BD5B1C3C
:10CE400008322588AB42EDDBF0BD0000D846020871
:10CE5000BE460208002205E08B4201D11046704711
:10CE6000401C521C0378002BF6D1581E704700203E
:10CE70007047007F012805D0022806D0032807D07C
:10CE80000020704740F6FF7070474FF6FF70704704
:10CE90006FF07040704710B50446816901F084F866
:10CEA000002809D0E06D00F5FF7000F0FFFAA0F552
:10CEB0002A41553901D0002010BDE06D417BA1779A
:10CEC0000B3000F0F3FAE085E06D0E3000F0EEFA82
:10CED0006084E06D017C6177113000F0E7FAA08595
:10CEE000E06D133000F0E2FA6062E06D163000F0A1
:10CEF000DDFA2084616AE9B9B8B9E06D283000F044
:10CF0000D5FAE087E06D2C3000F0D5FA2064E06DB2
:10CF1000303000F0CBFAA4F84400E06D323000F07D
:10CF2000C5FAA4F84600606A20B9E06D203000F030
:10CF3000C2FA6062208C20B9E06D243000F0BBFAA8
:10CF40002084012010BD10B5FFF716FF10F01F015F
:10CF500000D10121C0F303220C2A00D802B901221A
:10CF600041EA4211442202EB104041EA402080B2E3
:10CF700010BD10B5002280F87B2059B90267017FEF
:10CF8000032906D0828E81691144012280F87B201A
:10CF900003E0016CFEF72AFE0146084610BD027F41
:10CFA000012A04D0022A06D0032A0AD105E001EBA7
:10CFB0004101890A02E0090A00E0C909028C8A429B
:10CFC00001D8002070478269408C104408447047A3
:10CFD0002DE9F04105460E46C46E5CE02146284628
:10CFE000FFF7DDFF804601462846FEF701FD0028D9
:10CFF00038D0287F012804D0022823D0032830D13C
:10D0000027E004EB4400C0F34800B0F5FF7F04D8EC
:10D01000E96C084400F04AFA0DE0E86C08F10101FF
:10D0200090F8FF712846FEF7E3FC00281AD0E86C60
:10D03000007847EA0020E10701D000090FE0C0F3C3
:10D040000B000CE0E96C200601EBD05000F02EFA4A
:10D0500005E0E96C600601EBD05000F02CFA18B145
:10D0600018E00020BDE8F0810E48002102880E483B
:10D0700009E003889F0604D59B0702D58369A34274
:10D0800008D02430491C9142F3D33460641C012041
:10D09000EC66E7E7641C286B801CA0429ED8EC6617
:10D0A000DFE70000BC4602083C26002010B504461D
:10D0B0008069B4F844100144204600F075FF002850
:10D0C00029D0E06D00F5FE7000F0F5F914498842B2
:10D0D00020D1E06D00F0EFF9124988421AD1E06DDD
:10D0E00000F5F27000F0E7F90F49884212D1E06DC7
:10D0F00000F5F47000F0DFF9216B81420AD3A066DD
:10D10000E06D00F5F67000F0D6F9022802D3216B2D
:10D11000814201D2002010BDE066012010BD000058
:10D12000000055AA52526141727241612DE9FF5FC0
:10D13000054600200E46029001900390C969814681
:10D1400000913069FFF715FFB5F8047182464FF082
:10D15000000B306990F87B00E0B1B7F5007F10D08C
:10D160001CE07F1A016C009A914200D90091694637
:10D1700001F090F8002805D03069009900F00EFA0F
:10D1800018B1002004B0BDE8F09F30690099FEF7A7
:10D190002DFD82463069818FB942E2D909F101093A
:10D1A0000AEB1711306900F0FFFE0028EAD0306961
:10D1B00007F00F01C06D00EB411420780028E1D08A
:10D1C000E5285AD0E17A0F2902D0080755D407E0A4
:10D1D000400605D5012003900190607B029011E08C
:10D1E000039878B30F290BD000200390204600F05D
:10D1F000F1F90199002975D00299884248D001E0DF
:10D200000198D0B3617B0298814202D00020019046
:10D2100068E02078344B00F01F00401E00EB8001D6
:10D2200001EBC00805EB080100201A5CA25C0A545F
:10D23000401C0D28F9D3207808F10D08400601D5CF
:10D2400005F808B0E07A00F03F000F284AD0072127
:10D2500000E0491E605C2028FBD0491C002002E051
:10D26000225C2A54401C8842FAD3217A20290DD00E
:10D270002E212954401C082103E033E02A54491C84
:10D28000401C625C202A01D00B29F7D305F800B0BE
:10D2900005F58275298801EB09002880E07A307550
:10D2A00004F11C0000F007F97060B06004F1160092
:10D2B00000F0FCF8C10A2971C0F34511C00669717C
:10D2C000800EA87104F1180000F0F0F800F01F01C2
:10D2D000E971C0F34311400A297200F2BC70688101
:10D2E00001204FE77F1C34E7964E03082DE9F84FE5
:10D2F000834660480E4615464FF0000A4FF6FF7809
:10D30000824201DD062713E042F20F70854201DD03
:10D3100005270DE0B5F57A7F01DB042708E0632DD2
:10D3200001DD032704E0092D01DD022700E00127CC
:10D33000002003E02E2900D18046401C1BF800107D
:10D340000029F7D105B94F1E4FF00009C7F10700BA
:10D350004C46009018E000BF1BF809A0BAF1200F5E
:10D3600010D0BAF12E0F0DD0BAF1000F11D0AAF1E2
:10D370006100192801D82AF0200A504601F0A9F8C6
:10D380003055641C09F10109C14502D20098A04240
:10D39000E2D8EDB37E203055641C072F46D2DFE87B
:10D3A00007F04542352A1E12040032483249401C1B
:10D3B00095FBF0F0414305EB4115092800D9092000
:10D3C00030303055641C42F2107095FBF0F06FF471
:10D3D0001C7141433030305505EB0115641C4FF48E
:10D3E0007A7095FBF0F06FF07C014143303030559E
:10D3F00005EBC105641C642095FBF0F06FF018018B
:10D4000041433030305505EB8105641C0A2000E0B3
:10D410000CE095FBF0F04142303001EB81013055DA
:10D4200005EB4105641C30353555641CBAF1000F1D
:10D430001AD02E203055641CA8F57F414046FF3994
:10D4400012D0451C071D0DE01BF8050060B1A0F1CE
:10D450006101192901D820F0200001F03AF8305577
:10D46000641C6D1CBD42EFD3002030550120BDE887
:10D47000F88F00009F860100CBF3FFFF10B5FFF788
:10D480007FFCC0F344011D2900D90021C0F305220F
:10D490003B2A00D90022C0F3044041EA4211172878
:10D4A00000D9172041EAC02080B210BD4178007831
:10D4B00040EA01207047C1788278090641EA0241BA
:10D4C0004278007841EA02210843704710B50446CB
:10D4D00040680022B1B318B12068C00702D00BE049
:10D4E000032010BD2260606801680020884750B3A7
:10D4F000206840F001012160206820F01E012160B9
:10D5000060680021426908469047010603D52068FB
:10D5100040F0180106E0C10738D0800703D4206826
:10D5200040F010012160606801680120884750B117
:10D53000206840F0020120462160FEF769FF18B123
:10D54000022010BD0AE021E0206840F004012046DE
:10D550002160FFF701F8F0B90420F2E768B1206814
:10D56000C0070AD12260D4E90120E169126890471E
:10D5700060B1206840F001002060206840F00400A5
:10D580002060616821B1896811B104E00120D8E709
:10D5900040F0100020600020D3E70000007F012849
:10D5A00004D0022805D003280FD107E040F6F87018
:10D5B00001E04FF6F870814205D206E021F070409C
:10D5C0000349884201D301207047002070470000C2
:10D5D000F8FFFF0F024600200146C30700D080235A
:10D5E00003EB5000535C491C1844C0B20B29F4D320
:10D5F00070470000FBF7C2F8F9F7E8FCF8F794FC75
:10D60000F5F7BEFCFCF7BCFAFDF738F8F3F73EFF80
:10D61000F8F7BAFFFBF7B4FAF8F7E0FFF9F760FCA8
:10D62000F4F750FEF4F74EFE002063490860052031
:10D63000624908604FF41670614908600020614932
:10D64000087061490860012060490860F4F78AFEAB
:10D650006820FBF719FB044640F2E7325C4801689A
:10D660002046FDF717FD42F6A1016420FDF7CAFC34
:10D67000F4F77CFF4FF42F7056490860FCF7ECFE7E
:10D68000F4F7A8FAFDF75AFCF4F742FB00210A2050
:10D69000FDF7B8FC00210B20FDF7B4FC00210C20A5
:10D6A000FDF7B0FCFBF72AFE01204B4908604FF460
:10D6B0002F704A49086048607CE0FBF7E5FEF3F70D
:10D6C000C1FF3E48006810B9012045490870FBF7CA
:10D6D000EBFB3D4800683C490968491C3A4A116027
:10D6E000062836D006DC062845D2DFE800F01316FF
:10D6F0001924272F092835D004DC07282CD0082826
:10D7000039D12CE00A2830D0A0F59850883800286C
:10D7100031D12DE0F4F726FE31E0F4F7B9FA2EE02E
:10D72000F8F7EAFE27480078012803D141F2883053
:10D730002549086023E0F4F797FD20E01F480068C2
:10D7400018B142F210702049086018E0F4F77AFF2F
:10D7500015E0F4F7C3FB12E0F4F7F0FC0FE0F4F788
:10D7600023FB0CE0F4F762F909E0F4F793FA06E022
:10D77000F4F704FC03E000201349086000BF00BF79
:10D7800018480068B0F5FA7F05DA4FF48061164852
:10D79000F8F7FDFD04E04FF480611348F8F7F5FD5C
:10D7A000F5F7D6FDF4F7E2FEF4F78CFDF4F792F905
:10D7B000F8F7FAFE81E7000054000020B0000020D6
:10D7C000F80000203C0100200C0000200400002094
:10D7D00030000020340000204C000020B00B00205E
:10D7E0001000002014000020000C0140014A00F04D
:10D7F0005FB800004C2C0020014900F066B8000022
:10D800004C2C0020014900F05DB900004C2C002098
:10D81000014B00F067B900004C2C0020014900F0DA
:10D820008DB900004C2C0020014B00F093B9000092
:10D830004C2C00202DE9F04107461849184A12687F
:10D8400031F81200F8F746FE0646F8F7A5FD054642
:10D8500014481349096850F821002C1A002C00DAEA
:10D8600064420A2C0EDB10480D490968405C401CDC
:10D87000C0B20D490A4A12688854642802DC0B4879
:10D88000006848B107480649096840F8215000205F
:10D890000549034A12688854BDE8F0813C0D002018
:10D8A000C0000020B00B0020C4000020B000002009
:10D8B00018B1022807D0002070479068C06900B1F5
:10D8C000004780207047506870472DE9F8430C46A8
:10D8D00010B101287DD104E0886800688047BDE868
:10D8E000F883A068816901208847A06841694FF4E6
:10D8F000C87088470025A0688168FF2088476D1C94
:10D90000102DF8D3A06881690020884700222346A3
:10D910001146104600F04CF905460026012D07D0AF
:10D92000A0688168FF208847761C0546642EF5D3E1
:10D93000A068816901208847012DCBD1A068416989
:10D9400044F62060884700202070A068816900208C
:10D95000884704268DF8006023466A464FF4D57147
:10D96000082000F025F901280FD19DF8000060B9CA
:10D970009DF8010048B99DF80200012805D19DF8E5
:10D980000300AA2801D103202070A068816901202A
:10D99000884700254CF25038A068816900208847EC
:10D9A000002223461146372000F002F90746A068FE
:10D9B00081690120884778071AD4012F15D1A06802
:10D9C0008169002088472078032815D0002081072E
:10D9D00000E06EE023460022292000F0E9F8074627
:10D9E000A06881690120884747B16D1C4545D3D3A4
:10D9F0002078032807D01EE00120E8E720780328DC
:10DA000001D0022033E0A0688169002088478DF8AA
:10DA1000006023466A4600213A2000F0C9F8054616
:10DA2000A0688169012088472DB99DF80000400653
:10DA300001D526701CE02078D0B900254746A068A3
:10DA4000816900208847002223461146012000F00A
:10DA5000AFF80646A068816901208847012E01D0F1
:10DA60003EBB03E06D1CBD42E9D322E001202070E3
:10DA7000A068816900208847234600224FF4007186
:10DA8000102000F095F80546A068816901208847BC
:10DA90007DB9A0688169002088470022234611468D
:10DAA0003B2000F085F80546A06881690120884781
:10DAB0000DB1002013E7204600F002F90028F9D04C
:10DAC00001200CE770B505460C46084600F0F8F852
:10DAD000002806D02146284600F017F9002800D07B
:10DAE000012070BD2DE9F041064698680F461546A5
:10DAF00081691C460020884723462A46394630461D
:10DB000000F0A6F80646012D0FD900222346114643
:10DB10000C2000F04DF8084DA0688168FF20884770
:10DB2000FF2802D06D1EF7D10026A0688169012070
:10DB300088473046BDE8F08148E8010038B1012847
:10DB40004FF0000002D108704860012070478868DB
:10DB5000406800472DE9F041064698680F46154693
:10DB600081691C460020884723462A4639463046AC
:10DB700000F046F90646012D11D9A0688168FD2004
:10DB80008847A0688168FF208847084DA0688168A1
:10DB9000FF208847FF2802D06D1EF7D10026A0681D
:10DBA0008169012088473046BDE8F08148E80100DE
:10DBB0002DE9FC4140F040008DF80000080E8DF882
:10DBC0000100080C8DF80200080A8DF803000020FF
:10DBD00014461D468DF804106A46014605234E077B
:10DBE00007D1B3EBD10F04D902EBD106367846EA60
:10DBF0000000060401D580F409404000491C30298A
:10DC0000EDD3000A40F001008DF80500A868816896
:10DC1000FF208847A8680621C26868469047002709
:10DC2000A8688168FF2088470646FF2802D17F1C2C
:10DC3000082FF5D34CB1277805E0A8688168FF204C
:10DC4000884704F8010B7F1EF7D2F0B2BDE8FC81D3
:10DC50002DE9F04111250F4616461C46012A00D930
:10DC600012252178042900D24002014600222846CC
:10DC7000FFF79EFF10BB1CE046F2A815A068816864
:10DC8000FF208847FE2802D06D1EF7D116E0ADB107
:10DC9000A0684FF40071026938469047A068816817
:10DCA000FF208847A0688168FF20884707F5007734
:10DCB000761E002EE0D10120BDE8F0810020FBE7B8
:10DCC0007FB504468068816900208847234610227A
:10DCD00069460A2000F06CF80546A06881690120B9
:10DCE000884775B12078012868460CD00930016852
:10DCF000C07809BA21F0FF0101430120616004B03E
:10DD000070BD0020FBE70A30F1E77FB50446886864
:10DD10000D468169002088472B461022694609205C
:10DD200000F046F80646A868816901208847B6B128
:10DD30009DF80500012100F00F0001FA00F0A0801D
:10DD4000BDF80C0040BAC0F383108140E1809DF81B
:10DD50000000800906D0012819D0022802D0002036
:10DD600004B070BD9DF806009DF80710000440EA5D
:10DD700001209DF808100843BDF80910C0F38B106E
:10DD800049BAC1F3C211401C891C88400DE09DF8BE
:10DD900007009DF80810000440EA01209DF80910D2
:10DDA00008430004800900F5806020600120D7E767
:10DDB0002DE9F04117460E4600221C461146FFF79A
:10DDC000F7FED8B946F2A815A0688168FF208847F9
:10DDD000FE2802D06D1EF7D110E07DB1A068394653
:10DDE000026930469047A0688168FF208847A06894
:10DDF0008168FF2088470120BDE8F0810020FBE713
:10DE00002DE9F0411826884615461C46012A00D9FE
:10DE100019262178042900D240020146002230460A
:10DE2000FFF7C6FE38BBFE27012D29D9FC2727E0C6
:10DE3000A068816838468847A0684FF40071C268BE
:10DE400040469047A0688168FF208847A0688168A5
:10DE5000FF208847A0688168FF20884700F00F00F6
:10DE6000052812D10A4EA0688168FF208847FF2844
:10DE700002D0761EF7D108E03EB108F500786D1E9D
:10DE8000002DD5D10120BDE8F0810020FBE7000086
:10DE900020A1070070B500248020104908800320CD
:10DEA00088700420C8700E48F8F7ECF9002510E0DF
:10DEB0006006040EFBF7B6FFFEF742F98021084822
:10DEC000F8F755FA08B144F00104FBF7B5FF681CF8
:10DED000C5B2082DECDB204670BD00002C010020EF
:10DEE000000C014010B5FBF7C7FFFBF79BFFFBF7EA
:10DEF000A3FFFBF7ABFF10BD70B50446C0680D462D
:10DF0000164610B194F8641029B129462046BDE8A0
:10DF1000704000F049B894F8652082B1A16DA94223
:10DF20000DD80A44AA420AD9206E691A00EB412191
:10DF30004FF40072E06DF2F77EFB656517E0B042CA
:10DF400000D206466068E16D3246836828469847ED
:10DF5000012806D04FF0FF306065002084F865008E
:10DF600070BD65656D1C761EA56584F86560012031
:10DF700070BD70B50E460446C58A016A0069FEF799
:10DF8000F8FF00EB1511206900F00EF800280AD008
:10DF9000206905F00F012022C06D00EB41113046D1
:10DFA000F2F78EFB012070BD70B50446406D0D4642
:10DFB000A84201D1012070BDA06DA8420ED894F8EE
:10DFC00064100144A94209D9216E281A01EB4021AD
:10DFD0004FF40072E06DF2F72EFB0CE06068E16D2B
:10DFE0000122836828469847012804D04FF0FF306B
:10DFF0006065002070BD6565DCE72DE9F0410746EE
:10E00000086988B00C4690F87A609046002538463A
:10E01000FDF737FD60B1012E09D03846F2F7E0FA7E
:10E020000C300D21B0FBF1F0401CB04200D90125AD
:10E0300069462046FFF79DFF002817D02046FEF7CF
:10E040008FF8002812D045B120692146406FE06169
:10E050003846FDF71FFC002808D06B464246214693
:10E060003846FDF755FE002800D0012008B0BDE875
:10E07000F08100002DE9FF4F97B00C46012A19D01E
:10E080000020129001204FF0000ACDE90E0A039003
:10E09000E06900901798F2F7A3FA0490002010901E
:10E0A00021698346E06908671798FDF7EAFC0128B3
:10E0B00002D009E00120E4E704980D210C30B0FB08
:10E0C000F1F0401CC0B20E9009A91798FDF7E9FFC6
:10E0D000129808B1092000E00D20079020690099EE
:10E0E000FEF747FF81460026206990F87B1019B1A2
:10E0F000B6F5007F13D01BE0818FB14218D1016CBF
:10E10000009A0026914200D90091694600F0C2F8B9
:10E11000002805D020690099FFF740FA18B10020C7
:10E120001BB0BDE8F08F20690099FDF75FFD8146C7
:10E1300009EB16112069FFF737FF0028F0D020699E
:10E1400006F00F01C06D00EB411528780028E7D0DC
:10E15000E5286FD095F80B80B8F10F0F03D05FEA78
:10E16000087067D431E0410609D500991091697BA8
:10E170000F9120F04001491CC9B2B34603916A7B5C
:10E180000F998A4256D100F01F00401E00EB80011B
:10E1900001EBC0001799DFF8F8C00A18002000BF93
:10E1A0001CF80010135C695C81EA030737F0200754
:10E1B00008D103B911B1401C0D28F1D30AF10100B7
:10E1C00000F0FF0AB8F10F0F34D0039801280ED0E9
:10E1D00029D9A0F1010050451BD12846FFF7FAF9D3
:10E1E0000F99884215D10AF10100C0B21AE00E98C9
:10E1F000012803D007990498884214D200981090FF
:10E20000B34609A9284600F097F878B14FF0010A03
:10E2100012E00E98012806D109A9284600F08CF8D2
:10E2200008B1039882460398504505D001204FF06D
:10E23000000A0390761C57E7E87AC0F300111298A1
:10E240008142F3D11A9808BBE87A207505F11A00CB
:10E25000FFF72CF9074605F11400FFF727F907EB44
:10E260000040E061E68200982062216910984867CA
:10E2700021690020A1F878B0216981F87AA0E060D6
:10E2800005F11C00FFF717F96060A060012047E767
:10E29000964E03082DE9F0410D680E4604462946C6
:10E2A000FEF77DFE804601462046FDF7A1FB0028D3
:10E2B00007D0207F012806D0022825D0032828D0A7
:10E2C0000020BDE8F08105EB4500C0F34800B0F543
:10E2D000FF7F04D8E16C0844FFF7E8F80DE0E06C3C
:10E2E00008F1010190F8FF712046FDF781FB00283D
:10E2F000E7D0E06C007847EA0020E90701D0000988
:10E300000BE0C0F30B0008E0E16C2806C00D085AD2
:10E3100003E06806E16CC00D085830600120D0E7CA
:10E320000A0A4270017070470A0EC2700A0C8270AD
:10E330000A0A42700170704730B50022835C8C5C21
:10E3400083EA040535F0200501D0002030BD04B972
:10E3500013B1521C0B2AF1D3012030BD10B5FBF7CD
:10E3600075FDFBF75FFDFDF7EBFEFBF785FDFDF7A8
:10E37000E7FEFBF761FDFDF7E3FE10BD10B5FBF70F
:10E380007BFDFDF7DDFEFBF74DFDFDF7D9FEFBF74D
:10E390005DFDFDF7D5FE10BD2DE9F04700260127F4
:10E3A00004460D4602297DD379E0E06EA84200D9EB
:10E3B000E56629462046FEF7F2FD814601462046E5
:10E3C000FDF716FB00287AD0207F012804D0022810
:10E3D00046D0032872D14DE005EB4500C0F3480854
:10E3E000B8F5FF7F16D8E16C01EB0800FFF75EF887
:10E3F000E90703D000F00F01000903E000F47041C9
:10E40000C0F30B00E26C814602EB080089B2FFF713
:10E4100087FF3BE0E06CEA0790F8FF11884604D0E4
:10E4200001F00F0180F8FF1101E080F8FF6184F82E
:10E43000507009F101012046FDF7DAFA00283ED0BC
:10E44000E06CEB07017848EA012202D0067010095F
:10E4500004E001F0F0010170C2F30B00814615E009
:10E460002806C50DE06C2844FFF720F88146E06CD3
:10E4700046530BE06806C50DE06C2844FFF71BF817
:10E480008146E06C4651A06E401CA06684F8507036
:10E4900049462046FFF782F8012812D04D46206BEE
:10E4A000801C02E013E00AE008E0A8423FF67DAFDE
:10E4B00000212046FDF79CFA002800D00020BDE88E
:10E4C000F08700212046FDF793FA0028F7D00120BD
:10E4D000F5E710B5044600F005F808B1204610BD78
:10E4E000582010BDA0F12001012917D9C91E062905
:10E4F00014D92D2812D02E2810D00D3909290DD964
:10E5000040280BD01139192908D91D391D2905D9E1
:10E510007D2803D07E2801D000207047012070475D
:10E5200010B501210248F7F732FFFDF709FE10BDD3
:10E530000018014010B501210248F7F726FFFDF74A
:10E54000FFFD10BD0018014070B5044625460026A9
:10E550000FE005F0800010B1FBF778FC01E0FBF75D
:10E560008BFC6806050EFBF75DFCFBF765FC701C79
:10E57000C6B2082EEDDB70BD70B50125FBF766FC59
:10E58000FBF750FC80210A48F7F7F1FE00B10025A7
:10E59000FBF752FC07480068012806D1002402E07E
:10E5A000FDF7CEFD641C0A2CFADB284670BD000086
:10E5B000000C0140280100202DE9F04107460C46DF
:10E5C0000A201649086000BFFFF7C8FEA02101EB32
:10E5D0004701C8B200F072F805460DB9FFF7CEFE4C
:10E5E0001DB90E4800680028EED145B12646E11756
:10E5F00004EB1161C1F3072000F060F8054655B146
:10E600002646E11704EB11610912A4EB0121C8B2FF
:10E6100000F054F805462846BDE8F08120010020AE
:10E620002DE9F0410D46C1680446E1B100261DB355
:10E63000656594F864204FF400779AB3A06D831851
:10E64000AB4227D18A4225D204F15C04606821687C
:10E6500000EB42203A46F1F7EEFF207A401C207290
:10E660000120BDE8F081002DFAD00022294600F0FB
:10E670005BF90028F5D0F3E794F86420002AEFD086
:10E680006368216EA06DDB6898470028E9D084F8A4
:10E690006460E5E76368216EDB6898470028E0D096
:10E6A00084F8646004F158043A46D4E90110F1F7A3
:10E6B000C2FF0120256020736673D1E710B50446C0
:10E6C0002046FFF741FFFFF757FF08B1012010BDBB
:10E6D0000020FCE72DE9F0410446C769FEF7CEFEB5
:10E6E0000646FEF730FC804620694FF40071C06D8D
:10E6F000F2F718F820690B2234A1C56D2846F1F70E
:10E70000DFFF1020E872314605F10E00FFF708FE2A
:10E71000414605F11000FFF703FE414605F11200E6
:10E72000FFF7FEFD314605F11600FFF7F9FD414602
:10E7300005F11800FFF7F4FD05F12000202229461D
:10E740000646F1F7BDFFE069010C05F11400FFF783
:10E75000E7FDE06981B205F11A00FFF7E1FD2E2027
:10E7600070702069006F010C06F11400FFF7D8FDEE
:10E770002069006F81B206F11A00FFF7D1FD21690F
:10E78000E069086739462069FDF730FA064601223C
:10E790003146206900F0C8F8002814D020694021D3
:10E7A000C06DF1F7BFFF012506E07119002200F0EE
:10E7B000BBF8002807D06D1C2069817FA942F4D8DE
:10E7C0000220E0820120BDE8F08100002E20202000
:10E7D00020202020202020002DE9F0471546044667
:10E7E0000E46FEF7DCFB814601462046FDF700F9A8
:10E7F000002809D0207F4FF00108012806D0022808
:10E8000044D0032848D00020BDE8F08706EB46003E
:10E81000C0F34807C5F30B05B7F5FF7F13D8E06CCD
:10E820003844FEF743FEF10702D065F31F1002E003
:10E8300000F470402843E16CCA1981B24FEA02002B
:10E84000FFF76EFD38E0F007E06C06D090F8FF119E
:10E8500065F31F1180F8FF1101E080F8FF5184F883
:10E86000508009F101012046FDF7C2F80028CBD005
:10E87000F00703D0E16C280908701DE0E06C017816
:10E8800001F0F00141EA1521017015E0E16C30065C
:10E8900001EBD050A9B2D3E77006C60DE06C30444E
:10E8A000FEF709FE18B9A06E08B1401EA066E06C24
:10E8B00029463044FFF738FD84F850800120A3E753
:10E8C00010B50446C06D4FF40071F1F72BFF1449E9
:10E8D000E06DFFF729FDE06D124900F5F270FFF7DA
:10E8E00023FDE06DA16E00F5F470FFF71DFDE06DF6
:10E8F000E16E00F5F670FFF717FDE06D4AF6552161
:10E9000000F5FF70FFF70CFDB4F84410A069014456
:10E910002046FFF785FE002800D0012010BD000032
:10E92000525261417272416170B504460D464069B0
:10E93000E16D08B1012A09D060680122C368284648
:10E940009847002801D00120656570BD0B46002264
:10E950002946FEF78CFAF4E70000000030000020A2
:10E9600000000000000000009F0500000000000003
:10E9700040480000010000001C000020670000006B
:10E9800000000000030000000000000002E00000A2
:10E99000020000001C00002068000000650000006C
:10E9A000280C00006500000002A000000300000029
:10E9B0001C00002069000000D0070000B80B000018
:10E9C000DE07000002200000040000001C00002000
:10E9D0006A00000001000000E803000001000000E0
:10E9E00002200000050000001C000020650000005F
:10E9F0000100000040420F00010000000220000062
:10EA0000640000001C0000206B0000000A000000F1
:10EA1000640000002800000012880000650000006B
:10EA2000340000200000000000000000D0070000BB
:10EA3000BC02000011500000660000001C00002015
:10EA40007A010000010000000A0000000A00000036
:10EA500002200000670000003800002000000000D5
:10EA6000000000000A00000000000000012000007B
:10EA7000680000001C0000207B0100000000000076
:10EA800001000000000000000260000069000000BA
:10EA90001C0000207C0100000000000001000000BC
:10EAA00000000000026000006A0000001C0000205E
:10EAB0007D0100000000000078000000050000005B
:10EAC000C24800006B0000001C0000207E01000016
:10EAD00000000000D0070000D00700001350000025
:10EAE0006C0000001C0000207F01000000000000FE
:10EAF0009F05000000000000434800006D0000007A
:10EB00001C0000208001000000000000D007000071
:10EB100000000000135000006E0000001C000020E8
:10EB200081010000000000009F05000000000000BF
:10EB3000434800006F0000001C000020820100001C
:10EB40000000000001000000000000000260000062
:10EB5000700000001C000020830100000100000084
:10EB6000060000000100000002200000710000000B
:10EB70001C00002084010000000000009F05000030
:10EB80000000000042480000720000001C0000204D
:10EB900085010000000000000100000001000000ED
:10EBA00002600000730000001C00002086010000CD
:10EBB00000000000010000000000000002600000F2
:10EBC000C80000005C000020000000000000000001
:10EBD000D00700000000000011500000C900000034
:10EBE000600000200000000000000000D0070000CE
:10EBF0000000000011500000CA0000006400002066
:10EC00000000000000000000010000000000000003
:10EC100001600000CB000000680000200000000040
:10EC20000000000001000000000000000160000082
:10EC3000CC0000006C00002000000000000000007C
:10EC4000010000000000000001600000CD00000095
:10EC50007000002000000000000000000100000023
:10EC60000000000001600000CE00000074000020E1
:10EC700000000000000000000A000000000000008A
:10EC800000200000CF0000007800002000000000FD
:10EC90000000000001000000000000000060000013
:10ECA000D00000007C0000200000000000000000F8
:10ECB000D00700000000000021290000D100000062
:10ECC00080000020000000000000000001000000A3
:10ECD0000000000000600000D2000000840000205E
:10ECE0000000000000000000010000000000000023
:10ECF00000600000E80300001C0000206C00000021
:10ED000000000000050000000000000002000000FC
:10ED1000E90300001C0000206D000000BC020000A0
:10ED2000B00400008403000012500000EA03000059
:10ED30001C0000208600000001000000100E0000F2
:10ED40000A000000C2480000EB0300001C00002085
:10ED50006E000000000000009F05000000000000A1
:10ED600042480000EC0300001C0000206F0000007F
:10ED7000000000009F050000000000004248000065
:10ED8000ED0300001C0000207000000001000000E6
:10ED9000D00200003C00000042480000EE030000EA
:10EDA0001C0000207100000001000000D0020000E3
:10EDB0001E00000042480000EF0300001C0000207D
:10EDC00072000000000000009F050000000000002D
:10EDD00042480000F00300001C0000207300000007
:10EDE000000000009F0500000000000042480000F5
:10EDF000F10300001C00002074000000010000006E
:10EE0000D00200003C00000042480000F203000075
:10EE10001C0000207500000001000000D00200006E
:10EE20001E00000042480000F30300001C00002008
:10EE300076000000000000009F05000000000000B8
:10EE400042480000F40300001C000020770000008E
:10EE5000000000009F050000000000004248000084
:10EE6000F50300001C0000207800000001000000F5
:10EE7000D00200003C00000042480000F603000001
:10EE80001C0000207900000001000000D0020000FA
:10EE90001E00000042480000F70300001C00002094
:10EEA0007A000000000000009F0500000000000044
:10EEB00042480000F80300001C0000207B00000016
:10EEC000000000009F050000000000004248000014
:10EED000F90300001C0000207C000000010000007D
:10EEE000D00200003C00000042480000FA0300008D
:10EEF0001C0000207D00000001000000D002000086
:10EF00001E00000042480000FB0300001C0000201F
:10EF10007E000000000000009F05000000000000CF
:10EF200042480000FC0300001C0000207F0000009D
:10EF3000000000009F0500000000000042480000A3
:10EF4000FD0300001C000020800000000100000004
:10EF5000D00200003C00000042480000FE03000018
:10EF60001C0000208100000001000000D002000011
:10EF70001E00000042480000FF0300001C000020AB
:10EF800082000000000000009F050000000000005B
:10EF900042480000000400001C0000208300000024
:10EFA000000000009F050000000000004248000033
:10EFB000010400001C00002084000000010000008B
:10EFC000D00200003C0000004248000002040000A3
:10EFD0001C0000208500000001000000D00200009D
:10EFE0001E00000042480000030400001C00002036
:10EFF0008701000020202020FFFFFF7F31302D56A9
:10F0000002480100D00700001C000020870000001B
:10F0100000000000050000000000000002000000E9
:10F02000D10700001C00002088000000BC02000086
:10F03000B00400008403000012500000D20700005A
:10F040001C000020A100000001000000100E0000C4
:10F050000A000000C2480000D30700001C00002086
:10F0600089000000000000009F0500000000000073
:10F0700042480000D40700001C0000208A00000065
:10F08000000000009F050000000000004248000052
:10F09000D50700001C0000208B00000001000000CC
:10F0A000D00200003C00000042480000D6070000EB
:10F0B0001C0000208C00000001000000D0020000B5
:10F0C0001E00000042480000D70700001C0000207E
:10F0D0008D000000000000009F05000000000000FF
:10F0E00042480000D80700001C0000208E000000ED
:10F0F000000000009F0500000000000042480000E2
:10F10000D90700001C0000208F0000000100000053
:10F11000D00200003C00000042480000DA07000076
:10F120001C0000209000000001000000D002000040
:10F130001E00000042480000DB0700001C00002009
:10F1400091000000000000009F050000000000008A
:10F1500042480000DC0700001C0000209200000074
:10F16000000000009F050000000000004248000071
:10F17000DD0700001C0000209300000001000000DB
:10F18000D00200003C00000042480000DE07000002
:10F190001C0000209400000001000000D0020000CC
:10F1A0001E00000042480000DF0700001C00002095
:10F1B00095000000000000009F0500000000000016
:10F1C00042480000E00700001C00002096000000FC
:10F1D000000000009F050000000000004248000001
:10F1E000E10700001C000020970000000100000063
:10F1F000D00200003C00000042480000E20700008E
:10F200001C0000209800000001000000D002000057
:10F210001E00000042480000E30700001C00002020
:10F2200099000000000000009F05000000000000A1
:10F2300042480000E40700001C0000209A00000083
:10F24000000000009F050000000000004248000090
:10F25000E50700001C0000209B00000001000000EA
:10F26000D00200003C00000042480000E607000019
:10F270001C0000209C00000001000000D0020000E3
:10F280001E00000042480000E70700001C000020AC
:10F290009D000000000000009F050000000000002D
:10F2A00042480000E80700001C0000209E0000000B
:10F2B000000000009F050000000000004248000020
:10F2C000E90700001C0000209F0000000100000072
:10F2D000D00200003C00000042480000EA070000A5
:10F2E0001C000020A000000001000000D00200006F
:10F2F0001E00000042480000EB0700001C00002038
:10F300008801000020202020FFFFFF7F32302D5693
:10F3100002480100B80B00001C000020A200000001
:10F3200000000000050000000000000002000000D6
:10F33000B90B00001C000020A3000000BC0200006C
:10F34000B00400008403000012500000BA0B00005B
:10F350001C000020BC00000001000000100E000096
:10F360000A000000C2480000BB0B00001C00002087
:10F37000A4000000000000009F0500000000000045
:10F3800042480000BC0B00001C000020A50000004B
:10F39000000000009F05000000000000424800003F
:10F3A000BD0B00001C000020A600000001000000B2
:10F3B000D00200003C00000042480000BE0B0000EC
:10F3C0001C000020A700000001000000D002000087
:10F3D0001E00000042480000BF0B00001C0000207F
:10F3E000A8000000000000009F05000000000000D1
:10F3F00042480000C00B00001C000020A9000000D3
:10F40000000000009F0500000000000042480000CE
:10F41000C10B00001C000020AA0000000100000039
:10F42000D00200003C00000042480000C20B000077
:10F430001C000020AB00000001000000D002000012
:10F440001E00000042480000C30B00001C0000200A
:10F45000AC000000000000009F050000000000005C
:10F4600042480000C40B00001C000020AD0000005A
:10F47000000000009F05000000000000424800005E
:10F48000C50B00001C000020AE00000001000000C1
:10F49000D00200003C00000042480000C60B000003
:10F4A0001C000020AF00000001000000D00200009E
:10F4B0001E00000042480000C70B00001C00002096
:10F4C000B0000000000000009F05000000000000E8
:10F4D00042480000C80B00001C000020B1000000E2
:10F4E000000000009F0500000000000042480000EE
:10F4F000C90B00001C000020B20000000100000049
:10F50000D00200003C00000042480000CA0B00008E
:10F510001C000020B300000001000000D002000029
:10F520001E00000042480000CB0B00001C00002021
:10F53000B4000000000000009F0500000000000073
:10F5400042480000CC0B00001C000020B500000069
:10F55000000000009F05000000000000424800007D
:10F56000CD0B00001C000020B600000001000000D0
:10F57000D00200003C00000042480000CE0B00001A
:10F580001C000020B700000001000000D0020000B5
:10F590001E00000042480000CF0B00001C000020AD
:10F5A000B8000000000000009F05000000000000FF
:10F5B00042480000D00B00001C000020B9000000F1
:10F5C000000000009F05000000000000424800000D
:10F5D000D10B00001C000020BA0000000100000058
:10F5E000D00200003C00000042480000D20B0000A6
:10F5F0001C000020BB00000001000000D002000041
:10F600001E00000042480000D30B00001C00002038
:10F610008901000020202020FFFFFF7F33302D567E
:10F6200002480100A00F00001C000020BD000000E7
:10F6300000000000050000000000000002000000C3
:10F64000A10F00001C000020BE000000BC02000052
:10F65000B00400008403000012500000A20F00005C
:10F660001C000020D700000001000000100E000068
:10F670000A000000C2480000A30F00001C00002088
:10F68000BF000000000000009F0500000000000017
:10F6900042480000A40F00001C000020C000000031
:10F6A000000000009F05000000000000424800002C
:10F6B000A50F00001C000020C10000000100000098
:10F6C000D00200003C00000042480000A60F0000ED
:10F6D0001C000020C200000001000000D002000059
:10F6E0001E00000042480000A70F00001C00002080
:10F6F000C3000000000000009F05000000000000A3
:10F7000042480000A80F00001C000020C4000000B8
:10F71000000000009F0500000000000042480000BB
:10F72000A90F00001C000020C5000000010000001F
:10F73000D00200003C00000042480000AA0F000078
:10F740001C000020C600000001000000D0020000E4
:10F750001E00000042480000AB0F00001C0000200B
:10F76000C7000000000000009F050000000000002E
:10F7700042480000AC0F00001C000020C800000040
:10F78000000000009F05000000000000424800004B
:10F79000AD0F00001C000020C900000001000000A7
:10F7A000D00200003C00000042480000AE0F000004
:10F7B0001C000020CA00000001000000D002000070
:10F7C0001E00000042480000AF0F00001C00002097
:10F7D000CB000000000000009F05000000000000BA
:10F7E00042480000B00F00001C000020CC000000C8
:10F7F000000000009F0500000000000042480000DB
:10F80000B10F00001C000020CD000000010000002E
:10F81000D00200003C00000042480000B20F00008F
:10F820001C000020CE00000001000000D0020000FB
:10F830001E00000042480000B30F00001C00002022
:10F84000CF000000000000009F0500000000000045
:10F8500042480000B40F00001C000020D00000004F
:10F86000000000009F05000000000000424800006A
:10F87000B50F00001C000020D100000001000000B6
:10F88000D00200003C00000042480000B60F00001B
:10F890001C000020D200000001000000D002000087
:10F8A0001E00000042480000B70F00001C000020AE
:10F8B000D3000000000000009F05000000000000D1
:10F8C00042480000B80F00001C000020D4000000D7
:10F8D000000000009F0500000000000042480000FA
:10F8E000B90F00001C000020D5000000010000003E
:10F8F000D00200003C00000042480000BA0F0000A7
:10F900001C000020D600000001000000D002000012
:10F910001E00000042480000BB0F00001C00002039
:10F920008A01000020202020FFFFFF7F34302D5669
:10F9300002480100881300001C000020D8000000CD
:10F9400000000000050000000000000002000000B0
:10F95000891300001C000020D9000000BC02000038
:10F96000B004000084030000125000008A1300005D
:10F970001C000020F200000001000000100E00003A
:10F980000A000000C24800008B1300001C00002089
:10F99000DA000000000000009F05000000000000E9
:10F9A000424800008C1300001C000020DB00000017
:10F9B000000000009F050000000000004248000019
:10F9C0008D1300001C000020DC000000010000007E
:10F9D000D00200003C000000424800008E130000EE
:10F9E0001C000020DD00000001000000D00200002B
:10F9F0001E000000424800008F1300001C00002081
:10FA0000DE000000000000009F0500000000000074
:10FA100042480000901300001C000020DF0000009E
:10FA2000000000009F0500000000000042480000A8
:10FA3000911300001C000020E00000000100000005
:10FA4000D00200003C000000424800009213000079
:10FA50001C000020E100000001000000D0020000B6
:10FA60001E00000042480000931300001C0000200C
:10FA7000E2000000000000009F0500000000000000
:10FA800042480000941300001C000020E300000026
:10FA9000000000009F050000000000004248000038
:10FAA000951300001C000020E4000000010000008D
:10FAB000D00200003C000000424800009613000005
:10FAC0001C000020E500000001000000D002000042
:10FAD0001E00000042480000971300001C00002098
:10FAE000E6000000000000009F050000000000008C
:10FAF00042480000981300001C000020E7000000AE
:10FB0000000000009F0500000000000042480000C7
:10FB1000991300001C000020E80000000100000014
:10FB2000D00200003C000000424800009A13000090
:10FB30001C000020E900000001000000D0020000CD
:10FB40001E000000424800009B1300001C00002023
:10FB5000EA000000000000009F0500000000000017
:10FB6000424800009C1300001C000020EB00000035
:10FB7000000000009F050000000000004248000057
:10FB80009D1300001C000020EC000000010000009C
:10FB9000D00200003C000000424800009E1300001C
:10FBA0001C000020ED00000001000000D002000059
:10FBB0001E000000424800009F1300001C000020AF
:10FBC000EE000000000000009F05000000000000A3
:10FBD00042480000A01300001C000020EF000000BD
:10FBE000000000009F0500000000000042480000E7
:10FBF000A11300001C000020F00000000100000024
:10FC0000D00200003C00000042480000A2130000A7
:10FC10001C000020F100000001000000D0020000E4
:10FC20001E00000042480000A31300001C0000203A
:10FC30008B01000020202020FFFFFF7F35302D5654
:10FC400002480100701700001C000020F3000000B3
:10FC5000000000000500000000000000020000009D
:10FC6000711700001C000020F4000000BC0200001E
:10FC7000B00400008403000012500000721700005E
:10FC80001C0000200D01000001000000100E00000B
:10FC90000A000000C2480000731700001C0000208A
:10FCA000F5000000000000009F05000000000000BB
:10FCB00042480000741700001C000020F6000000FD
:10FCC000000000009F050000000000004248000006
:10FCD000751700001C000020F70000000100000064
:10FCE000D00200003C0000004248000076170000EF
:10FCF0001C000020F800000001000000D0020000FD
:10FD00001E00000042480000771700001C00002081
:10FD1000F9000000000000009F0500000000000046
:10FD200042480000781700001C000020FA00000084
:10FD3000000000009F050000000000004248000095
:10FD4000791700001C000020FB00000001000000EB
:10FD5000D00200003C000000424800007A1700007A
:10FD60001C000020FC00000001000000D002000088
:10FD70001E000000424800007B1700001C0000200D
:10FD8000FD000000000000009F05000000000000D2
:10FD9000424800007C1700001C000020FE0000000C
:10FDA000000000009F050000000000004248000025
:10FDB0007D1700001C000020FF0000000100000073
:10FDC000D00200003C000000424800007E17000006
:10FDD0001C0000200001000001000000D002000013
:10FDE0001E000000424800007F1700001C00002099
:10FDF00001010000000000009F050000000000005D
:10FE000042480000801700001C0000200201000092
:10FE1000000000009F0500000000000042480000B4
:10FE2000811700001C0000200301000001000000F9
:10FE3000D00200003C000000424800008217000091
:10FE40001C0000200401000001000000D00200009E
:10FE50001E00000042480000831700001C00002024
:10FE600005010000000000009F05000000000000E8
:10FE700042480000841700001C000020060100001A
:10FE8000000000009F050000000000004248000044
:10FE9000851700001C000020070100000100000081
:10FEA000D00200003C00000042480000861700001D
:10FEB0001C0000200801000001000000D00200002A
:10FEC0001E00000042480000871700001C000020B0
:10FED00009010000000000009F0500000000000074
:10FEE00042480000881700001C0000200A010000A2
:10FEF000000000009F0500000000000042480000D4
:10FF0000891700001C0000200B0100000100000008
:10FF1000D00200003C000000424800008A170000A8
:10FF20001C0000200C01000001000000D0020000B5
:10FF30001E000000424800008B1700001C0000203B
:10FF40008C01000020202020FFFFFF7F36302D563F
:10FF500002480100581B00001C0000200E01000098
:10FF6000000000000500000000000000020000008A
:10FF7000591B00001C0000200F010000BC02000003
:10FF8000B004000084030000125000005A1B00005F
:10FF90001C0000202801000001000000100E0000DD
:10FFA0000A000000C24800005B1B00001C0000208B
:10FFB00010010000000000009F050000000000008C
:10FFC000424800005C1B00001C00002011010000E2
:10FFD000000000009F0500000000000042480000F3
:10FFE0005D1B00001C000020120100000100000049
:10FFF000D00200003C000000424800005E1B0000F0
:020000040802F0
:100000001C0000201301000001000000D0020000CD
:100010001E000000424800005F1B00001C00002082
:1000200014010000000000009F0500000000000017
:1000300042480000601B00001C0000201501000069
:10004000000000009F050000000000004248000082
:10005000611B00001C0000201601000001000000D0
:10006000D00200003C00000042480000621B00007B
:100070001C0000201701000001000000D002000059
:100080001E00000042480000631B00001C0000200E
:1000900018010000000000009F05000000000000A3
:1000A00042480000641B00001C00002019010000F1
:1000B000000000009F050000000000004248000012
:1000C000651B00001C0000201A0100000100000058
:1000D000D00200003C00000042480000661B000007
:1000E0001C0000201B01000001000000D0020000E5
:1000F0001E00000042480000671B00001C0000209A
:100100001C010000000000009F050000000000002E
:1001100042480000681B00001C0000201D01000078
:10012000000000009F0500000000000042480000A1
:10013000691B00001C0000201E01000001000000DF
:10014000D00200003C000000424800006A1B000092
:100150001C0000201F01000001000000D002000070
:100160001E000000424800006B1B00001C00002025
:1001700020010000000000009F05000000000000BA
:10018000424800006C1B00001C0000202101000000
:10019000000000009F050000000000004248000031
:1001A0006D1B00001C000020220100000100000067
:1001B000D00200003C000000424800006E1B00001E
:1001C0001C0000202301000001000000D0020000FC
:1001D0001E000000424800006F1B00001C000020B1
:1001E00024010000000000009F0500000000000046
:1001F00042480000701B00001C0000202501000088
:10020000000000009F0500000000000042480000C0
:10021000711B00001C0000202601000001000000EE
:10022000D00200003C00000042480000721B0000A9
:100230001C0000202701000001000000D002000087
:100240001E00000042480000731B00001C0000203C
:100250008D01000020202020FFFFFF7F37302D562A
:1002600002480100401F00001C000020290100007E
:100270000000000005000000000000000200000077
:10028000411F00001C0000202A010000BC020000E9
:10029000B00400008403000012500000421F000060
:1002A0001C0000204301000001000000100E0000AF
:1002B0000A000000C2480000431F00001C0000208C
:1002C0002B010000000000009F050000000000005E
:1002D00042480000441F00001C0000202C010000C8
:1002E000000000009F0500000000000042480000E0
:1002F000451F00001C0000202D010000010000002F
:10030000D00200003C00000042480000461F0000F0
:100310001C0000202E01000001000000D00200009F
:100320001E00000042480000471F00001C00002083
:100330002F010000000000009F05000000000000E9
:1003400042480000481F00001C000020300100004F
:10035000000000009F05000000000000424800006F
:10036000491F00001C0000203101000001000000B6
:10037000D00200003C000000424800004A1F00007C
:100380001C0000203201000001000000D00200002B
:100390001E000000424800004B1F00001C0000200F
:1003A00033010000000000009F0500000000000075
:1003B000424800004C1F00001C00002034010000D7
:1003C000000000009F0500000000000042480000FF
:1003D0004D1F00001C00002035010000010000003E
:1003E000D00200003C000000424800004E1F000008
:1003F0001C0000203601000001000000D0020000B7
:100400001E000000424800004F1F00001C0000209A
:1004100037010000000000009F0500000000000000
:1004200042480000501F00001C000020380100005E
:10043000000000009F05000000000000424800008E
:10044000511F00001C0000203901000001000000C5
:10045000D00200003C00000042480000521F000093
:100460001C0000203A01000001000000D002000042
:100470001E00000042480000531F00001C00002026
:100480003B010000000000009F050000000000008C
:1004900042480000541F00001C0000203C010000E6
:1004A000000000009F05000000000000424800001E
:1004B000551F00001C0000203D010000010000004D
:1004C000D00200003C00000042480000561F00001F
:1004D0001C0000203E01000001000000D0020000CE
:1004E0001E00000042480000571F00001C000020B2
:1004F0003F010000000000009F0500000000000018
:1005000042480000581F00001C000020400100006D
:10051000000000009F0500000000000042480000AD
:10052000591F00001C0000204101000001000000D4
:10053000D00200003C000000424800005A1F0000AA
:100540001C0000204201000001000000D002000059
:100550001E000000424800005B1F00001C0000203D
:100560008E01000020202020FFFFFF7F38302D5615
:1005700002480100282300001C0000204401000064
:100580000000000005000000000000000200000064
:10059000292300001C00002045010000BC020000CF
:1005A000B004000084030000125000002A23000061
:1005B0001C0000205E01000001000000100E000081
:1005C0000A000000C24800002B2300001C0000208D
:1005D00046010000000000009F0500000000000030
:1005E000424800002C2300001C00002047010000AE
:1005F000000000009F0500000000000042480000CD
:100600002D2300001C000020480100000100000014
:10061000D00200003C000000424800002E230000F1
:100620001C0000204901000001000000D002000071
:100630001E000000424800002F2300001C00002084
:100640004A010000000000009F05000000000000BB
:1006500042480000302300001C0000204B01000035
:10066000000000009F05000000000000424800005C
:10067000312300001C0000204C010000010000009C
:10068000D00200003C00000042480000322300007D
:100690001C0000204D01000001000000D0020000FD
:1006A0001E00000042480000332300001C00002010
:1006B0004E010000000000009F0500000000000047
:1006C00042480000342300001C0000204F010000BD
:1006D000000000009F0500000000000042480000EC
:1006E000352300001C000020500100000100000024
:1006F000D00200003C000000424800003623000009
:100700001C0000205101000001000000D002000088
:100710001E00000042480000372300001C0000209B
:1007200052010000000000009F05000000000000D2
:1007300042480000382300001C0000205301000044
:10074000000000009F05000000000000424800007B
:10075000392300001C0000205401000001000000AB
:10076000D00200003C000000424800003A23000094
:100770001C0000205501000001000000D002000014
:100780001E000000424800003B2300001C00002027
:1007900056010000000000009F050000000000005E
:1007A000424800003C2300001C00002057010000CC
:1007B000000000009F05000000000000424800000B
:1007C0003D2300001C000020580100000100000033
:1007D000D00200003C000000424800003E23000020
:1007E0001C0000205901000001000000D0020000A0
:1007F0001E000000424800003F2300001C000020B3
:100800005A010000000000009F05000000000000E9
:1008100042480000402300001C0000205B01000053
:10082000000000009F05000000000000424800009A
:10083000412300001C0000205C01000001000000BA
:10084000D00200003C0000004248000042230000AB
:100850001C0000205D01000001000000D00200002B
:100860001E00000042480000432300001C0000203E
:100870008F01000020202020FFFFFF7F39302D5600
:1008800002480100102700001C0000205F0100004A
:100890000000000005000000000000000200000051
:1008A000112700001C00002060010000BC020000B5
:1008B000B004000084030000125000001227000062
:1008C0001C0000207901000001000000100E000053
:1008D0000A000000C2480000132700001C0000208E
:1008E00061010000000000009F0500000000000002
:1008F00042480000142700001C0000206201000094
:10090000000000009F0500000000000042480000B9
:10091000152700001C0000206301000001000000FA
:10092000D00200003C0000004248000016270000F2
:100930001C0000206401000001000000D002000043
:100940001E00000042480000172700001C00002085
:1009500065010000000000009F050000000000008D
:1009600042480000182700001C000020660100001B
:10097000000000009F050000000000004248000049
:10098000192700001C000020670100000100000082
:10099000D00200003C000000424800001A2700007E
:1009A0001C0000206801000001000000D0020000CF
:1009B0001E000000424800001B2700001C00002011
:1009C00069010000000000009F0500000000000019
:1009D000424800001C2700001C0000206A010000A3
:1009E000000000009F0500000000000042480000D9
:1009F0001D2700001C0000206B010000010000000A
:100A0000D00200003C000000424800001E27000009
:100A10001C0000206C01000001000000D00200005A
:100A20001E000000424800001F2700001C0000209C
:100A30006D010000000000009F05000000000000A4
:100A400042480000202700001C0000206E0100002A
:100A5000000000009F050000000000004248000068
:100A6000212700001C0000206F0100000100000091
:100A7000D00200003C000000424800002227000095
:100A80001C0000207001000001000000D0020000E6
:100A90001E00000042480000232700001C00002028
:100AA00071010000000000009F0500000000000030
:100AB00042480000242700001C00002072010000B2
:100AC000000000009F0500000000000042480000F8
:100AD000252700001C000020730100000100000019
:100AE000D00200003C000000424800002627000021
:100AF0001C0000207401000001000000D002000072
:100B00001E00000042480000272700001C000020B3
:100B100075010000000000009F05000000000000BB
:100B200042480000282700001C0000207601000039
:100B3000000000009F050000000000004248000087
:100B4000292700001C0000207701000001000000A0
:100B5000D00200003C000000424800002A270000AC
:100B60001C0000207801000001000000D0020000FD
:100B70001E000000424800002B2700001C0000203F
:100B80009001000020202020FFFFFF7F30312D56F4
:100B900002480100FFFF000000000000000000000C
:100BA0000000000000000000000000000000000045
:100BB0000000000054220E00010000000A000000A6
:100BC0002A070D000200000014000000E7030C00DB
:100BD000030000001E00000064160B00040000006B
:100BE00028000000AF3C0A000500000032000000B1
:100BF00004750900070000003C000000CBBD0800A0
:100C00000800000046000000911508000A000000DE
:100C100050000000077B07000B0000005A00000096
:100C2000FCEC06000D000000640000005A6A06009B
:100C30000F0000006E00000028F205001100000007
:100C4000780000007F830500130000008200000090
:100C5000921D0500160000008C000000A2BF0400D9
:100C60001800000096000000046904001B0000004A
:100C7000A00000001B1904001D000000AA000000D5
:100C800058CF030021000000B40000003A8B03009D
:100C900024000000BE000000494C030027000000B3
:100CA000C80000001A1203002B000000D200000050
:100CB0004ADC02002F000000DC0000007DAA0200D8
:100CC00033000000E6000000637C020037000000F3
:100CD000F0000000AE5102003C000000FA000000ED
:100CE0001A2A020041000000040100006905020008
:100CF000460000000E0100005FE301004C00000010
:100D000018010000C8C301005200000022010000C9
:100D100073A60100580000002C010000348B010074
:100D20005F00000036010000E17101006600000074
:100D300040010000565A01006E0000004A01000008
:100D40006F44010076000000540100000D300100E6
:100D50007E0000005E010000131D010087000000FE
:100D600068010000660B01009000000072010000A5
:100D7000EDFA00009A0000007C01000091EB0000F9
:100D8000A4000000860100003EDD0000AF0000006E
:100D900090010000E0CF0000BA0000009A010000BE
:100DA00066C30000C6000000A4010000BFB7000039
:100DB000D3000000AE010000DCAC0000E000000049
:100DC000B8010000AFA20000EE000000C201000068
:100DD0002B990000FC000000CC01000044900000B2
:100DE0000C010000D6010000EF8700001B0100008D
:100DF000E0010000228000002C010000EA01000058
:100E0000D47800003D010000F4010000FC710000F6
:100E10004F010000FE010000916B00006201000024
:100E2000080200008D65000076010000120200003B
:100E3000E85F00008B0100001C0200009C5A0000CB
:100E4000A001000026020000A3550000B60100002A
:100E500030020000F8500000CD0100003A0200000E
:100E6000944C0000E50100004402000075480000B9
:100E7000FE0100004E020000944400001702000032
:100E800058020000EE400000320200006202000042
:100E9000803D00004D0200006C020000453A000059
:100EA00069020000760200003A3700008702000065
:100EB000800200005D340000A50200008A020000EC
:100EC000AA310000C4020000940200001E2F00009E
:100ED000E40200009E020000B82C000005030000A0
:100EE000A8020000752A000026030000B2020000DC
:100EF0005228000049030000BC0200004E260000FA
:100F00006C030000C602000067240000900300008C
:100F1000D00200009B220000B5030000DA020000AE
:100F2000E8200000DB030000E40200004D1F000089
:100F300002040000EE020000C91D000029040000A8
:100F4000F8020000591C00005104000002030000D8
:100F5000FD1A00007A0400000C030000B419000020
:100F6000A4040000160300007D180000CD0400005A
:100F70002003000056170000F80400002A030000B8
:100F80003F16000023050000340300003615000062
:100F90004F0500003E0300003B1400007B050000ED
:100FA000480300004D130000A80500005203000094
:100FB0006B120000D50500005C03000095110000D5
:100FC0000206000066030000CA1000002F060000A1
:100FD00070030000091000005D0600007A030000A5
:100FE000520F00008B06000084030000A40E0000D6
:100FF000B90600008E030000FF0D0000E8060000A7
:1010000098030000620D000016070000A203000014
:10101000CD0C000044070000AC0300003F0C0000B2
:1010200072070000B6030000B80B0000A007000024
:10103000C0030000380B0000CE070000CA03000008
:10104000BD0A0000FC070000D4030000490A0000AC
:101050002A080000DE030000DA090000570800003B
:10106000E80300007109000084080000F20300009A
:101070000C090000B1080000FC030000AC080000EF
:10108000DD08000006040000510800000909000006
:1010900010040000FA070000350900001A040000DF
:1010A000A7070000600900002404000058070000A2
:1010B0008A0900002E0400000C070000B40900009B
:1010C00038040000C4060000DE09000042040000ED
:1010D0007F060000070A00004C0400003D060000E7
:1010E0002F0A000056040000FF050000560A000009
:1010F00060040000C30500007D0A00006A040000CF
:1011000089050000A40A00007404000053050000D3
:10111000CA0A00007E0400001E050000EF0A00005D
:1011200088040000EC040000130B0000920400008F
:10113000BC040000370B00009C0400008E0400007B
:101140005A0B0000A6040000630400007C0B0000A2
:10115000B0040000390400009E0B0000BA04000037
:1011600010040000BE0B0000C4040000EA030000ED
:10117000DF0B0000CE040000C5030000FE0B0000E2
:10118000D8040000A20300001D0C0000E2040000CF
:10119000800300003B0C0000EC0400005F03000033
:1011A000580C0000F604000040030000750C00001D
:1011B0000005000023030000910C00000A05000058
:1011C00006030000AC0C000014050000EB02000058
:1011D000C70C00001E050000D0020000E00C00005B
:1011E00028050000B7020000FA0C000032050000DC
:1011F0009F020000120D00003C0500008802000064
:101200002A0D00004605000071020000420D00009A
:10121000500500005C020000580D00005A05000057
:10122000470200006E0D000064050000330200005C
:10123000840D00006E05000020020000990D0000E2
:10124000780500000E020000AD0D000082050000D0
:10125000FC010000C10D00008C050000EC01000045
:10126000D40D000096050000DB010000E70D000032
:10127000A0050000CC010000F90D0000AA05000047
:10128000BD0100000B0E0000B4050000AE0100001F
:101290001C0E0000BE050000A00100002D0E000085
:1012A000C8050000930100003D0E0000D2050000BB
:1012B000860100004D0E0000DC05000079010000F1
:1012C0005C0E0000E60500006E0100006B0E0000E1
:1012D000F005000062010000790E0000FA05000030
:1012E00057010000870E0000040600004C010000BA
:1012F000950E00000E06000042010000A20E000044
:101300001806000038010000AF0E000022060000A1
:101310002E010000BB0E00002C060000250100007D
:10132000C70E0000360600001C010000D30E0000AE
:101330004006000013010000DE0E00004A06000017
:101340000B010000E90E000054060000030100003C
:10135000F40E00005E060000FB000000FE0E000020
:1013600068060000F4000000080F0000720600008C
:10137000ED000000120F00007C060000E6000000F7
:101380001C0F000086060000DF000000250F000093
:1013900090060000D90000002E0F00009A06000001
:1013A000D2000000360F0000A4060000CC000000B0
:1013B0003F0F0000AE060000C6000000470F00000F
:1013C000B8060000C10000004F0F0000C206000078
:1013D000BB000000570F0000CC060000B600000064
:1013E0005E0F0000D6060000B1000000650F00008F
:1013F000E0060000AC0000006D0F0000EA060000EF
:10140000A7000000730F0000F4060000A200000017
:101410007A0F0000FE0600009E000000800F000012
:10142000080700009A000000860F00001207000065
:10143000950000008D0F00001C07000091000000C7
:10144000930F0000260700008D000000980F000099
:10145000300700008A0000009E0F00003A070000DD
:1014600086000000A30F0000440700008200000077
:10147000A80F00004E0700007F000000AE0F000024
:10148000580700007C000000B20F00006207000057
:1014900078000000B70F00006C0700007500000026
:1014A000BC0F00007607000072000000C10F0000B2
:1014B000800700006F000000C50F00008A070000D1
:1014C0006C000000C90F00009407000069000000D4
:1014D000CD0F00009E07000067000000D10F000044
:1014E000A807000064000000D50F0000B20700004C
:1014F00062000000D90F0000BC0700005F00000080
:10150000DD0F0000C60700005D000000E00F0000D6
:10151000D00700005A000000E40F0000DA070000C6
:1015200058000000E70F0000E4070000560000002C
:10153000EB0F0000EE07000054000000EE0F00006B
:10154000F807000052000000F10F00000208000040
:1015500050000000F40F00000C0800004E000000D6
:10156000F70F0000160800004C000000FA0F000002
:10157000200800004A000000FD0F00002A080000BB
:1015800048000000FF0F0000340800004700000082
:1015900002100000000000002110000042200000A6
:1015A0006330000084400000A5500000C6600000C9
:1015B000E770000008810000299100004AA10000A6
:1015C0006BB100008CC10000ADD10000CEE1000085
:1015D000EFF1000031120000100200007332000031
:1015E00052220000B552000094420000F772000041
:1015F000D662000039930000188300007BB300001E
:101600005AA30000BDD300009CC30000FFF30000FC
:10161000DEE30000622400004334000020040000E8
:1016200001140000E6640000C7740000A444000038
:10163000855400006AA500004BB500002885000015
:1016400009950000EEE50000CFF50000ACC50000F4
:101650008DD50000533600007226000011160000E0
:1016600030060000D7760000F666000095560000B0
:10167000B44600005BB700007AA70000199700008D
:1016800038870000DFF70000FEE700009DD700006C
:10169000BCC70000C4480000E55800008668000090
:1016A000A778000040080000611800000228000030
:1016B00023380000CCC90000EDD900008EE90000FD
:1016C000AFF9000048890000699900000AA90000EC
:1016D0002BB90000F55A0000D44A0000B77A000088
:1016E000966A0000711A0000500A0000333A0000A8
:1016F000122A0000FDDB0000DCCB0000BFFB000075
:101700009EEB0000799B0000588B00003BBB000063
:101710001AAB0000A66C0000877C0000E44C0000BF
:10172000C55C0000222C0000033C0000600C00009F
:10173000411C0000AEED00008FFD0000ECCD00006C
:10174000CDDD00002AAD00000BBD0000688D00005B
:10175000499D0000977E0000B66E0000D55E000037
:10176000F44E0000133E0000322E0000511E000017
:10177000700E00009FFF0000BEEF0000DDDF0000E4
:10178000FCCF00001BBF00003AAF0000599F0000D3
:10179000788F000088910000A9810000CAB1000084
:1017A000EBA100000CD100002DC100004EF10000A3
:1017B0006FE1000080100000A1000000C2300000B6
:1017C000E3200000045000002540000046700000A7
:1017D00067600000B983000098930000FBA300003D
:1017E000DAB300003DC300001CD300007FE300001B
:1017F0005EF30000B102000090120000F32200002E
:10180000D23200003542000014520000776200001E
:1018100056720000EAB50000CBA50000A8950000B4
:10182000898500006EF500004FE500002CD5000012
:101830000DC50000E2340000C3240000A014000025
:101840008104000066740000476400002454000016
:1018500005440000DBA70000FAB7000099870000EC
:10186000B89700005FE700007EF700001DC700008A
:101870003CD70000D3260000F2360000910600009D
:10188000B01600005766000076760000154600008E
:10189000345600004CD900006DC900000EF900005C
:1018A0002FE90000C8990000E98900008AB900000A
:1018B000ABA900004458000065480000067800000D
:1018C00027680000C0180000E1080000823800000E
:1018D000A32800007DCB00005CDB00003FEB000094
:1018E0001EFB0000F98B0000D89B0000BBAB000082
:1018F0009ABB0000754A0000545A0000376A000085
:10190000167A0000F10A0000D01A0000B32A000085
:10191000923A00002EFD00000FED00006CDD00008B
:101920004DCD0000AABD00008BAD0000E89D000079
:10193000C98D0000267C0000076C0000645C00007C
:10194000454C0000A23C0000832C0000E01C00007D
:10195000C10C00001FEF00003EFF00005DCF000043
:101960007CDF00009BAF0000BABF0000D98F0000F1
:10197000F89F0000176E0000367E0000554E0000F4
:10198000745E0000932E0000B23E0000D10E0000F5
:10199000F01E0000000000000000000000005F00DA
:1019A000000000000007000700000000147F147F03
:1019B00014000000242A7F2A120000002313086468
:1019C0006200000036495522400000000005030077
:1019D00000000000001C2241000000000041221C09
:1019E0000000000014083E081400000008083E082B
:1019F000080000000050300000000000080808083F
:101A000008000000006060000000000020100804D2
:101A1000020000003E4141413E00000000427F4084
:101A20000000000042615149460000002141454B41
:101A3000310000001814127F1000000027454545B2
:101A4000390000003C4A4949300000000171090595
:101A5000030000003649494936000000064949297B
:101A60001E00000000003636000000000056360060
:101A700000000000081C3E7F000000001414141435
:101A800014000000007F3E1C080000000201510904
:101A900006000000324979413E0000007E1111111C
:101AA0007E0000007F494949360000003E41414127
:101AB000220000007F4141221C0000007F4949496B
:101AC000410000007F090909010000003E41494929
:101AD0003A0000007F0808087F00000000417F41B5
:101AE000000000002040413F010000007F08142258
:101AF000410000007F404040400000007F020C0297
:101B00007F0000007F0408107F0000003E4141413B
:101B10003E0000007F090909060000003E415121F6
:101B20005E0000007F091929460000004649494926
:101B30003100000001017F01010000003F404040F2
:101B40003F0000001F2040201F0000003F40704069
:101B50003F000000631408146300000007087008C9
:101B6000070000006151494543000000007F4141EA
:101B70000000000002040810200000000041417F26
:101B80000000000004020102040000004040404048
:101B900040000000000102000000000020545454E6
:101BA000780000007F444444380000003844444436
:101BB00020000000384444487F000000385454544A
:101BC00018000000087E09010200000018A4A4A467
:101BD0007C0000007F0804047800000000447D4081
:101BE000000000002040443D000000007F10284419
:101BF0000000000000417F40000000007C04180449
